:020000040000FA
:1000000040450020991E0000CD670000851E0000BD
:10001000851E0000851E0000851E000000000000F7
:10002000000000000000000000000000991F000018
:10003000851E000000000000851E0000851E0000D7
:100040005D2100005D2100005D2100005D210000B8
:100050005D2100005D2100005D2100005D210000A8
:100060005D2100005D2100005D2100005D21000098
:100070005D2100005D2100005D2100005D21000088
:100080005D2100005D2100005D2100005D21000078
:100090005D2100005D2100005D2100005D21000068
:1000A0005D2100005D2100005D2100005D21000058
:1000B0005D2100005D2100005D2100005D21000048
:1000C0005D2100005D2100005D2100005D21000038
:1000D0005D2100005D2100005D2100005D21000028
:1000E0005D2100005D2100005D2100005D21000018
:1000F0005D2100005D2100005D2100005D21000008
:1001000053B94AB9002908BF00281CBF4FF0FF317E
:100110004FF0FF3000F00CB8ADF1080C6DE904CEE3
:1001200000F008F8DDF804E0DDE9022304B07047D0
:10013000704700BF2DE9F04786468C460846089E6A
:10014000154674461946002B40F0C2808542B2FA2B
:1001500082F245D94AB1C2F1200300FA02FC2EFA1C
:1001600003F3954043EA0C0C94404FEA154EA8B2B5
:10017000BCFBFEF8230C0EFB18CC08FB00F943EA8D
:100180000C43994528D9EB1808F1FF3704D299455B
:1001900002D9A8F102072B44A3EB0903A4B2B3FBD5
:1001A000FEFC0EFB1C330CFB00F044EA0344A042AF
:1001B00014D92C190CF1FF3304D2A04202D9ACF1AE
:1001C00002032C44241A43EA07401EB1D440002302
:1001D00034607360BDE8F0874746DDE76346F1E7CA
:1001E00092BB431B01214FEA154EAFB2B3FBFEFC9D
:1001F000200C0EFB1C330CFB07F840EA0343984528
:1002000062D9EB180CF1FF3004D2984502D9ACF159
:1002100002002B44A3EB0803A4B2B3FBFEFC0EFBCD
:100220001C330CFB07F744EA0344A7424ED92C19B0
:100230000CF1FF3304D2A74202D9ACF102032C44E3
:10024000E41B43EA0040C0E7C2F1200320FA03F1B7
:10025000954090402EFA03F303434FEA154EAFB298
:10026000B1FBFEFC0EFB1C10190C0CFB07F841EA5D
:100270000041884504FA02F422D969180CF1FF30D4
:1002800004D2884502D9ACF102002944A1EB08014F
:100290009BB2B1FBFEFC0EFB1C110CFB07F743EA03
:1002A00001439F420ED9EB180CF1FF3104D29F425B
:1002B00002D9ACF102012B44DB1B41EA004192E779
:1002C0006046E3E76146F7E76046A3E76346B7E7C2
:1002D000834206D916B9002108467BE7C6E900E04B
:1002E000F9E7B3FA83F78FB9834201D3724508D88F
:1002F000BEEB020460EB030301209C461EB9002103
:1003000068E73846FAE7C6E9004CF8E7C7F1200C81
:10031000BB4022FA0CF41C432EFA0CF120FA0CF329
:10032000B84001434FEA14490EFA07F5B3FBF9F858
:100330001FFA84FE09FB18300B0C08FB0EFA43EA87
:1003400000439A4502FA07F240D9E31808F1FF305A
:1003500004D29A4502D9A8F102002344A3EB0A0370
:1003600089B2B3FBF9F809FB183308FB0EFE41EA2A
:1003700003418E452CD9611808F1FF3304D28E4514
:1003800002D9A8F10203214443EA0040A0FB0298ED
:10039000A1EB0E014145CE46434602D306D14D4561
:1003A00004D2B9EB020E68EB04030138002EA6D08C
:1003B000B5EB0E0261EB030101FA0CFC22FA07F324
:1003C0004CEA0303F940C6E9003198E74046C5E727
:1003D0004346D9E7F0B52E4B2E4AC3F800262E48E7
:1003E000C3F8042685B0C3F808264921C3F80C26B3
:1003F000C3F81026C3F81426C3F81826C3F81C2621
:1004000006F05BF905F030FD01A800F09DFC234BE0
:100410001B68834204D02248452106F04EF9FEE7CE
:10042000039A2048492106F048F91F48492106F05F
:1004300044F94FF44041002006F08CFC044620B102
:100440001A48452106F039F9FEE769469DF808008B
:1004500000F030F8009B039D1D44019B1E8902F0B3
:10046000FDFFAF1900F0CCFF00F0A0FF01F050FD40
:10047000AB5983F3088884F31488BFF36F8FBFF3FD
:100480006F8F7B6898470A48452106F016F9FEE70A
:10049000000001403546526E04770000F80100204C
:1004A0001D770000407700006F7700009477000010
:1004B000C777000008B5024638B10548002345213A
:1004C00006F0FBF86FF0150008BD0860FCE700BF00
:1004D000EA77000021B1012906D06FF015007047BE
:1004E000044B53F830007047024B03EBC0035868CD
:1004F000704700BF687300002DE9F04F7E4FDDB0FC
:10050000DDE9688914461D46DDF8A8B13E6800F0B3
:1005100017FF7A4B0122C3F800253CA804F0C8FB62
:10052000B8F1000F07D0B9F1000F04DD4A4641468B
:100530003CA805F0BDFF23896289D4F80CA01344C0
:100540009A444FF00008C24551D80FA93CA804F0C6
:1005500021FC6A4B0022C3F80025C3F80025BBF13B
:10056000000F04D020220FA9584606F08FF900236F
:1005700000932A464FF6FF73214609A805F075FC43
:100580000390002844D128460E9C00F079F984425B
:100590003ED8DFF870B1DFF864914FF0FF340DF111
:1005A0001E0307AA08A909A805F0ADFC00282FDB47
:1005B00040F09B80BDF81EA0BAF1100F31D1BDF8FC
:1005C0001C80B8F1200F23D1089943463CAA284645
:1005D00006F081F8E0B942463CA90FA805F00BFDF2
:1005E000474B1B68834213D101230393D7E7679BD3
:1005F000669AAAEB0809994528BF99464B46414699
:10060000284606F068F828B13C4B0022C3F80025C4
:100610003E686DE066994A463CA805F049FFC8442B
:1006200091E7BAF1010F3FD1BDF81C30202BEFD874
:1006300008993CAA284606F04EF804460028E7D15F
:100640009DF81C300493202B0AD8DBF80030DFF82B
:10065000B8800593059B9C4205DB0023C9F8003553
:100660004FF0FF349BE700F06BFEC9F800A51FA810
:1006700004F01EFBD8F8042058F8081B12681FA8C5
:1006800005F016FF17A91FA804F084FB0022C9F883
:100690000025049A3CA917A806F0E8F810B9C9F893
:1006A00000057CE70134D5E7BAF1220F7FF477AF7C
:1006B000631C3FF474AFDBF80030A342D0DDBDF81B
:1006C0001C30802BA4D808993CAA284606F003F8D1
:1006D00000289DD1E4B2BDF81C3000943CAA202132
:1006E0000FA800F013F80646BAE7039B002B8FD043
:1006F00030465DB0BDE8F08F0400002000A002503D
:10070000F801002070730000747300002DE9F047B9
:1007100096B016461D469DF87820374BDFF8E880E6
:1007200053F83210019103EBC20307465B68D8F817
:100730000090186802AA0144302301A805F046FE83
:10074000002851D1DDE901431C4403AA06AB214630
:1007500001A805F063FE002846D1049A072A43D178
:100760002649059806F082F800283DD1079A082A04
:100770003AD12349089806F079F8A8BB02AA214685
:1007800001A805F037FE78BBDDE901A30AEB0302FF
:10079000944229D1412B27D13544302303AA29463D
:1007A00002A8029605F012FEE0B9DDE90232134418
:1007B0009D4217D32A4602A906A805F0F0FB88B986
:1007C0002A4602A90EA805F0EAFB58B99AF80030AB
:1007D000042B07D1202306AA0AF10101384600F0B4
:1007E000C7FD28B1D8F80090484616B0BDE8F0879C
:1007F000044BD3F80090F7E77473000019780000F9
:1008000010780000F801002004000020094A0B784D
:10081000400052F820108B4209D0013052F82000DD
:10082000834214BF4FF0FF304FF4C07070474FF455
:10083000C07070477C7300001FB50F4B13F8300079
:100840000C4601F075F950B92068816810236A469A
:10085000103905F040FF28B1206805F03BFF4FF04C
:10086000FF3006E005491022684605F0FFFF00282A
:10087000F2D104B010BD00BF7C730000F47600001C
:1008800013B5044605F0BEFB6A460146204605F056
:10089000D2FA30B10448452105F00FFF002002B024
:1008A00010BD0098FBE700BF217800002DE9F04162
:1008B000364B88B0064600200D461C68FFF70AFE3E
:1008C00006A9C0B201F034F9002858D12946FFF733
:1008D00001FE2C2407A9C0B204FB056401F028F92D
:1008E000002833D02C276F4306EB0708069BD8F867
:1008F000101011F0100138D14FF480720192244A87
:100900000092CDE90311224602910846FFF7F4FD5B
:100910000446204BF25906989A420CD1D8F80C2084
:10092000B8F808309B1806D28268934203D21A4B5B
:100930001B68A34220D035B38268002105F0F5FE84
:10094000164A1748452105F0B8FE13E0079805F050
:1009500009FF0746079805F0BDFE631EE21C13F869
:10096000011FB942BED19342F9D11DB1069930465B
:1009700005F032FC0B4B1C68069805F0ABFE2046D8
:1009800008B0BDE8F081084ADBE700BF04000020A2
:10099000C40F00203DB8F396F801002064780000F1
:1009A0006E780000000000205C7800007FB50D46E6
:1009B000044600212846CDE9021105F0CCFB28B3FE
:1009C0002368194EB34203D103AA204605F058FB11
:1009D000E36AB34204D102AA0121204605F050FB8C
:1009E000DDE90232934288BF0393039BAB60039A15
:1009F0002946204600F0A2FB0C4B1A68002A03DDB2
:100A00000B48572105F059FE04B070BD01A9FFF74E
:100A100013FF019805F1080105F0FFFAAB68019892
:100A2000039305F057FEE2E73DB8F3965C0E002015
:100A3000967800002DE9F84FDFF878B01B4C1C4D7C
:100A4000884691469A4600260B9B9E4201D3002081
:100A50000FE00B9B174A9F1BB7F5806F28BF4FF421
:100A600080673B4606EB0A01404605F034FE10B1B4
:100A70000120BDE8F88F0A993B465A46711848464E
:100A800005F03EFE0028F3D1C4F800563E44C4F8F9
:100A90000456C4F80856C4F80C56C4F81056C4F8E6
:100AA0001456C4F81856C4F81C56CDE7000001408F
:100AB0003546526EFC090020F0B5994B43620E4654
:100AC000984B0365002189B004460846FFF702FDF4
:100AD00004F120010546C0B201F02AF80346E8B946
:100AE0000121FFF7F7FC04F14C010546C0B201F00B
:100AF0001FF80346E0B9204605F003FB0546C8B9D8
:100B000000221146204605F0A5FA054660B3864846
:100B10000022572105F0D1FD01239CE00022CDE900
:100B20000023824800232A46452105F0C6FDFEE742
:100B30000122F4E77E488022572105F0BEFD012303
:100B40009D4284F85830DBD194F858308DF8173036
:100B5000042B00F28380012B00F2878000F09A8042
:100B6000FF2384F8583095E0204600F0FFF9002874
:100B7000D2D004A805F0E6FA0146204605F081FB34
:100B800018B16C482A465721C4E704A805F0E3FAD7
:100B900080F0010104AAC9B2204605F05BFA0246C2
:100BA0000028B4D104A805F0D6FA054660BB04A914
:100BB0002046FFF7FBFE9DF8173084F85830033BC2
:100BC000012B06D8284600F0E5F810B1FF2384F881
:100BD00058309DF81730023B022B0BD8002000F054
:100BE000C3F838B1FF2384F858305348452105F045
:100BF00064FDFEE794F85830FF2BF6D004AA0021DC
:100C0000204605F027FA87E79DF81770012F17D1C6
:100C1000104602F0CFFC831E022B05460DD8394644
:100C20002046FFF743FE454B1B68984205D0444BD6
:100C30001D68A84214BF0525012584F8585083E794
:100C400001212046FFF732FE3C4B1B6898420CBF47
:100C50009DF81730052384F8583075E7052B7FF48D
:100C60007FAF002000F096F811E004A92046FFF7BE
:100C70009DFE94F85830DA1E012A14D8002000F0A6
:100C800089F800287FF46CAF002000F06DF8002890
:100C90007FF466AF94F85830FF2B07D126484521E2
:100CA00005F00BFDFEE7022BF4D1EDE70022012B4E
:100CB000244D039214D01146204605F0CBF978B1AB
:100CC0002D68102200210DEB020005F0EAFDE06C1A
:100CD00005F000FD206A05F0FDFC284609B0F0BDD6
:100CE00000212046FFF7E2FD144F3B689842E7D110
:100CF0002B689842E4D0124B1B689842E0D0039BCB
:100D000001330393039B012B00D0FEE7206A05F01B
:100D100090F83071236A5B6834603D68B360D0E757
:100D2000FC050020FC01002054790000C57800007B
:100D30001279000080790000AA790000F8010020F3
:100D4000000000200400002038B5064D0446602253
:100D50000021284605F0A5FD21462846FFF7ACFEF8
:100D600038BD00BFFC0D002013B5094B01A913F8D5
:100D7000300000F0DDFE48B9019806F0A8F80446FE
:100D8000019805F0A7FC204602B010BD0124FAE747
:100D9000847300001FB50F4B01A913F8300000F059
:100DA000C7FEA8B9019802A902F0AEFB044668B9D3
:100DB0009DF80B30032B03D1019806F056F804463A
:100DC000019805F087FC204604B010BD0124F7E728
:100DD0000124F8E7847300002DE9F34106460C4630
:100DE00017461D460BB9002628E0184605F0B3F952
:100DF0000028F8D16946FFF71FFD009838B9012493
:100E0000009805F067FC204602B0BDE8F08101A91A
:100E100005F003F90028F2D1009805F05BFC30469C
:100E2000019905F06AFA736A5E686B79012B21D12A
:100E3000002CD8D12B68834298BF00262146002081
:100E4000FFF748FB6946C0B200F072FE0028D6D119
:100E5000009820233A46314605F03DFC0446002820
:100E6000CDD1002DCCD03C680D4BE41A18BF4FF00B
:100E7000FF34C5E7022BB6D12B68012B05D983427D
:100E8000B1D8B4FA84F46409ADE7ACD1002CD5D064
:100E9000012CA8D12C79023C18BF0124A3E700BF84
:100EA0003DB8F3962DE9F04F074685B00C46014654
:100EB00000201646FFF7AAFC051E50DB3846E46DFD
:100EC00005F0A0F85FFA84F96B1E09FB03084FF0E8
:100ED000000A4FF0010B4FF0FF349DB9BAF1010F3A
:100EE00003DD2148452105F0E8FB631C06D07F2C7B
:100EF0002ADC013440F201133460B380284605B087
:100F0000BDE8F08F6B1E00930DF10F0201234146E7
:100F1000384605F0E0FB031E019322DB01220DF1B0
:100F20000F01384605F03CFF019B40B15B4501D005
:100F30000AF1010A009DA8EB09089B46CDE7B4F130
:100F4000FF3F08BF2C46F5E70223803C7371631016
:100F500004F001040133013433603471CEE7072516
:100F6000CCE70125CAE700BFB679000038B5816A31
:100F7000426D914208D0531C8B4205D01348572133
:100F800005F09BFB002038BD80291CD91048572153
:100F9000F6E7446A056D04EBC30405EBC30564681A
:100FA0006D68AC4202D00B485721E9E701339A4201
:100FB000EFD1914205D9436A03EBC2035B68A342B8
:100FC000F1D10120DFE700231C46F0E7D9790000CA
:100FD000117A0000407A000000B589B004A902200F
:100FE00005F050FF9DF81020012A41D0254B2649DD
:100FF000032A08BF0B469DF8132002929DF8122089
:1010000001929DF81120214800924921204A05F0C3
:1010100054FB06A9052005F035FF9DF81820012A8C
:1010200028D0184B1849032A08BF0B469DF81B20EF
:1010300002929DF81A2001929DF8192000921348FF
:10104000144A492105F039FB9DF81030012B13D1CA
:101050009DF81230032B0FD19DF81830012B0BD0C7
:101060000D48492105F029FB022009B05DF804FB79
:101070000A4BC0E7094BD9E70948492105F01DFB98
:101080000020F2E76C7A0000757A0000897A00008F
:101090007B7A0000CA7A0000DA7A0000707A0000D9
:1010A000F97A000070B54B6814461E4A03F0FF231E
:1010B000934286B006460D462FD10B68012B2CD1EA
:1010C00004A9204602F020FA9DF81020012A26D01B
:1010D000154B1649032A08BF0B469DF813200292B0
:1010E0009DF8122001929DF8112000921048114A9B
:1010F000492105F0E2FA9DF81030032B0DD121466D
:10110000304605F069F8204605F0AFFEA968204694
:1011100004F091FF204602F0D7F906B070BD064BEF
:10112000DBE700BF000100046C7A0000757A000064
:10113000897A0000CA7A0000707A00002DE9F04F29
:10114000164689B005460C467448492105F0B5FAA3
:101150003146284605F0D1F86B6A824620465E6823
:1011600004F0F9FFE8B1E86D04F047FFAF6A00232F
:10117000013F3344834201D2013FFAE7BA4510D31D
:101180006748572105F099FA07FB06F365480AFB03
:101190000662572105F091FA0123E37109B0BDE819
:1011A000F08F06A9022000F0C3FC07A9052000F07B
:1011B000BFFC079A21462846FFF774FF6379012B8D
:1011C0004BD1DFF864B1574641E02268C2F1010318
:1011D00053449F423AD86B6A196853F8370003EBBF
:1011E000C703012A53F8083CA3EB0103A0EB010954
:1011F000049311D1079B0393E368022B08D0414667
:10120000284604F0E9FF22464146284605F01AF830
:101210000399284604F0E0FF32464946404604F070
:10122000D9FF049B42464146CDE900962846FFF788
:1012300001FC2146284604F09BFF2368013323600C
:1012400020B1DBF800300133CBF80030013FDDF88E
:101250001880002FB9D10123236002236371012775
:10126000BA45DDF8189006D2484605F033FA0798DB
:1012700005F030FA92E723689F424DD36A6ADDF8A1
:101280001CB052F837100491FB00083B1168039121
:10129000D1582A6DD0581368A0EB03082379012B8D
:1012A00038D1039B3246C91A4846059104F092FF93
:1012B0000599009143464A46594601962846FFF74C
:1012C000B9FB2146284604F053FF0223237118B1CD
:1012D000154A13680133136032464146584604F0FC
:1012E00079FFDDE9032349469B1ACDE900865A467A
:1012F0002846FFF79FFB2146284604F039FF236864
:10130000013323600123237130B1074A136801338D
:10131000136001E0022BDFD00137A1E7107B000052
:10132000397B0000687B00005C0E00200A4619B182
:10133000024B00211B681847704700BF08000020BF
:1013400070B5094D2B780BB1002070BD074C0126FC
:10135000C4F8006503F04EFD18B92E70C4F80005FE
:10136000F2E74FF0FF30F0E7C410002000A0025079
:101370002DE9F041DFF83080ACB01F4606460C4640
:101380001546FFF7DDFF0123C8F800352A4633462E
:101390000097214603A805F070FE0023C8F8003529
:1013A0002CB0BDE8F08100BF00A00250BFF36F8FEA
:1013B00072B6124B4FF0FF32C3F88020C3F884207E
:1013C000C3F88820C3F88C20C3F89020C3F8942079
:1013D000C3F89820C3F89C20C3F88021C3F8842167
:1013E000C3F88821C3F88C21C3F89021C3F8942155
:1013F000C3F89821C3F89C21704700BF00E100E0CA
:10140000164A4FF0FF3301215160C2F84833C2F849
:10141000083302F5C0425160C2F84833C2F80833BD
:1014200002F598325160C2F84833C2F80833A2F589
:1014300008320021C2F80015C2F8083302F518324C
:10144000C2F80015C2F80833A2F51042C2F80835F8
:101450004FF08042C2F80833704700BF00B0004030
:10146000014B1B68184700BF0C000020014B18609F
:10147000704700BF0C00002007B50B460021024654
:101480000091034800F014F903B05DF804FB00BFBD
:10149000611400002DE9F047058B044628079046AB
:1014A00011D4022905F0070540F0CD80204605F053
:1014B00029F878B10138218B042811D8DFE800F031
:1014C000C3106D85950001290CBF45F0100545F04E
:1014D0002005258388F31188BFF36F8FBDE8F0875F
:1014E00001F0070AAA4500F0A6800027B9463E464B
:1014F000A368002B00F0BD8041F00801218388F330
:101500001188BFF36F8FA168002900F0BB800D68C0
:10151000002900F0B780D1F80480334652462046B7
:10152000C047002D76D02B6829461D46F0E701F014
:1015300007035A1F012A1BD8002221F00701062B9E
:10154000276889B2C4E9002209D13B4603E0628BD7
:10155000013262831B68002BF9D141F00201218323
:10156000204604F0CFFF00287BD041F0200177E037
:10157000042B0AD121F0070189B22183204604F00F
:10158000C1FF10B141F020012183218B01F0070A36
:10159000AA4550D00027B946AAE7236921F00701E0
:1015A00041F00601062DD3F8009021832DD1B9F129
:1015B000000F40D041F00801218388F31188BFF368
:1015C0006F8F3A492046C84729E021F00701236977
:1015D00041F0040189B2042DD3F804902183E6D0B0
:1015E00000273E464FF0040A82E721F007012369F5
:1015F00041F0050189B2052DD3F808902183D6D09A
:1016000000273E464FF0050A72E700273E464FF09E
:10161000060A6DE72B4687E7B9F1000FD1D14FF0ED
:101620002003EFF3118883F31288BFF36F8F238BAE
:1016300023F008032383258BEA062ED525F010031B
:10164000238305F007056669218B002EBFF66FAF77
:1016500000232768C4E9003321F0070141F00101AC
:101660002183218B01F0070AAA454FF000097FF47E
:101670003FAF002F9BD041F00801218388F31188F0
:10168000BFF36F8F002FC7D03D68394633465246AF
:10169000204604F063FF2F46F4E7AB067FF51AAF50
:1016A00025F02003238305F00705FFE68965000088
:1016B0002DE9F04F8DB01D46531E824601910393D4
:1016C0004FF00009039B5878252803F1010419D134
:1016D0001E4600204FF0FF38023603460290444673
:1016E00031780396392954D81F2914D8002900F0DD
:1016F000EE8101992520D04701993078D04709F132
:101700000209DFE7002800F0E2810199D04709F1E2
:1017100001090394D6E7A1F12002192AE9D801A70B
:1017200057F822F08D170000F3160000F3160000A2
:101730008D170000F31600000D180000F3160000CE
:10174000F3160000F3160000F3160000591800000D
:101750008D170000F31600006D1800001918000026
:10176000F316000027180000471800004718000073
:1017700047180000471800004718000047180000ED
:1017800047180000471800004718000008460136B7
:10179000A6E7582900F0EB80A1F16302D7B2172F1A
:1017A000A7D8172AA5D801A757F822F0151A0000C4
:1017B00093180000F3160000F3160000F316000063
:1017C0007318000093180000F3160000F3160000D1
:1017D00073180000F3160000F3160000F316000063
:1017E00049190000F3160000F3160000E919000083
:1017F000F316000093180000F3160000F316000023
:1018000049190000F3160000731800000199252003
:10181000D04709F1010955E7029A02F0FE0202924F
:101820004FF00008B3E7002C0DDAB8F1000F0DDA25
:10183000029A002A00F0438124EAE4740A2202FB9F
:101840000414303CA3E7B8F1000FF5DB0A2202FBD9
:101850000812A2F130089AE7B8F1000F55F8042BEE
:1018600080F22F81002A80F22E81544202220292BD
:101870008DE7682903D1682B06D1482387E76C29B7
:1018800002D16C2B00F02181002B7FF432AF0B468C
:101890007DE77A2B06D1752955F8046B14D14FF0EA
:1018A000000B0CE06C2BF6D04C2BF4D1073525F057
:1018B00007037529D3E9006B03F1080506D1202839
:1018C0003BD1854F013C09E04FEAE67BBBF1000FBD
:1018D000F5DA7642814F6BEB4B0B013C0DF12D039A
:1018E000059300230493304659460A220023FEF74D
:1018F00007FC059B303203F8012DB4460593049B89
:101900005A46BCF10A0F8B4672F1000203F1FF3117
:1019100006460491E7D2C3F1010B30330DEB030609
:10192000B8F1000FA6F104066DDA029BD9077DD449
:10193000A8EB0B03A4EB0B0413E02B280ABF684FA2
:10194000684F04F1FF34C9E770290FD155F8042B13
:101950000023FAB9634F644E053C6FF004034FF067
:10196000050B029A920770D4A04666E078216C2B92
:1019700003D155F8042B002308E04C2BF9D107358F
:1019800025F007031D465B6855F8082B232825D151
:10199000880621D5554F023C01F06001A1F1390BB9
:1019A0000DF12D0E002602F00F01092988BF5944C0
:1019B00030310EF8011D102A4FEA121141EA03716D
:1019C0004FEA131C73F1000306F1FF3008D2C6F191
:1019D000010B06F13003A1E7454FDCE7414FDBE7A0
:1019E00006460A466346DEE755F8046B304604F0C7
:1019F00036FFB8F1000F834602DB4045A8BFC3465F
:101A0000384F4FF00008A8EB0B03002B92DDA4EB3E
:101A10000804A6E755F8043B8DF81830314F013C17
:101A20004FF0FF334FF0010B06AE9AE7A046EAE70E
:101A3000029301992020D047029BB8F10108F7D505
:101A400024EAE472013C9144A41AB84606E00493E7
:101A500002920199D047029A049B9046424612F89E
:101A6000010B0028F3D11A46013A15D5002BACBF63
:101A7000C7EB03077F425B46013B15D5BBF1000F67
:101A8000A8BF5F444F442646013E14D5002CA8BF92
:101A90003F1907EB080915E60493029201993020DB
:101AA000D047049B029ADFE70293019916F8010BD5
:101AB000D047029BE0E701992020D047E4E70122CC
:101AC000D5E6904663E6144661E64C235FE6484659
:101AD0000DB0BDE8F08F00BFF67B0000F47B000086
:101AE000F87B0000B5790000007C0000FA7B000064
:101AF000FD7B000008B504464FF02002EFF3118390
:101B000082F31288BFF36F8F01F0A8FC204600F02B
:101B1000EDF9034804F0E9FC00F0FAFAFCE700BF35
:101B2000067C0000014B03600020704790730000AA
:101B300070B5114B1C680D46DCB1104B19680023C1
:101B40008B4202DB6FF0010070BD224612F8106B71
:101B5000864202D001331446F2E7E06810B96FF014
:101B60001200F1E705F064FA0028F8D02C6000209C
:101B7000EAE76FF00C00E7E7100000209073000028
:101B800070B588B005460C46C0B269461646FFF7E8
:101B9000CFFF00281BDB0098C8B14368029383681D
:101BA00022680195CDE903360023CDE9062305938C
:101BB000C56804F08FFD6DB12846084901AA04F0FC
:101BC00068FF079808B9059B236008B070BD6FF0E7
:101BD0001500FAE76FF01200F7E700BF7367000027
:101BE000014802F0B7BD00BFF473000030BFFFF73B
:101BF000FDBF00BF704700BF70B5264B15469A6AFF
:101C000012F0100F9A6A14BF1124102412F0080F5A
:101C10009A6A18BF1224920706460AD5586B9A6A28
:101C2000140634D519B19A6A22F080029A621324FC
:101C300001E06FF01500174B9A6A12F0010F9A6AD3
:101C400018BF142412F0200F9A6A18BF1524D20668
:101C500002D49B6A9B070AD50E4B5B68190506D513
:101C6000314600F01FFA10B180F309880224094BB5
:101C70009A6A920642BF5A6A22F400525A629A6ADB
:101C800042F0FF029A6200232B70204670BD6FF075
:101C90001500CCE700ED00E0134B9A6A12F0007FCC
:101CA0009A6A14BF1E201D2012F0807F9A6A18BF06
:101CB0001F2012F4002F9A6A18BF212012F4802FDF
:101CC0009A6A18BF222012F4003F9A6A18BF232094
:101CD00012F4803F9A6A6FEA02426FEA12429A62F5
:101CE00018BF2420704700BF00ED00E010B5194B6D
:101CF0000246986A9C6A10F4805F14BF1720162071
:101D000014F4006F9C6A18BF1820A40509D5986BBD
:101D1000986A000404D51AB19A6A22F400429A62C1
:101D200019200C4B9A6A12F4806F9A6A18BF1A2015
:101D3000D2050CD49B6A13F4005F18BF1C20054A1F
:101D4000936A43F47F43936200230B7010BD1B2002
:101D5000F5E700BF00ED00E070B5454B5B688AB069
:101D60000546C3F30803002686F31188BFF36F8F7F
:101D700002F07F40B0F17F4F11D102F00C00082833
:101D80000DD010074CBF0D4601260022033B8DF8F5
:101D90000720032B05D8DFE803F01E5D615A3546A6
:101DA000F3E700249DF807309BB92022294602A8BA
:101DB00004F06CFD099B002E54D0C3F3080222B935
:101DC0006FEA53236FEA4323099302A9204604F0E4
:101DD000F7FC0AB070BD264BDA6A9107E1D4DA6AE3
:101DE000002ADEDBDA6A5200DBD55A69A96942F4BF
:101DF00080725A61BFF34F8FBFF36F8F5A6931F80A
:101E0000021C22F480725A61BFF34F8FBFF36F8FB1
:101E10004DF6027291420AD09A6AD2B24AB10DF1DD
:101E2000070201212846FFF7E7FE0446BAE72C68BF
:101E3000B8E79A6A12F47F4F05D00DF1070101202F
:101E4000FFF754FFF1E79B6AB3F5803FA9D3FFF793
:101E500023FFEAE70DF107020021E3E70DF1070197
:101E60000020EDE723F4FF7323F00103ACE700BF8C
:101E700000ED00E0024A536943F0100353617047DC
:101E800000ED00E0EFF30880EFF3098101B5724641
:101E9000FFF762FF01BD00BF002080F31488BFF38D
:101EA0006F8F00F05DFA00200D490860BFF34F8F7F
:101EB0000C4880F3088800F03DF8202080F311885A
:101EC00009484FF40461401880F30988EFF3148047
:101ED0000221084380F31488BFF36F8F00F0B4F839
:101EE00094ED00E04045002000150020BFF34F8F27
:101EF0000549064BCA6802F4E0621343CB60BFF3A6
:101F00004F8F00BFFDE700BF00ED00E00400FA05C1
:101F10000749D1F890200023C2F3072218469342C4
:101F200000DB7047C1F89830C1F8A0000133F6E734
:101F300000ED00E008B572B6002383F31388FFF7C5
:101F4000E7FF144B4FF0FF32C3F88020C3F8842022
:101F5000C3F88820C3F88C20C3F89020C3F89420DD
:101F6000C3F89820C3F89C20C3F88021C3F88421CB
:101F7000C3F88821C3F88C21C3F89021C3F89421B9
:101F8000C3F89821C3F89C2162B6BFF34F8FBFF30B
:101F90006F8F08BD00E100E01EF0040F0CBFEFF3EF
:101FA0000880EFF30980816911F8021C0229FFD033
:101FB00001B504F007FC01BD40B2002807DB044A6C
:101FC0004109012300F01F00834042F8213070478F
:101FD00000E100E040B200280CDB4309064900F0B4
:101FE0001F0020330122824041F82320BFF34F8F8E
:101FF000BFF36F8F704700BF00E100E0054B42095F
:1020000000F01F0053F82220012303FA00F01040D3
:10201000704700BF00E100E040B20028A8BF00F117
:10202000604001F10101B8BF064B4FEA4111ACBF5E
:1020300000F5614000F00F00C9B2B4BF195480F838
:102040000013704714ED00E0144A08B5144B22F059
:102050007F029A60BFF34F8FBFF36F8FD3F8882052
:1020600022F47002C3F88820D3F8882042F4A0023A
:10207000C3F888204FF04042C3F83422BFF34F8F9B
:10208000BFF36F8F0023E1EE103A02F003FA02F083
:1020900049FA00F057F802F009FA00BF000000000A
:1020A00000ED00E010F1160F074B08D0984208D35E
:1020B0004033834205D98B4203D9044870474033EB
:1020C000F9E70020704700BF401D0020801D002060
:1020D0000446084611461A460023E1EE103A084B22
:1020E000202583F3098863B64FF0000383F311883A
:1020F000BFF36F8FA04785F31188BFF36F8FFEE7A3
:1021000080450020014910220A60704710ED00E070
:1021100072B6404080F31188BFF36F8FBFF34F8FCB
:1021200030BF62B6BFF36F8F704700BF72B64940D1
:1021300081F31188BFF34F8F20BF80F3118862B6FF
:10214000704700BF044800232021C2180133302B00
:1021500082F80013F9D1704700E100E001B5EFF318
:102160000580A0F110004FEAC0000449014409C9EC
:102170009847BDE80140024908470000BC710000D3
:10218000F51B0000024B034A0348022100F030B85F
:102190000000042000000020FC730000084AC2F880
:1021A00098000B6823F01F03034343F01003C2F8A9
:1021B0009C308B6843F00103C2F8A030704700BF29
:1021C00000ED00E0044B0522C3F89420BFF34F8FCD
:1021D000BFF36F8F704700BF00ED00E0BFF35F8F6C
:1021E000024B0022C3F89420704700BF00ED00E0CE
:1021F00010B5034C0123227804F003FB207010BDBE
:10220000C5100020F0B5454D2C68082C85B000F2B3
:102210008280FFF7E3FF00200C2684420DD1404D61
:10222000404F2C706846FFF77DFC00240646A6420E
:102230000AD1FFF7C7FF00201CE0696806FB001108
:10224000FFF7ACFF0130E8E7009800EB04114FEA1C
:10225000041CCB683B40B3F5000F4AD00CD8B3F553
:10226000001F30D0B3F5800F38D0B3F5801F12D0E7
:102270006FF0150005B0F0BDB3F1807F42D0B3F12F
:10228000007FF5D150F80C3088684A6804F0A9FA4C
:1022900040F4802009E050F80C3088684A6804F067
:1022A000A0FA40F0885040F43020039028780728A6
:1022B000CDE90123DCD801A9FFF770FF2B780133AA
:1022C0002B700134B3E750F80C3088684A6804F08A
:1022D00088FA40F0885040F40020E6E750F80C30CF
:1022E00088684A6804F07DFA40F0007040F40030DD
:1022F000DBE750F80C3088684A6804F072FA40F066
:102300008270D2E750F80C3088684A6804F069FAA5
:1023100040F08870C9E74FF0FF30ABE7147400005D
:10232000C51000200000F0FF014B1860704700BF8F
:1023300014000020044A0123C2F840354FF08042C7
:102340000020C2F87835704700E0014020B1034B0F
:10235000800143F001031847704700BF607300001D
:1023600001F0C2B9084B70B5C31A0D4607499B105E
:10237000044659430648402204F0BBFA2B46014666
:102380002046BDE870401847740E0020B76DDBB6DC
:102390004471000073B50C4C0C4A4023041B00939D
:1023A0000D460B460A49A41061430646094804F04D
:1023B000CCFA011E05DA30462B4602B0BDE870406B
:1023C000184702B070BD00BF740E0020BB6900004A
:1023D000B76DDBB64471000010B54FF02003EFF38A
:1023E000118483F31288BFF36F8F074A136823F0B9
:1023F0000201DB07116002D4012004F07DFD84F3AB
:102400001188BFF36F8F10BDC40E0020002270B57D
:10241000012104461046FFF7FFFD0F4801F0F6FAD0
:102420000E4B984215D101F001FB26690C4930464C
:1024300004F0B9F800280BDB01253564246908494C
:1024400004F11C0004F0AFF8002801DBE564002073
:1024500070BD6FF00400FBE7992400000000AD0B95
:102460003474000070B501460C2309484B43C4186E
:10247000D4E90E56403300221844A26304F026FA31
:102480002DB132462B460348BDE87040184770BD59
:10249000740E00204471000010B1012804D0704770
:1024A000034B1B6C5B0701D1FFF7DCBF704700BF1C
:1024B000740E002008B54FF02003EFF3118183F371
:1024C0001288BFF36F8F124A136843F00200106046
:1024D000DA0708D481F31188BFF36F8F0120BDE8BC
:1024E000084001F0B5BA4FF08043D3F80C24D3F87C
:1024F0000C34DB07EED5074804F0E8F981F31188C6
:10250000BFF36F8F0020BDE80840FFF7ABBF00BFEF
:10251000C40E0020B40E00202DE9F8433649BFF365
:102520005B8F0746012251E8003F41E80020002868
:10253000F9D1BFF35B8F33B9304931484B60CB6081
:102540008A6004F043F87B1E012B2DD8012F07D1A0
:102550004FF08043D3F81C3403F00303012B23D046
:1025600004F085FD054608BB264B1B78F3B14FF000
:1025700080430222C3F808230646DFF88C904FF010
:1025800080444FF00108D4F81824D4F81834D2034A
:1025900016D503F00303012B01D0012F10D12DB369
:1025A00086F31188BFF36F8FBDE8F8834FF02003E7
:1025B000EFF3118683F31288BFF36F8F0125DCE7F9
:1025C0003046FFF7B3FDD4F81835002BDBD1D4F833
:1025D0000421002AD7D0C4F80431D4F80431C4F857
:1025E0001885C9F88081C4F80880CCE74FF0804393
:1025F0000222C3F80423D7E7700E0020600E0020EB
:10260000900E0020DB14002000E100E008B5074830
:1026100004F00EFD38B10648FFF786FE0448FEF7C9
:1026200025FF002008BD6FF01200FBE7807100005D
:10263000352600000A2838B5074D044604D1AB689A
:102640000D215B6828469847AB6803485B68E1B298
:102650009847204638BD00BF80710000024B0B60D8
:1026600001231360704700BFC80E00200048704768
:102670008874000010B504F0CBFC034C206004F01B
:10268000C3FC6060002010BDC80E00204FF08042E7
:10269000D2F81015D2F8103501F01E0123F01F03F7
:1026A0000B4343F00103C2F81035024B00221A70AD
:1026B000704700BFC61000204FF08053D3F8303170
:1026C000082B20D14FF08042D2F81015CB071AD535
:1026D000D2F8103501F01E0123F01F030B43C2F89E
:1026E0001035D2F808315BB1D2F8103523F01F0352
:1026F0000B4343F00103C2F810356FF08B007047B5
:10270000024B01221A700020704700BFC610002043
:102710002DE9F0410D46164604F076FC3146074699
:10272000284604F05AF928B3B5FBF7F307FB135317
:1027300003BBB6FBF7F407FB1464DCB9B74213D84C
:1027400004F062FCDFF834800746FFF7B5FF04466B
:1027500068B9284601F0FAFD98F800300BB1FFF790
:1027600095FFF61B3D44F0D12046BDE8F0816FF0A7
:102770008B04F9E76FF01504F6E700BFC6100020E0
:102780002DE9F8430E463046194617461C4604F01C
:1027900024F930B346EA040515F0030521D11CB332
:1027A000DFF84C906319032BA6EB050807D80F4AF6
:1027B000D2F80034DB07FBD50020BDE8F883FFF733
:1027C0007BFF58B97B1B4046196801F0DFFD99F883
:1027D00000300BB1FFF75AFF043DE3E76FF08B00C9
:1027E000EBE76FF01500E8E72046E6E700E0014080
:1027F000C6100020F0B54068057B01F01F0444EAD4
:102800004514056987B0002D64D0B2F5001F00F1B2
:10281000100506D12146284604F0EEFB002007B043
:10282000F0BD01AE0027B2F5800F0197776039D176
:10283000B3F1007F14BF052304238DF80430002377
:10284000CDE904630393836823FA01F111F00101D8
:102850001AD1B2F1A07F17D104F01F03620903F56A
:10286000E0732AD0012A3BD11F4A52F82330DB07FC
:102870000AD40DF1030632462146284601F0C6FB74
:102880001A4B98421CD0029603AA2146284601F012
:102890007FFA174B984220D101222146284601F0A9
:1028A0001DFCBBE7B3F1C06F05D0B3F1007F14BFCF
:1028B00001230223C1E70323BFE74FF0A042D4E77F
:1028C0003146284601F004FC094B9842DBD06FF0FA
:1028D0000B00A4E76FF08500A1E76FF015009EE7FD
:1028E00051F82330FFDE00BF000300500400AD0BA1
:1028F0000000AD0B38B545682B69B3B110352846DB
:1029000001F0D6FB044680B90146284601F098FB49
:10291000084B98420BD108492246284601F070FB2B
:10292000224605210620FFF777FB002038BD6FF017
:102930000400FBE70000AD0B3D290000420970B523
:10294000034602D0012A17D070BD0D4E326951687E
:102950000029F9D003F01F0301250C689D400029D0
:10296000F2D08A682A4002D04B68304698472CB192
:10297000236821461C46F2E7024EE7E72346F8E7C4
:102980006C710000587100002DE9F043466840F278
:102990000635D006337B87B002EA050554BFC2F383
:1029A0004010032001F01F07B5F5837F144647EA66
:1029B00043178DF8030044D00FD8062D18D007D840
:1029C000B5B1022D3FD06FF0150007B0BDE8F08320
:1029D000B5F5807FF7D101250AE040F20222954249
:1029E00033D0B5F5407F32D0B5F5007FEBD102256D
:1029F00022032ED5726801238B40C2F80835326954
:102A000092BB07F01F037F092BD0012F79D13F4ADA
:102A100002EB830284F48033D2F80017C3F300433F
:102A2000C4F3404444EA430421F4E16144EA8004ED
:102A300021F0070144EA05230B43C2F800370020C8
:102A4000C3E70725D4E70425D2E70525D0E703250A
:102A5000CEE7630341BF012372688B40C2F80C3597
:102A6000CDE74FF0A042D3E710360DF10202394610
:102A7000304601F0CBFA14F4403F80460CD1394681
:102A8000304604F0B7FA224B9845D8D19DF8021091
:102A9000304601F017FBD2E701AB4FF0000903AA63
:102AA00039463046CDE90439CDE90199CDF80C908D
:102AB00001F06EF9164B984285D114F4003315D00D
:102AC0009DF803308DF80E3084F48034C4F3004454
:102AD0004B4603AA394630468DF80C508DF80D4010
:102AE00001F010FA0A4B9842CDD06CE7CDE90433DF
:102AF00003AA0DF1030339463046039301F048F968
:102B0000F0E703F5E07352F82330FFDE00030050D6
:102B10000000AD0B2DE9F0411A4804F089FA68B3C2
:102B2000DFF86080184CD8F80870D8F810600025DD
:102B300021786368D80206D513F4402F03D0DA0752
:102B400048BF83F4402330684FF0010C23F4801217
:102B50000CFA01FCDB074CBF40EA0C0020EA0C0039
:102B600030603B6840469847002805DB0135032D5F
:102B700004F10804DCD10020BDE8F0816FF0120000
:102B8000FAE700BF6C710000E4740000036803F012
:102B90001F025B09026004D0012B034818BF00200C
:102BA00070474FF0A0407047000300502DE9F04FF0
:102BB000DFF85C81DFF85C9185B01546824600EB5A
:102BC0008101514503D1002005B0BDE8F08FDAF84E
:102BD0000030D804C3F3432203F07F0400F1918056
:102BE0007F2C4FEA134318F8027008BF4FF0FF34F0
:102BF000132B00F28980DFE803F00A11171A1D2356
:102C00001A8787878734606366696C6F7275C5F849
:102C10000C45631C69D10AF1040AD2E7C5F81445D2
:102C2000661CF8D000266AE0C5F80845F1E7C5F84B
:102C30001045F5E7601CC5F80845ECD0002604E017
:102C4000C5F80C45621CE6D0012603A80394FFF7E3
:102C50009DFF039B4FF0010B0BFA03F3C0F80C35FB
:102C600008E0C5F80845002FDAD1631CD3D0002650
:102C7000B3460627DAF80030019303F40052002A25
:102C800003A81CBF4FF0000B01260394FFF77EFF43
:102C9000039A019B00EB8200C3F3C114D0F8002714
:102CA0003B0243EA840343EA0B0302EA09021343AB
:102CB00043EA4603C0F80037ADE7C5F80C45D2E754
:102CC000C5F86445BEE7C5F86445A9E7C5F8684599
:102CD000B8E7C5F86845A3E7C5F86C45A0E7C5F8AF
:102CE0007045AFE7C5F86045ACE703A80394FFF76C
:102CF0004DFF039B012606FA03F3C0F80835B346DF
:102D0000B8E76FF015005FE76FF085005CE700BF84
:102D10008F7C0000F0F8FCFFF8B5044607690D460B
:102D200004F0A5F990B92C4B1B787BB16426606840
:102D300003F05EFFE0B9012004F0D2F8013EF6D1C5
:102D4000F4E786F31188BFF36F8FEFE74FF02003AE
:102D5000EFF3118683F31288BFF36F8F60683146FB
:102D600003F046FF90B986F31188BFF36F8FEDE74C
:102D70004FF02003EFF3118683F31288BFF36F8FB8
:102D80006068314603F034FF0028DAD03B691D70DB
:102D9000626838691368C3F844050120C3F8480520
:102DA0000020C3F82001D3F82051C3F8580152681D
:102DB000D3F85801D20608D5626812680820C2F814
:102DC00000054FF48002C3F8042301229A6081F3C6
:102DD0001188BFF36F8FF8BDDB1400202DE9F74396
:102DE000476805693C684FF00008C4F80085286012
:102DF000D7F80C90064601AA4146484603F0CAFEA1
:102E000000283CDB019BD9F8002019791868FFF7EE
:102E1000CDFE002833DB6B7A3169012B03D0032B05
:102E20002BD14FF01008AB7A032B26D195F80BC0AD
:102E3000BCF1000F02D0BCF1010F1ED12A7A12B1F1
:102E4000022A1AD10E226B687068B3F5164F00681B
:102E500000F0B28034D8B3F5165F00F0B0801AD815
:102E6000B3F5966F00F0AD800CD8B3F5967F00F007
:102E7000AB80B3F5167F00F0AA806FF0850003B039
:102E8000BDE8F083B3F5166F00F0A480B3F5965F4C
:102E9000F3D15C4B43E0B3F5E14F00F09E8008D8DE
:102EA000B3F5615F00F09B80B3F5964FE5D1564BCB
:102EB00035E047F6122E7345DFD14FF400032EE0C4
:102EC000B3F5613F00F08D8015D8B3F5963F00F063
:102ED0008B800AD84DF6C02E734500F08780B3F57D
:102EE000614FCAD14FF46B0319E0B3F5E13FC4D190
:102EF0004FF0EB7313E0B3F5612F7AD009D8DFF808
:102F000020E1734578D0B3F5E12FB6D14FF0E863F7
:102F100005E0DFF810E17345AFD14FF08053C0F802
:102F20002435736848EA0C081B6842EA0802C3F8B3
:102F30006C250B1DD5E9010183E803007B68990727
:102F400012D505F1180001F02FFA304B984256D1F6
:102F5000287E04F10C0204F5907103F0C3FF2B7E70
:102F60000120984000F0EAFC0823C4F800353B7AC1
:102F700053B9C4F81031D4F810316B69C4F8343542
:102F80000123C4F8383523607B689A075CBF4FF48F
:102F90008073C4F804337B68DB0644BF4FF48003BE
:102FA000C4F804332B69C4F8443500200123C4F865
:102FB0004805A360E36062E74FF41D03AFE7144BDD
:102FC000ADE74FF49E23AAE74FF4A033A7E74FF4F1
:102FD0001C33A4E74FF41D23A1E70E4B9FE70E4BD4
:102FE0009DE74FF06C739AE70C4B98E74FF465033D
:102FF00095E74FF0706392E74FF080638FE76FF0D3
:1030000004003CE700B0130000A04E000000AD0B30
:103010000050270000C0750000F03A0000903A010F
:1030200090D0030040420F0070B5012383400E4A48
:10303000BFF35B8FDC4352E8001F01EA040542E85E
:103040000056002EF7D1BFF35B8F4FF480328240E1
:103050000648C0F80823BFF35F8FBFF36F8F0B42A2
:1030600014BF0120002070BDEC0E002000100140B4
:1030700070B40E49D1E90034D01AC31844F10004E9
:1030800022F07F46C1E90034A6F50013B3F5400FE6
:1030900009D2074B1B681A0A1B069C19054B42F103
:1030A0000005C3E9004570BC01F09CBA6001002036
:1030B000F00E00206801002011B3BFF35B8F0123E5
:1030C000104A834052E800CF4CEA030C42E800C1AA
:1030D0000029F7D1BFF35B8F0B4A4FF48033834055
:1030E000C2F80433094BBFF35B8F1B68BFF35B8FE0
:1030F000C340DB0742BF064B4FF40032C3F8002148
:10310000704700BFEC0E002000100140E80E0020C8
:1031100000E100E00D4B1868010A0006BFF35F8F65
:103120000B4BD3F80435181841F10001B3F5801F9B
:103130000AD2084BD3E90023904271EB030303D278
:1031400010F1807041F10001704700BFF00E0020C7
:1031500000100140680100202DE9F04F85B01646AF
:103160001F469DF840A00446FFF75EFF0190FFF761
:10317000D1FFB04271EB070354D23E4B301A67EBDC
:103180000101984271F100014FD23B4B03EB041354
:10319000D3E902239F4208BF96425ED037494FF4DD
:1031A000803804F1500508FA04F8AD00C1F84883EE
:1031B0002046ADB203F083FD26F07F4B05F180453C
:1031C00004F5A87305F58835DC464FF00309029332
:1031D000029A2CF07F4341F82230C1F84483D1F8A1
:1031E0000435274A6FF00200C01A604420F07F4087
:1031F000904232D9286868B1D1F804350393A3EB23
:103200000B0020F07F40B0F5000F26D9204603F0D8
:1032100056FD039BBAF1000F07D109EB030C09F12E
:103220000109D5E7BAF1000F09D06FF01505204666
:103230000199FFF741FF284605B0BDE8F08F012353
:10324000104ABFF35B8FA34052E8000F184342E8D7
:1032500000010029F8D1BFF35B8F07490E982301C5
:1032600001EB0412C8500F9B5360C2E902670025AE
:10327000DDE700BF01008000500100200010014088
:10328000FDFF7F00E80E00207FB51C4C1C4BC4F8EE
:103290000833C4F848331B4B00254FF0FF304FF084
:1032A000FF31C4F80855C3E902014FF48033C4F874
:1032B0000433154B02264FF400320121C4F8046395
:1032C0001120C3F880212A46FEF7A6FE1120FEF742
:1032D00073FE0E4A0123A360236013600C4B0D4A5A
:1032E0000093CDE9015500232846FFF735FF30460E
:1032F000FFF712F9284604B070BD00BF001001406E
:1033000003000F005001002000E100E0EC0E00205F
:1033100071300000FFFF7F002DE9F7432F4CD4F8F8
:10332000043399070BD5D4F8043143B12C4A002358
:10333000C4F80431D4F80431136801331360D4F8AD
:103340000433DA032AD5BFF35B8F264B53E8002FF3
:1033500022F0010143E800100028F7D1BFF35B8F92
:10336000D30702D4D4F84031C3B10025C4F840518A
:10337000D4F84031FFF7CEFE4FF02003EFF3118277
:1033800083F31288BFF36F8F174BD3E90267B04204
:10339000B94106D282F31188BFF36F8F03B0BDE845
:1033A000F0834FF0FF384FF0FF39C3E90289D3E9CA
:1033B00000101D604FF48033C4F84833C4F8405106
:1033C000D4F8403182F31188BFF36F8F0029E5D024
:1033D000009032463B4628468847DFE70010014010
:1033E000F00E0020E80E00205001002030B5431CF4
:1033F000124C85B005D08442A8BF0446012CB8BF4A
:103400000124FFF787FE0E4B0C4DD3E90013401A41
:10341000B0F5000F10D22218AA4228BF2A4652182F
:103420004FF0000007490091CDE9010043F100038E
:10343000FFF792FE05B030BD2A46F0E7FFFF7F00A0
:10344000600100207130000008B5FFF763FE024BF9
:103450001B68C01A08BD00BF6001002010B5084CF1
:10346000012363601120FEF7B5FD064BC4F8083355
:10347000C4F84833044B4FF40032C3F8802110BD28
:103480000010014003000F0000E100E030B50C49DE
:103490000C4D0B680246002405EB0310D0F8080819
:1034A000C0B218B904B10B60002007E00133072B4C
:1034B0004FF00104F0D90B606FF01B00136030BDBA
:1034C000F40E002000E0014030B5816885B010396D
:1034D00021F00704054603F045F91022014668462D
:1034E00003F0DFF907491022684603F0CFF91023F3
:1034F0006A462146284603F003F9003818BF012028
:1035000005B030BDF476000030B50D46816887B057
:10351000102302AA1039044603F0DDF8002802DA6D
:10352000012007B030BD102202A9204603F038FC6C
:1035300000283AD11E49102202A803F097F900286A
:103540000CBF012302232B70204603F015FC01233E
:1035500001460DF10702204603F0BDF80028DFDB2D
:103560009DF8073003F00F021B096A702B710122CE
:103570000DF10701204603F013FC10B96B78042B02
:1035800003D901236B7000232B71A268183A22F033
:103590000702083AA91C204603F015FC0028BFD1F9
:1035A000E91C204603F068FCBBE70323CBE700BF20
:1035B000F4760000F0B5354F460085B00546694603
:1035C00057F8260003F05EFC044610B1FF2005B05A
:1035D000F0BD013602A957F8260003F053FC01287C
:1035E00037D12B482A46492103F067F8294B02932B
:1035F0008DF80C409DF800609DF80870264C002264
:103600002078314603F0BEFB50B36078394603F0B2
:10361000B9FB28B3A378042B03D09DF8031099427B
:103620001ED1E378042B03D09DF80B10994217D1DB
:103630002379042B10D16279022A1DD1174B184827
:103640002A46492103F039F86079831E022BBED93E
:10365000BCE70028CED0B9E79DF802109942EAD025
:103660000132032A04F10604CAD10E482A46492130
:1036700003F023F80120AAE7032A05D00A4B0B49DF
:10368000042A08BF0B46DAE7094BD8E7607500004B
:10369000D67C0000030103036B7D0000B87C0000B2
:1036A000217D0000457D0000BD7C0000CF7C000036
:1036B000B37C00004FF08053D3F83021082A06D1A4
:1036C000D3F83431052B02D8024AD05C7047002071
:1036D000704700BF837D0000024AD2F80034002BFF
:1036E000FBD0704700E0014008B54FF08053D3F89D
:1036F0003021082A4ED14FF080420021C2F80C112F
:10370000C2F81011C2F8381502F54042D3F804147B
:10371000C2F82015D3F80814C2F82415D3F80C14F5
:10372000C2F82815D3F81014C2F82C15D3F81414C5
:10373000C2F83015D3F81814C2F83415D3F81C1495
:10374000C2F84015D3F82014C2F84415D3F8241455
:10375000C2F84815D3F82814C2F84C15D3F82C1425
:10376000C2F85015D3F83014C2F85415D3F83414F5
:10377000C2F86015D3F83814C2F86415D3F83C14B5
:10378000C2F86815D3F84014C2F86C15D3F8443465
:10379000C2F87035FFF78EFF18B13E4B3E4AC3F8B2
:1037A0008C26FFF787FF18B13C4BFB22C3F8182586
:1037B000FFF780FF70B14FF080414FF08053D1F898
:1037C000E42ED3F8583222F00F0203F00F03134314
:1037D000C1F8E43EFFF76EFF20B1314B4FF40072A9
:1037E000C3F840264FF08053D3F83031082B09D16D
:1037F0004FF08043D3F80024D20744BF6FF001029A
:10380000C3F80024274AD2F8883043F47003C2F882
:103810008830BFF34F8FBFF36F8F4FF08053D3F8D3
:103820003021082A0ED1D3F83431052B02D81E4A94
:10383000D35C3BB14FF01023D3F808224FF0804304
:10384000C3F858254FF01021D1F80C32DB071FD5F3
:1038500016480123C0F80435FFF73EFFD1F80C32BB
:1038600023F00103C1F80C32FFF736FF0023C0F844
:103870000435FFF731FFBFF34F8F0A490C4BCA687D
:1038800002F4E0621343CB60BFF34F8F00BFFDE74C
:1038900008BD00BF005000404881030000F0004018
:1038A0000090024000ED00E07D7D000000E001405E
:1038B0000400FA0530B50468CCB1BFF35B8FB4FAED
:1038C00084F3C3F11F03DBB201229A4024EA02020F
:1038D00050E8005FA54204D140E8002CBCF1000F85
:1038E000F6D1BFF35B8FE6D102480B7030BD0248C2
:1038F000FCE700BF0000AD0B0200AD0B10B5036884
:10390000CB40DB0714D401238B400268BFF35B8FED
:1039100043EA020150E8004F944204D140E8001C01
:10392000BCF1000FF6D1BFF35B8FEED1014810BDA3
:103930000148FCE70000AD0B0400AD0B014BC3F8E0
:103940000405704700F00140F7B5044618B101289E
:1039500023D003B0F0BD4FF080430222C3F8082308
:103960000122DA60C3F80401D3F8043106460123CA
:103970008DF8073042F210754FF08047D4B1012C1A
:10398000E7D1D7F80C3403F48033AEBB83B3012006
:1039900003F0A6FA013DF4D12AE04FF08043002263
:1039A000C3F808035860C3F80021D3F800310DF1C3
:1039B0000706DCE7D7F8183403F480333EB9002B50
:1039C000C7D0012003F08CFA013DF3D1C1E7D7F84D
:1039D000182402F003023260002BBAD09DF80700D1
:1039E000012803D103F07CFA013DC7D1012CB0D1ED
:1039F000054B00225A71ACE7D7F80C2402F0010203
:103A00003270002BEAD1F3E7F80E0020044B1A794C
:103A100022B9012218609A80024870470248704714
:103A2000F80E00200000AD0B0C00AD0B08B5074BE5
:103A30001B682BB10020FEF7E1FA08B9FEF7BCFACB
:103A40004FF080430022C3F8182508BDF80E00206F
:103A500010B510B1012843D010BD4FF08043D3F80A
:103A60001814D3F81824C80321D502F00303012B3E
:103A700004D013B10020FFF767FF00234FF080420E
:103A80000220C2F8183508224FF4827303F18043F4
:103A90000021196002F180421C6801241460154A5B
:103AA00012680AB34FF08043C3F80403D4E7D3F895
:103AB0001424D107E1D5D3F81C249207DAD40D4A97
:103AC00012681AB10222C3F80423C5E7D3F804210F
:103AD000002AFBD00022C3F80421D3F80431BBE74D
:103AE00000224FF48073D1E71A68002AFCD01960D5
:103AF0001B68B1E7F80E002010B54FF08043D3F8F3
:103B000000216AB10022C3F80021D3F8002101226C
:103B1000C3F80823114B587910B95A711B6898479C
:103B20004FF08043D3F8042172B10022C3F804217E
:103B3000D3F80421D3F81824D3F81824920704D119
:103B40000122C3F818259A6010BD0222C3F8082389
:103B5000024BBDE810401B6801201847F80E0020FA
:103B6000036803F01F025B09026004D0012B0348C5
:103B700018BF002070474FF0A0407047000300506E
:103B8000034A430900F01F00D35C1844C0B27047D9
:103B9000897D000070B50546FFF7F2FF0C4C083038
:103BA0000E4634F81030DA0508D5C3F3432304EB8E
:103BB000C302284654F8333052689847A3682BB1A3
:103BC000E26831462846BDE87040184770BD00BF26
:103BD0005000002008B5FFF7D3FF034B083033F83F
:103BE0001000400B08BD00BF5000002008B5FFF7D3
:103BF000C7FF034B083033F81000C0F3400008BD86
:103C00005000002008B5FFF7BBFF034B083033F826
:103C10001000C0F3401008BD50000020034611F012
:103C2000010010B5CCB20DD1A207C4F3400012D5EB
:103C3000094AD2F820055860C2F82005003818BF9C
:103C4000012008E04FF0A041D1F820251A60C1F80A
:103C50002025002AE8D010BD0003005010B5FFF762
:103C60008FFF124A083032F81030D9051CD5C3F343
:103C7000432123F4F85322F8103002F10E040020FF
:103C800034F8023F13F4807F03D0C3F343239942F7
:103C90000AD001303028F3D1002342F831300448F3
:103CA000BDE81040FFF72ABE10BD00BF5000002045
:103CB000C8000020F0B5054600200446012607464E
:103CC0008C420BD1114BD3F87C2132B10022C3F8C6
:103CD0007C21D3F87C3140F00040F0BDE3B29B0082
:103CE00003F580729B0806FA03F31D420BD002F124
:103CF000804202F5C042D2F800C0BCF1000F02D0F1
:103D00001760126818430134DAE700BF0060004012
:103D1000F7B506460846FFF733FF194F00F10805CF
:103D20000C4637F81530DB0727D5304603F03EF94F
:103D30002046FFF767FF40B12046FFF74BFF316891
:103D400000F5A270002341F820302046FFF786FFDF
:103D5000002301A827F815300194FFF701FF019B0C
:103D600000EB8300074BD0F80027134043F0020319
:103D7000C0F80037044803B0F0BD0448FBE700BFBB
:103D800050000020F0F8FCFF0000AD0B0400AD0B6C
:103D90002DE9FF41164680460846FFF7F1FE0D4625
:103DA0003168044609B32846FFF720FF18B12846BA
:103DB000FFF728FF10BB0023CDE900338DF80E304C
:103DC0008DF80F300DF10F020B4628460DF10E0154
:103DD00003F094F8474A04F1080132F8113023F057
:103DE000020343F0010322F81130736863B32846DD
:103DF0001F785968FFF7FAFE10B1D1B13E4826E0AE
:103E00003C4A04F1080032F8103023F02003DB04B0
:103E1000DB0C22F8103061B1032FEFD871684968CC
:103E200091F800C0D8F80010A7B90CF5A27C41F8B1
:103E30002C70304A04F1080132F8113023F01C03D1
:103E400043EA870322F81130B3684BBB2B4804B018
:103E5000BDE8F08101EB8C0143EA4C33D1F810E569
:103E60002EF0030EC1F810E5D8F8001001EB8C0E0F
:103E700043F02003DEF8101522F8103021F44F3102
:103E800021F44071CEF810152902DEF8108501F4F6
:103E90007C5141EA074141EA0801CEF81015C8E714
:103EA000D3E900672846FFF7D9FE002ECED0114D8A
:103EB000D5E90023964203D19F4201D1002209E0B7
:103EC0000F480DF10F01FFF7F5FC0C4B9842BED1E6
:103ED0009DF80F2045F8326005EBC20308345F609F
:103EE00035F8143043EA422343F4807325F8143044
:103EF000ACE700BF500000200400AD0B0000AD0B8C
:103F0000C80000202DE9F0430C4685B080462046CD
:103F100011461E46FFF734FE054629B32046FFF73B
:103F200065FE18B92046FFF76DFE18BB314F05F14D
:103F3000080937F8193013F01C0F02D04B78012B09
:103F400018D001238DF80F300023CDE900134A1C4F
:103F50008B1C20460DF10F0102F0D0FF37F819300D
:103F600043F0030327F81930002E41D02046FFF715
:103F70003DFE18B9204805B0BDE8F08396F800C0B2
:103F8000D8F800301B4F0CF5A272002143F8221024
:103F900005F1080237F8121021F02001C904C90CFC
:103FA00027F8121075781DB3D8F80000B67800EB2A
:103FB0008C002D04D0F8103523F4991323F4F85312
:103FC000C0F81035230203F47C5305F44035360560
:103FD000D0F810E52B4306F4801641EA4C31334308
:103FE00041F0200143EA0E0327F81210C0F8103503
:103FF0000248C0E7500000200400AD0B0000AD0BEC
:10400000014BC3E9021270475000002010B508466A
:104010001446FFF7F7FD50B10846FFF7B1FD054B19
:10402000083033F8103004485B0B237010BD034890
:10403000FCE700BF500000200000AD0B0400AD0BFA
:1040400070B5184E96F8804005464CBB214660225C
:1040500006F1100002F025FC2D68306F21468842E1
:1040600012D10023C5F87C3145F30730D5F87C31F7
:10407000FDF7A2FF4FF00043C5F804330A480123BF
:1040800086F88030B36770BDCBB29B0003F58072B9
:104090007C2B08BFAC5001F1010108BFAB58DEE733
:1040A0000248F0E7500000200000AD0B0C00AD0B03
:1040B000034B93F88000003818BF0120704700BF01
:1040C000500000200148FFF719BC00BFC4000020C9
:1040D0000148FFF7EFBB00BFC400002073B50546E1
:1040E00008460C461646FFF78DFD00B30846FFF75D
:1040F0007DFD0146D8B92046FFF76CFD04B2A4004F
:1041000004F580720346286881502968825821444A
:10411000D1F8102542F00102C1F810252EB129680E
:10412000012202FA03F3C1F8043302B070BD204645
:10413000FFF726FD0F4B083033F81030C3F382032E
:10414000042B12D0052B12D001A80194FFF708FD13
:10415000019AD0F81035D34003F00103991C204692
:1041600002B0BDE8704002F012BF0321F7E7022160
:10417000F5E700BF500000202DE9F04F694BDFF854
:10418000B081D3F80403D8F87010C0B289B040F001
:104190000040FFF78FFD051E2FDAC24600235AF8B4
:1041A0007C1F06A8CDE90633FFF738FD5E4B01936F
:1041B0000DF118094FF0000B019A12F8013B019222
:1041C000DA0803F007031AF8022022FA03F3DA07E9
:1041D0001CD409F10409BBF1000F14D0D8F87010F9
:1041E0004FF00040FFF766FDD8F87C1006A8FFF7F7
:1041F00015FD0028DAD125F000450124002D79D1E4
:1042000009B0BDE8F08F4FF0010BD5E7474B5B4499
:104210000293D9F800100029DBD0029B91FAA1F19A
:104220001C78B1FA81F141EA44142046FFF7A8FC5A
:104230000830059438F81070C808BB0819F8002039
:10424000039301F00701012303FA01F122EA0102BD
:1042500009F8002005A8FFF783FC059A039B02F5E7
:10426000E072C7F3820650F822205B073746C2F39C
:10427000014224D520463946D6B2FFF78BFC05A86B
:104280000594FFF76DFC059B03F5E07350F82330B0
:10429000C3F301439E4207D10021204602F077FE7E
:1042A0003146204602F073FE05A80594FFF758FC3E
:1042B000059B012202FA03F3C0F82035A9E7022A80
:1042C0000CD10321204602F062FE06F00503012B0B
:1042D000EAD139462046FFF75DFCE5E7022120469A
:1042E000039202F054FE032EF3D0039A032ADBD18B
:1042F000022EEDE795FAA5F3B3FA83F304FA03F27D
:104300009B0003F1804303F5C04325EA0205D3F87F
:104310001005D3F81015C0F30520C1F30141FFF7D4
:1043200039FC6BE700600040997D0000997D00003A
:1043300050000020044AD2F80034DB07FBD50160AE
:10434000BFF35F8F704700BF00E001404FF0805324
:104350001A69B0FBF2F302FB130373B9084B022294
:10436000C3F80425C3F80805D3F80024D207FBD509
:1043700000220448C3F8042570470348704700BF73
:1043800000E001400000AD0B0A00AD0B10B5054C7C
:104390000123C4F80435FFF7CDFF0023C4F804352A
:1043A00010BD00BF00E0014001460148FFF782BA9E
:1043B000D400002010B5144CA8220021204602F0A1
:1043C00070FA03232361114A6361114BA261E36117
:1043D0004FF4806323620023A3626362E362226678
:1043E0000C4A62661022A2662367E3666367BFF326
:1043F0005F8F094A12F8011DE1540133102BF9D1E6
:10440000BFF35F8F10BD00BF000F00209B7D000039
:10441000DB100020CB100020B47D0000104B70B5E5
:1044200053F82040013053F82060A64200D870BDF8
:10443000D4E9003595B153B12846984738B10028E2
:10444000B8BF4042EB68FF28A8BFFF201870EA6899
:10445000537843F0010353700834E6E79847FBE7CD
:104460006875000008B5094B012203201A70FFF798
:10447000D5FF00F01FF90420FFF7D0FFFBF7AAFFDC
:10448000034A137B23F00103137308BDDB140020E0
:104490007001002008B50348034A0021121A02F0F7
:1044A000E2FD08BD50010020DC14002008B500200A
:1044B000FFF7B4FF184B83F30888184C636943F483
:1044C000007363610025E02384F82230E5772576C8
:1044D0006576A57684F82050636A43F4E02363622E
:1044E00084F82350FDF7C6FCFDF70CFE4FF0FF33B8
:1044F000A362E362FDF786FEFDF744FE02F097FD3E
:104500000120FFF78BFF0220FFF788FF04482B46AE
:104510002A462946FDF7DCFD401D002000ED00E0A5
:104520006544000008B50648064A0749121A02F019
:104530009CFDBDE80840054A0549064802F095BDC6
:10454000000000204C010020E87D00000000000079
:10455000E87D000000000020034B1B680BB9FEF74C
:1045600073BF0020704700BFA80F002010B50E4B8E
:104570001C689C4204D1FFF7EFFF6FF0004010BDB4
:10458000FFF7EAFF002CF8D0D4E904321B1A62EBE3
:10459000E072B3F1004F72F10001EEDA002AACBF15
:1045A00018460020EBE700BFD800002030B570B1FE
:1045B0000B4B5B6898420AD0036843B1D3E90421EE
:1045C000D0E90445121941EB0501C3E90421D0E902
:1045D000003213605A600023C0E9003330BD00BFD1
:1045E000D80000202DE9F84F4FF02003EFF311879A
:1045F00083F31288BFF36F8FDFF8B4902A4E2B4CF1
:104600003060D9F800004FF0000A484508BF00208C
:104610004FF0000BD4E9001E33683D4688B3D0E963
:1046200004874FEAE37C43457CEB070206DAB8EBEC
:10463000030267EB0C07C0E9042722E018EB010135
:104640004EEBE873C0E904ABC4E90013FFF7AEFF1B
:1046500085F31188BFF36F8F836898474FF020036D
:10466000EFF3118583F31288BFF36F8F3368D9F8A6
:104670000000A3EB080348452F463360CAD1D4E9B4
:10468000001E59184EEBE373C4E900130024346094
:10469000FFF76CFF2146FEF7A9FE85F31188BFF3F3
:1046A0006F8FBDE8F88F00BFA80F0020F001002039
:1046B000D8000020014801F018BF00BFB57D000000
:1046C00010B50A4C23681BB101232360002010BDE4
:1046D00000F048F80028F7D00138062803D8044B2A
:1046E00053F8200010BD034810BD00BFAC0F0020E0
:1046F00080750000FE8FFFFFBFF34F8F0549064B0B
:10470000CA6802F4E0621343CB60BFF34F8F00BF6F
:10471000FDE700BF00ED00E00400FA0510B40A4B0D
:104720000A490B4C4FF0FE32C3F800244968C3F825
:104730000424C3F80824C3F80C240023C4F800356B
:104740005DF8044B084700BF00B00250E0000020B5
:1047500000A00250D0E90012014BC3E900127047DB
:10476000E000002038B500F02FF820B1032400F05D
:1047700063F8204638BD00F031F898B900F0ACF885
:1047800098B90F4DD5F828391B0EF02B08D1D5F864
:10479000242A0C4B9A420AD0072400F017F8E6E7C7
:1047A0000624FAE70424204638BD0024F5E701205A
:1047B00000F092F804460028F7D1C5F80C0AD8E7B3
:1047C00000B002500000E020002070470020704739
:1047D000014BC3F8040A704700B0025010B51148ED
:1047E00000F048F800B110BD0F4800F043F8002871
:1047F000F9D10E4C204600F03DF80028F3D10C4BC7
:104800000C481C6000F036F801460028EBD100F09F
:104810002DF8044608B1204610BD00F03FF82046B0
:10482000FAE700BFF8000020F4000020F0000020AC
:10483000E8000020EC00002008B5084800F024F84B
:10484000074800F021F8074800F01EF8064800F07D
:104850001BF8BDE8084000F00BB800BFF8000020CE
:10486000F4000020F0000020EC0000200020704741
:10487000704700BF08B5034B02681B681068984773
:10488000002008BD1001002008B5034B02685B68DA
:1048900010689847002008BD1001002070B5094C31
:1048A000094D2069AB68984718B1084B08485B6808
:1048B0009847084AEB68206900211160BDE8704004
:1048C000184700BFFC00002010010020E00000207D
:1048D0009C750000B00F0020F8B51A4D1A4E044622
:1048E000B26828699047E8B9184F3B684CB1A3B14A
:1048F000012B19D0013B3B602869F36898470020E1
:10490000F8BD43B9124A0121C2F800151149D1F886
:104910001029002AFBD101333B60F36828699847CE
:104920000020F8BD0C48F8BD0A4AD2F81039002B17
:10493000FBD1074A6FF07E40C2F80035FFF748FF11
:104940003B68D7E7FC00002010010020B00F0020DA
:1049500000A0025000B00250E98FFFFF10B50446DE
:1049600050B1636813F0685F05D0064A934202D0E5
:1049700000232360626010BD034B04485B689847C6
:10498000EFE700BF2C5F5CA9E0000020BC750000D1
:10499000C8B143680D4A934213D013F0685F0ED03C
:1049A000012350E8002F194640E8001C9CF0000F3E
:1049B000F7D1012AF5D0BFF35F8F0020704704487C
:1049C0007047044870476FF4E04070472C5F5CA963
:1049D000E98FFFFFEA8FFFFF80B14368094A9342E6
:1049E0000AD013F0685F05D0BFF35F8F0023036028
:1049F0001846704704487047044870476FF4E04019
:104A0000704700BF2C5F5CA9E98FFFFFEA8FFFFFB3
:104A100010B5044620B1044B63600022226010BD33
:104A20000248FFF77BFEF6E73A00003AE475000023
:104A300030B10268034B04489A4208BF0020704717
:104A400002487047DD55AABB8208F0007108F000EB
:104A500038B50D460446B0B1A0220021043002F062
:104A600025FB95B10822294604F1640002F024FBDD
:104A7000082205F1200104F1840002F01DFB044B23
:104A80002360002038BD0348FCE70348FAE700BF75
:104A9000DD55AABB7108F0008308F0002DE9F7434B
:104AA00005460E4699461146FFF7C2FF0446002808
:104AB00040F08480002E00F08580002900F0848082
:104AC000B9F1200F40F0828005F14404082205F17D
:104AD0000408204602F0F0FA05F1240708223146C6
:104AE000404602F0E9FA06F120010822384602F0B9
:104AF000E3FA02A94FF4807041F8049D02F0D0FA65
:104B0000002865D1334A4FF480731360012193600C
:104B10000823314A00F02EFB0121084605232F4AC5
:104B200000F028FB0823424601211C2000F022FB54
:104B300008233A460121032000F01CFB22460823EB
:104B40000121022000F016FB0823254A01211A202A
:104B500000F010FB0523234A01211B2000F00AFB73
:104B60000823214A0121142000F004FB08231F4AD6
:104B70000121152000F0FEFA082305F1640201214D
:104B8000162000F0F7FA082305F18402012117200E
:104B900000F0F0FA0823164A01210B2000F0EAFA8F
:104BA00000F044FB0446019800F0D2FA114B002CAF
:104BB00018BF1C46A421284602F07AFA204603B00A
:104BC000BDE8F0830C4CF9E70C4CF7E70C4CF5E72B
:104BD000084CEFE790B0025048760000C076000025
:104BE00008760000AC7600006C7600008C76000041
:104BF000287600008408F0007608F0008008F000B5
:104C00008108F0000C4BC2691A60826943F8042CD9
:104C1000426943F8082C026943F80C2CC26843F837
:104C2000102C826843F8142C426843F8182C026850
:104C300043F81C2C704700BF5CB602500C4B1B683D
:104C4000C3610C4B1B6883610B4B1B6843610B4BAF
:104C50001B6803610A4B1B68C3600A4B1B688360B7
:104C6000094B1B684360094B1B680360704700BF1A
:104C70005CB6025058B6025054B6025050B60250BC
:104C80004CB6025048B6025044B6025040B60250EC
:104C900030B10268034B04489A4208BF00207047B5
:104CA00002487047DD55AABB0202F0000002F00086
:104CB00038B5044668B1051D7021284602F0F8F9A0
:104CC00028462022044902F0EFF9044B236000201B
:104CD00038BD0348FCE700BFD4760000DD55AABB11
:104CE0000002F0002DE9F043284B04460E4615461D
:104CF0000FCB85B06F4687E80F002DB94FF0000944
:104D0000484605B0BDE8F0832046FFF7C1FF814665
:104D10000028F5D1231D0193636AA3BB236F8BB1D8
:104D2000C3F14008A84528BFA84604F13000314629
:104D30001844424602F0B8F9236F434446442367BF
:104D4000A5EB0805226F402A06D104F13001384650
:104D500000F0AEFB0023236705F03F0835F03F0568
:104D600005D031462A46384600F0A2FB2E44B8F161
:104D7000000FC3D04246314604F1300002F094F9EE
:104D8000C4F87080BCE7DFF80890B9E75073000002
:104D90000C02F0002DE9FF41144B04460E460FCBE8
:104DA0006F4687E80F002046FFF772FF8046B0B9D4
:104DB000CEB1636A251D01953BB901236362226F61
:104DC00004F13001384600F073FB2B46043E2434D6
:104DD00053F8042B12BAA34246F8042FF8D14046E8
:104DE00004B0BDE8F081DFF80880F8E750730000F8
:104DF0000502F000084B1B681B0EF02B08D1074B77
:104E00001A68074B9A4205D1064B0020186070477C
:104E1000052070470620704728B9025024BA025076
:104E20000000E0200CBA0250002230B549001346C1
:104E3000023840F6FC7502F1A05404F52C44A4009D
:104E4000904202F10102CABF236025605B181E2A4E
:104E5000F1D1044A13600B445360034B034A1A60B8
:104E600030BD00BF78B0025084B0025020F80F006F
:104E700030B51E4B85B01A46196800910099CC07D1
:104E8000FAD500F1A05000F52C40800001681368AD
:104E90000193019BD807FAD5154B164C1868164D8F
:104EA0001F30202390FBF3F00138002810DA002394
:104EB0000130400153B1A0F120014FF000421342F4
:104EC00004D1013888424FEA5202F8D105B030BD12
:104ED00013680393039BDB07FAD5431823602B6801
:104EE0000293029B002BE3D10138DEE7B4B00250FD
:104EF000ACB00250E4B00250DCB00250F0B51D6816
:104F000085B001F01F040DB91F2C25D1154D2E467B
:104F10002F680197019FFF07FAD500F1A05000F517
:104F20002C408000006835680395039DED07FAD595
:104F30000D4D00EB611028600C48006802901F2C9A
:104F400018BFC94302980FBF106001F01F0100FA9B
:104F500001F111600021196010684300C00F136057
:104F600005B0F0BDB4B00250E4B00250DCB0025065
:104F70000C4B18603F3020F03F00890140305860F2
:104F80009960D9601961596199611C3306481960AB
:104F900082B002680192019AD207FAD5196002B074
:104FA000704700BF90B00250B4B0025038B5A0F1C5
:104FB0002003B3F5426F05462CD88F2826D800F180
:104FC000470300F16604DB064FEA541400D00134B5
:104FD00064013F34A409013411B1A1421AD30C4633
:104FE000E3004FF48050B0FBF3F0202828BF2020CE
:104FF00002B11060084B01221A602146FFF714FF2E
:1050000028462146FFF7B4FF002038BD00F11F04F9
:105010006409DDE70148F8E71CB802502221F000DE
:10502000F0B5454B89B01D461C680194019CE4070E
:10503000FAD5424BDFF80CE1DFF80CC113449B00BA
:1050400000241A680B181E2B88BFC0F11E011F32E6
:105050000B1852095343B3F5806F82BF4FF4806140
:10506000B1FBF2F1091A00F1A05000F52C402746DF
:10507000A14233DC2B680493049BDB07FAD5304B49
:105080001B68296805910599CF07FAD52D4C2E4943
:10509000236000231E46934203F1010040D120F01B
:1050A00001022948194600268A423CD829680691FF
:1050B0000699CE07FAD52549096828680790079808
:1050C000C007FAD52160204800210C468B422DD123
:1050D0001D4900209A422CD809B0F0BD2B680293DC
:1050E000029BDB07FAD503199B001B682E68039609
:1050F000039EF607FAD5CEF800300023934203F161
:10510000010306D1164623F00103B34204D801344B
:10511000AEE7CCF80070F1E7CCF800700136F4E7A8
:105120000E600346B7E706600131BDE70460013158
:10513000CCE708600133CDE7B4B0025024AC0014D2
:105140007CB00250D4B00250D8B0025078B00250B7
:1051500008B540B1202801464FF0070228BF2021A2
:105160000020FFF75DFF024B00221A6008BD00BF60
:105170001CB80250F0B5294D85B02C462E6800961B
:10518000009EF607FAD500F1A05000F52C408000F3
:105190000568206801900198C707FAD52048214F7B
:1051A000056002EB8306B24229D15A1C1D4E22F043
:1051B000010200279A4227D823680293029BDE0748
:1051C000FAD5194B0B449B001B681F335B099A42AD
:1051D00013D2216803910399C907FAD51544002118
:1051E0009B1A104A056008468B4210D85A1C0D497C
:1051F00022F0010200209A420CD805B0F0BD52F80E
:1052000004CBC7F800C0CEE737600133D2E71060A7
:105210000131E9E708600133EDE700BFB4B00250A7
:10522000D4B00250D8B0025024AC00142DE9F041A3
:10523000814B1D6898682033A0B01E461A68019201
:10524000019AD707FAD57D4B7D4A1A6032680292DF
:10525000029AD407FAD57B4A1A607B4A1446116831
:1052600003910399C907FAD5784A1168C1F340211F
:1052700037680497049FFF07FAD5754F1F602768AA
:105280000597059FFF07FAD51768002900F0CF8022
:10529000B90540F1CC80316806910699CF07FAD55F
:1052A0006C491960216807910799C907FAD51168F7
:1052B000C1F3402137680897089FFF07FAD5664F6A
:1052C0001F6027680997099FFF07FAD51268002910
:1052D00000F0AF80910540F1AC8032680A920A9AE2
:1052E000D207FAD5564A1A6032680B920B9AD70742
:1052F000FAD55A4A1A6031680C910C99CC07FAD544
:105300005749196031680D910D99C907FAD555496A
:10531000196031680E910E99CF07FAD5524919607C
:1053200031680F910F99CC07FAD550491960504B4D
:105330001E46196810911099C907FAD53F4C4D4B7C
:10534000236033681193119BDB07FAD54A4B236026
:1053500033681293129BDF07FAD5484B23603A4B10
:105360009846196813911399C907FAD5324F3860D6
:1053700033681493149BDB07FAD5226033681593C6
:10538000159BD807FAD53E4B236033681693169BBE
:10539000D907FAD53B4B236033681793179BDA077D
:1053A000FAD5394B236033681893189BDB07FAD57D
:1053B000364B236033681993199BD807FAD5344BC1
:1053C000236033681A931A9BD907FAD5314B2360AF
:1053D00033681B931B9BDA07FAD52F4B236000F031
:1053E0001DFC08BBD8F800301C931C9BDB07F9D5CB
:1053F0003D6033681D931D9BD907FAD5274B236069
:1054000033681E931E9BDA07FAD5254B2360D8F824
:1054100000301F931F9BDB07F9D50C4B1B6813F45F
:10542000805F204B08BF184620B0BDE8F0811E48C1
:10543000FAE71E48F8E700BF90B0025080B0025073
:1054400000100251C01F7229B4B0025088B002503F
:10545000C0CF0129C01F0E29C03F002940010249C9
:10546000003184A800001649400108A18044088842
:10547000B0B00250C044708880077A41C0077E41B6
:1054800000006A498006164940006E49000200216A
:1054900000822021408220218082242140A161A11C
:1054A00000C861510308F1000108F1000208F10091
:1054B0002DE9F74F314B44688046924699461A6869
:1054C000002AFCD12E4B9B461A68002AFCD14FF0D3
:1054D000FF30019100F094FC802000F097FC294DF2
:1054E000294A2A4F2A4E012307202B60A2F59E72DB
:1054F000C2F83C011360636A3B60A36A3360D8F86A
:10550000003042F8043CD8F808302046984701990A
:10551000D9F80030002BFBD1BAF1000F20D11D4B80
:1055200004221A60D9F80030002BFBD1DBF800A070
:10553000BAF1000FFAD1D8F80C30204698473B68F2
:1055400063623368A362144BC3F800A0C3F844A19C
:10555000D9F80030002BFBD12B6003B0BDE8F08FF1
:10556000236A012B04BF0C4A13600C4B40201960C6
:10557000C3F804A000F050FCD4E700BF10B90250FB
:1055800020BC025018B8025000B90250CCB70250EB
:10559000D0B70250C8B7025084B6025028BC02509F
:1055A00010B5544B98B019461A680192019AD20767
:1055B000FAD5514B514A1A600A680292029AD407EE
:1055C000FAD54F4A1A600A680392039AD007FAD5AF
:1055D0004C4818600A680492049AD207FAD54A4ADD
:1055E0001A600A680592059AD407FAD5474A1A60E4
:1055F0000A680692069AD207FAD5454A1A600A68DE
:105600000792079AD407FAD5424A1A600A680892A4
:10561000089AD207FAD5404A1A600A680992099A8C
:10562000D407FAD53D4A1A600A680A920A9AD20744
:10563000FAD53B4A1A600A680B920B9AD407FAD53E
:10564000384A1A600A680C920C9AD207FAD5364A80
:105650001A600A680D920D9AD407FAD5334A1A6077
:105660000A680E920E9AD207FAD5314A1A600A6871
:105670000F920F9AD407FAD52E4A1A600A68109230
:10568000109AD207FAD52C4A1A601A4B19461C6890
:105690001194119CE407FAD5174B18600868129012
:1056A0001298C407FAD51A600A681392139AD007A1
:1056B000FAD5124A1A600A681492149AD207FAD5D7
:1056C0001E4A1A600A681592159AD407FAD51C4A20
:1056D0001A600A681692169AD007FAD5194A1A6003
:1056E0000A681792179AD207FAD5174A1A6018B0A3
:1056F00010BD00BFB0B0025080B0025000936521D1
:1057000000043190409665900083612100C33021F0
:1057100000C3649000816190004610210081112136
:105720000041442100C320290C4610C800863121C5
:1057300000C3602140C128294096652100133190A3
:1057400040962529594614C84004324910B5494BA2
:1057500094B019461A680092009AD207FAD5464BBF
:10576000464A1A600A680192019AD407FAD5444A57
:105770001A600A680292029AD007FAD54148186066
:105780000A680392039AD207FAD53F4A1A600A6858
:105790000492049AD407FAD53C4A1A600A68059222
:1057A000059AD207FAD53A4A1A600A680692069A0A
:1057B000D407FAD5374A1A600A680792079AD207BF
:1057C000FAD5354A1A600A680892089AD407FAD5B9
:1057D000324A1A600A680992099AD207FAD5304A01
:1057E0001A600A680A920A9AD407FAD52D4A1A60F2
:1057F0000A680B920B9AD207FAD52B4A1A600A68EC
:105800000C920C9AD407FAD5284A1A600A680D92AD
:105810000D9AD207FAD5264A1A600A680E920E9A95
:10582000D407FAD5234A1A600A680F920F9AD20752
:10583000FAD5214A1A600F4B19461C681094109C27
:10584000E407FAD50C4B1860086811901198C4074A
:10585000FAD51A600A681292129AD007FAD5174A36
:105860001A600A681392139AD207FAD5144A1A607A
:1058700014B010BDB0B0025080B0025080906521CD
:105880000004099040966590808061218020082165
:1058900080206490008161900046102100811121D8
:1058A0000041442180202029024610C80086092199
:1058B0008020602140212829409665214096252995
:1058C000594614C810B5504B96B01C461A68019240
:1058D000019AD207FAD54D4B4D4A1A6022680292BE
:1058E000029AD207FAD54B4A1A604B4A42EA8040E4
:1058F00022680392039AD207FAD5186022680492AC
:10590000049AD007FAD5454A1A60A2F5800242EA05
:10591000814122680592059AD207FAD5196022685A
:105920000692069AD007FAD53D4A1A602268079275
:10593000079AD107FAD53B4A1A6022680892089A5A
:10594000D207FAD5384A1A6022680992099AD00714
:10595000FAD5364A1A6022680A920A9AD107FAD50D
:10596000334A1A6022680B920B9AD207FAD5314A51
:105970001A6022680C920C9AD007FAD52E4A1A6047
:1059800022680D920D9AD107FAD52C4A1A60226826
:105990000E920E9AD207FAD5294A1A6022680F92FF
:1059A0000F9AD007FAD5274A1A60216810911099EA
:1059B000C907FAD51A60144B1A4619681191119942
:1059C000C807FAD5114B2049196011681291129934
:1059D000C907FAD51D491960116813911399CC07AD
:1059E000FAD50B491960116814911499C807FAD5B2
:1059F00017491960116815911599C907FAD5154A03
:105A00001A6016B010BD00BFB0B0025080B0025096
:105A10004004419000862929D81001C840144190C3
:105A200040142129401465210034409000310C902D
:105A3000C0400C90C030202940960D9000416090ED
:105A4000031645C80086112100416021594644C80B
:105A50004014459040142D9070B5264888B00546F6
:105A600004680094009CE607FAD52348234C0460A0
:105A7000234C44EA83432C680194019CE407FAD543
:105A80000360930143EA824242F0104444F4C0446C
:105A90002B680293029BDE07FAD504602B68039300
:105AA000039BDB07FAD5174B03608B0143EA814167
:105AB00041F0104343F4C0432E680496049EF60759
:105AC000FAD503602B680593059BDE07FAD50460C1
:105AD00041F058412B680693069BDC07FAD501601C
:105AE00042F058422B680793079BDB07FAD5026008
:105AF00008B070BDB0B0025080B00250C021022981
:105B00008071009880611890354B8EB019461A68E4
:105B10000092009AD207FAD5324B334A1A600A68CB
:105B20000192019AD007FAD5304A1A600A680292A7
:105B3000029AD207FAD52E4A1A600A680392039A8B
:105B4000D007FAD52B4A1A600A680492049AD20741
:105B5000FAD5294A1A600A680592059AD007FAD53B
:105B6000264A1A600A680692069AD207FAD5244A8B
:105B70001A600A680792079AD007FAD5214A1A6074
:105B80000A680892089AD207FAD51F4A1A600A686A
:105B90000992099AD007FAD51C4A1A600A680A9233
:105BA0000A9AD207FAD51A4A1A6008680B900B981D
:105BB000C007FAD51A600A680C920C9AD007FAD579
:105BC000144A1A600A680D920D9AD207FAD5124A41
:105BD0001A600E210D230F2200200EB0FFF73CBFEC
:105BE000B0B0025080B00250804301294063392197
:105BF000807001298020542100D13490C04034901D
:105C0000C0302029C0530D9000413890832308C82C
:105C100080E3102100413821CF4308C82DE9F0412D
:105C2000012392B0CDE90333624B1D461A680592F9
:105C3000059AD207FAD5604C604B2360604B194639
:105C40001A680692069AD707FAD55E4B1A68D604E8
:105C500000F1A8802A680792079AD007FAD55A4A15
:105C600022600A680892089AD207FAD51E68C6F31D
:105C70000036002E40F098801220FFF7F9F8074612
:105C80001320FFF7F5F887428CBF12201320FFF78F
:105C9000EFF8471EFFF738FF03AB01AA3946122081
:105CA000FFF72CF904AB804602AA39461320FFF710
:105CB00025F900EB4800022832D003283ED0012805
:105CC00074D12B680993099BDB07FAD53F4B2360FE
:105CD0002B680A930A9BD807FAD53D4B23602B68A3
:105CE0000F930F9BD907FAD53A4B23602B6810937B
:105CF000109BDA07FAD5384B23602B681193119B60
:105D0000DB07FAD5354B2360013F25D51023192237
:105D100018210020FFF7A0FE304612B0BDE8F08148
:105D20002B680B930B9BD907FAD52D4B23602B685F
:105D30000C930C9BDA07FAD52A4BCFE72B680D930F
:105D40000D9BDB07FAD5284B23602B680E930E9B27
:105D5000D807FAD5254BC1E703AB01AA3946122073
:105D6000FFF7CCF804AB044602AA39461320FFF72C
:105D7000C5F810EB440402D1FFF712FCC4E7FFF7AB
:105D8000E5FC022C08D0032C09D0012C10D11721DE
:105D90001620FFF797FDB7E715211420F9E70F212B
:105DA0000E20F6E7124EB7E7124EB5E7124EB3E7F4
:105DB000124EB1E7B0B0025080B0025000084A5114
:105DC000B4B0025088B0025000084E5100065A4943
:105DD00040065E49000442410014424940042E49F5
:105DE000000652494006564900063A4940063E49D7
:105DF0000608F1000708F1000408F1000508F100A9
:105E0000014B1860704700BF08BA0250014B186080
:105E1000704700BF04BA0250034A13681842FCD00E
:105E2000024A10601846704700BA025008BA025081
:105E300070470020704730B583688B4285B00446B8
:105E400015460ED96368C068194401AA00F01DFE0A
:105E500028B96268019B9B1A2B60029B6B6005B09E
:105E600030BD6FF02100FAE770472DE9F7430E4689
:105E700017469946044628B94FF0FF38404603B00C
:105E8000BDE8F0830029F7D0002AF5D0CB680D8952
:105E90001D4404230DEB03022946384600F01BFC89
:105EA00080460028E8D1BDF80410738946F6081230
:105EB000914225D1BDF806109942DDD104230DEBA6
:105EC00003022944384600F006FC0028D4D1BDF86E
:105ED000042046F607139A42CED1C4E900679DF824
:105EE0002830A4F80890A3727389BDF806202B44CB
:105EF000E360738913442B44043563612561BDE776
:105F0000002BE4D0B8E72DE9F3410E4617461D46B5
:105F1000044620B94FF0FF3002B0BDE8F0810368BD
:105F2000002BF7D04368002BF4D04FF6FF78D4E96C
:105F300004239A4216D223685B8923B1E368934213
:105F400004BF043323610423216960680DEB03025D
:105F500000F0C1FB0028DDD1A37A2BB1D4E90332D4
:105F60009A4201D30120D7E72389BDF806104345A3
:105F700001F1040203D0BDF804C09C450BD115B15A
:105F8000BDF804302B8023690433336039802369E2
:105F900013442361C0E7236913442361C7E773B542
:105FA0000C4606461146022301AA204600F00EFACE
:105FB0000546E8B9019A1F2A0ED92368A2F12001EB
:105FC00019442022304600F061FC2368019A1344F2
:105FD0002360284602B070BD0146C2F1200230465F
:105FE00000F05FFC019A2168C2F120003044EAE72A
:105FF0006FF00205EDE700F039BC4FF4C073584371
:106000003030704710B5044600F0A5FBA3684FF48C
:10601000C072303B02FB103010BD70B50D46044617
:1060200000F0AAFE2A46A0F1080104232046BDE89C
:10603000704000F050BB13B50446019100F09CFE87
:106040000423A0F108010DEB0302204600F0D7FE67
:1060500002B010BD70B513460E461546002102462B
:106060000446FAF7B9FE50B92B4604F12C0201217F
:106070002046FAF7B1FE10B1002E08BF002070BD17
:1060800073B5044600200D461646FAF723FA694612
:10609000C0B2FBF74DFD30BB2C2303FB0544009839
:1060A000E36825891D4404230DEB0302294600F013
:1060B00012FBC0B9BDF804206489009846F60813A5
:1060C0009A4215D1BDF806309C420CD104230DEB49
:1060D0000302611900F0FFFA28B9BDF8042046F662
:1060E00007139A4207D0009800F0F4FA02B070BD8E
:1060F000002CF2D0F7E7BDF80610214429443160A6
:10610000F1E737B50446426A802501A902200195CE
:10611000FBF736FD58B9019B226DA36201A905204A
:106120000195FBF72DFD054628B1092500E0012565
:10613000284603B030BD019B206A636500F00BFB6D
:10614000E065F5E70123036003F1012343600023C9
:10615000C0E9023370474379012B07D10368012B53
:1061600004D10079431E58425841704700207047BF
:106170007FB506460D46022001A9FBF7D9FC38BBC6
:106180000198FFF73FFFF16D0446284600F0BFF885
:106190000444019800F0DFFA0646019800F0E2FAA4
:1061A000082201460DEB020000F07BFB2B798DF8F5
:1061B000083021460198334602AA00F0A1FA041ED5
:1061C000019818BF012400F085FA204604B070BD84
:1061D0000124FAE700F0A9BA2DE9F8430E460021A0
:1061E00007460846FAF776F9012104460020FAF737
:1061F00071F933789C4221D0984221D101252C237A
:1062000003FB0575F86DAC6AFFF7F7FE013C074626
:106210004FF000086B6A03EBC40253F83410D2F855
:1062200004901B684A46C91A3046C844FFF7D2FF9B
:10623000B84504F1FF34EDD3BDE8F8830025DEE76F
:106240000120F9E737B515460C460520694600F0F0
:1062500019FEE979012903D00022204600F026FE2C
:106260009DF80330012B02D1204600F0FEFDA96805
:106270002046FFF7E0FE2046FDF726F9002003B098
:1062800030BD73B50D460646FAF7A6FE0446E86033
:1062900050B302282DD101A9FBF74AFC58BB019845
:1062A0002A463146FAF7FEFD0446D0B9019800F0BF
:1062B00063FD012301460DF10302019800F00BFA82
:1062C0000446A0B9019801220DF1030100F068FD18
:1062D00010B101238DF803309DF8033003F00F0354
:1062E000EB71019800F0F6F9204602B070BD012470
:1062F000F7E70724F8E70124F6E7436A00205A6825
:10630000034613448B4200F10100FAD3704710B5E5
:1063100043790279012B14BFCB01002302F1FF3234
:1063200001FB0233026814BF4C000C46013A04FB27
:10633000023010BD70B50368CD1A002D02DC6FF07D
:106340005F0070BD93F900601C78002E0ADB5C1CB6
:1063500004601B7813600368C91A13688B42EED877
:106360000020EEE704F07F04013C032C2BD8DFE88B
:1063700004F0020A1421012DE1D05B781360036858
:1063800002330360E7E7022DD9DDB3F801305BBAD1
:106390009BB2136003680333F3E7032DCFDD9C78D2
:1063A0005D78DB78240244EA0544234313600368E4
:1063B0000433E6E7042DC2DDD3F801301BBA1360C5
:1063C00003680533DDE76FF06300BAE770B4046873
:1063D0000E1B002E07DD26789E4208D10134046092
:1063E00070BCFFF7A7BF6FF05F0070BC70476FF025
:1063F0006100FAE738B503230446FFF7E7FF18B951
:10640000136813B96FF0670038BD013B1360236850
:106410001A78002AF6D101332360F5E72DE9F3411C
:1064200090461F4601AA302305460E46FFF7CEFFD1
:106430000446F0B92B68F61A002E34DD42461B786C
:1064400042F8043B019B2E681E4431460623284631
:10645000FFF7BCFF044660B92B68D8F80420C8F8E1
:1064600008309918B142296007D10C213846FAF753
:106470005DFF204602B0BDE8F0819B5C3A463146A4
:1064800042F8043B2B6801332B602846FFF752FF8C
:1064900060B92B687A68BB601344B3422B6018BFA5
:1064A0006FF06504E5E76FF05F04E2E70446E0E7BC
:1064B000F8B5B1F1005F00AF0546144610D2D31D08
:1064C00023F007036E46ADEB030D684600F0DEF9DE
:1064D000694622462846FEF705FCB546BD46F8BD8E
:1064E000FEF700FCFAE7002070470FB407B504A9D7
:1064F00051F8040B0191FAF7BFFF03B05DF804EB0C
:1065000004B07047038B13F0070305D10368002B19
:106510000CBF002003207047022B05D1408BB0FA3E
:1065200080F0400980007047012B05D10368002BE3
:106530000CBF0020052070470020704710B50C46A6
:1065400000B111B96FF0150010BD081D00F096F8EC
:106550000028F9D1A368032BF6D9F3E72DE9F04120
:106560000D4607461946281D90461E4600F097F82E
:10657000044638B13346424629463846A446BDE86B
:10658000F0416047BDE8F08110B44FF02004EFF314
:10659000118284F31288BFF36F8F41615DF8044B61
:1065A0000121FAF777BF38B50C46054658B151B10D
:1065B0000B6843B14B6833B11C22002100F071F924
:1065C0002C61002038BD6FF01500FBE770B5054663
:1065D0000E46FFF7B3FF041E15DB4FF02003EFF369
:1065E000118283F31288BFF36F8F6B8B2C8B4FF666
:1065F000FF718B4204F0070407D182F31188BFF3C7
:106600006F8F6FF00A04204670BD022C0CD101334D
:106610006B8382F31188BFF36F8F002322463146CC
:106620002846FFF79BFFEEE7062C14D8DFE804F0BE
:1066300004131313041A0400002333606B683BB97E
:10664000C5E90066ACB902212846FAF723FFDAE76C
:106650001E606E60F6E782F31188BFF36F8F6FF0F4
:106660000404D0E782F31188BFF36F8F6FF08504C5
:10667000C9E782F31188BFF36F8FC4E7034658B1AF
:10668000426802F00302012A03D0032A04D10268FF
:1066900012B10020986070476FF015007047426893
:1066A000816002F00302032A4FF0000203460CBF90
:1066B000006810465A60704770470FB407B504A9C8
:1066C00051F8040B0191FAF7D7FE03B05DF804EB23
:1066D00004B070477047002930B4044618460BDBFD
:1066E000A5680844A84207D8E06864682144846823
:1066F0002468A44630BC60476FF0150030BC70477A
:10670000002930B4044618460BDBA5680844A842AB
:1067100007D8E0686468214484686468A44630BC93
:1067200060476FF0150030BC70470029034610B475
:1067300010460BDB9C680844A04207D8D8685B6809
:10674000194483685DF8044B9B6818476FF0150087
:106750005DF8044B704708B5C0688368DB689847EC
:10676000006808BD08B5C0688368DB689847007991
:1067700008BD70B54C680368A34201D2012070BD0A
:106780008A682244934201D30020F8E7D1E9032527
:106790004E69B54203D36FF00B038B61F4E71B1B0B
:1067A00042F835304368086902EBC00253600B6958
:1067B00001330B61E2E708B50020FBF79BF9704756
:1067C00000F041BC0146006800F03DBC08B5FBF795
:1067D0000DFABDE80840FBF70DBA00210120FFF7D4
:1067E000EFBF202809D9B0F1004F08D80138B0FA1E
:1067F00080F0C0F11F0040007047082070473E2025
:1068000070472DE9FF410E4698461446054600277D
:10681000B74220DA6868C8B1B8F1000F07D0431E4C
:10682000184216D11F2814D92A68134211D12B6897
:106830000193FFF7D6FFAB6803430393E3B2072B43
:1068400007D8204601A9FBF7A9FC013401370C3514
:10685000DEE76FF01504204604B0BDE8F081034682
:1068600000201A5C02B970470130FAE710B55AB13E
:106870000139841810F8012B11F8013FA04201D012
:106880009A42F7D0D01A10BD1046FCE710B5431E4F
:106890000A44914200D110BD11F8014B03F8014F99
:1068A000F7E7C9B202440346934200D1704703F8A8
:1068B000011BF9E74FF0FF3070470369C9B20C22A2
:1068C00001FB0233186C00F0070070474FF0200303
:1068D000EFF3118283F31288BFF36F8F036803F025
:1068E000C00343F00203036082F31188BFF36F8F8C
:1068F000704770B5C9B203694FF02004EFF31185FA
:1069000084F31288BFF36F8F0C2606FB0134246CCE
:1069100014F0C00408D0A24206D085F31188BFF35A
:106920006F8F4FF0FF3070BD71430B4401221A642A
:1069300085F31188BFF36F8F43680B445B689847FA
:106940000020F0E78022FFF7D4BFF8B5069F046966
:10695000C9B24FF02005EFF3118685F31288BFF31B
:106960006F8F0C2569430C44256C05F0070CBCF1B6
:10697000010F0BD1276486F31188BFF36F8FC4E931
:106980000E2343685B5898470020F8BD05F0C0050A
:10699000AF4286F31188BFF36F8F0CBF6FF07700A3
:1069A0004FF0FF30F1E713B580240094FFF7CDFFDF
:1069B00002B010BD6FF08500704710B40069CBB213
:1069C0001C2403FB040000215DF8044B1047002049
:1069D000FDF73EB8002000F08FBA38B505460C46EA
:1069E00000F00CFB002D07DBA84205D9401B8442B8
:1069F0008CBF0020012038BD0020FCE770B50D469B
:106A00002846194616461C46FFF7E7FF38B124B161
:106A1000224629463046FFF739FF002070BD6FF04F
:106A20001500FBE72DE9F3411C46904600238268E0
:106A30002360A36013690D4601AA69469847019B2C
:106A40005A1E019223B96FF0150002B0BDE8F08123
:106A50000098A26847682168676085B9A8EB0203BF
:106A60000668B34228BF33461A4403FB071121606E
:106A7000A26002689A4206D808300090DFE76B1ADD
:106A8000B3FBF7F3ECE70020DFE713460022FFF744
:106A9000C9BF2DE9F047836886B01B6988469146D7
:106AA00001A902AA98470024A2462546029BAB42B0
:106AB00002D806B0BDE8F087019F07EBC5070026A6
:106AC0007B6804933A68B2420AEB060302D80135A8
:106AD0009A46EBE703940593494603A8C04700286C
:106AE000E7D0049B01361C44ECE743685B68D3F8AD
:106AF00010350B600020704743685B6802EA0100B4
:106B000021EA0201C3F80805C3F80C1500207047FC
:106B100043685B680020C3F80815704743685B68EA
:106B20000020C3F80C15704743685A68D2F8043542
:106B300021EA03000B40C2F80805C2F80C3500201A
:106B4000704710B503695868F8B1884219D19C683C
:106B500008685860A14200D19860002008602AB1FE
:106B60005A680A609A68596002B99960002010E07A
:106B7000814206D10868206098688142EDD19C600E
:106B8000EBE7044600680028F2D1002AE8D16FF054
:106B9000150010BD30B543681360057A446804EBF6
:106BA000C504A34202D36FF0010030BD5C798C4272
:106BB00001D00833F0E70020F7E743681B68D3F8FB
:106BC0008004C3F880047047436802691B68D3F8E7
:106BD000100150B15269002012780A70C3F81001F8
:106BE000D3F8102101221A6070474FF0FF30704730
:106BF00002680346D2F8580140B95B689B0706D487
:106C0000D2F82001003818BF0120704701207047DA
:106C100042681368D3F80413C90518D5D3F82011B6
:106C2000A9B14FF02000EFF3118180F31288BFF378
:106C30006F8FD3F8200130B10020C3F82001D3F8C2
:106C400020010120D86081F31188BFF36F8F526853
:106C5000D20615D54FF02001EFF3118281F312888F
:106C6000BFF36F8FD3F8581111B10021C3F800158D
:106C70004FF48001C3F8081382F31188BFF36F8FBC
:106C8000704710B50022044601212820FBF7C4F903
:106C90002820FBF791F92046BDE81040FCF79EB88C
:106CA00010B50022044601210220FBF7B5F90220AD
:106CB000FBF782F92046BDE81040FCF78FB800F1E1
:106CC00050039B009BB203F1804303F588330022FD
:106CD0001A601B68704773B5054601A80C46164636
:106CE000FCF7D4FB70BB4FF080531969B5FBF1F290
:106CF00001FB125242BB1969B4FBF1F201FB1242D3
:106D000012BB1A695B695343A3421DD3E4B1019BD3
:106D10001B0103F1804101F5F031C1F80058C1F8C1
:106D20000448C1F80868D1F8002895420FD1D1F87D
:106D3000042894420BD1D1F80838DBB2B34218BF13
:106D40006FF00D0002B070BD6FF01500FAE76FF044
:106D50000D00F7E70222FFF7BEBF08B50020FBF7E2
:106D6000C5F8FDF7ADBC08B5FAF73AFFFFF727FD08
:106D7000BDE80840FDF7A4BC8068183820F0070083
:106D800010387047042809D0052803D1481E18BFC1
:106D900001207047431A58425841704701207047FC
:106DA00038B515460C4661B15AB1FFF7DBFC2544F6
:106DB000214611F8013B834203D1A942F9D10120B8
:106DC00038BD0020FCE738B50C46012311462246A9
:106DD0000546FFF780FC00280FDB012221462846EC
:106DE000FFF7DEFF38B92378012B14BF02230123FC
:106DF0002370002038BD0323FAE70120FAE72DE9CC
:106E0000F7431D4606460F469046FFF7A4FC6C1E4E
:106E1000044440420440082C1AD83046FFF7A2FC34
:106E20002A46814641466846FFF730FD621B4946C7
:106E30000DEB0500FFF735FD23466A46394630461F
:106E4000FFF75EFC003818BF012003B0BDE8F083F7
:106E50004FF0FF30F9E707B501238DF8042001AAB0
:106E6000FFF7CDFF03B05DF804FB816818390122FC
:106E700021F00701FFF7EFBF8268183A22F00702FE
:106E8000FFF7A1BF13B50C46C0B201A9FAF750FE37
:106E900050B921460198FCF737FB04460198FFF7EB
:106EA00019FC204602B010BD0124FAE713B541EAEF
:106EB000021104468DF80710FFF75EFF012301461B
:106EC0000DF107022046FFF79AFF02B010BD81685E
:106ED000183921F0070101220839FFF7BCBF00472C
:106EE00000F0A1B8C00000F1804000F5F830C0F813
:106EF0001015C0F814257047FCF726BDF7B50190B2
:106F000001A8DDE9084716461D46FCF729FE019B4E
:106F1000B6F1000C18BF4FF0010C00EB83000B1E04
:106F200018BF0123002D43EA4C0314BF4FF00C0C93
:106F30004FF0000C002C43EA0C0314BF4FF4E06C3C
:106F40004FF0000C002F43EA0C03D0F8002714BFC9
:106F50004FF4403C4FF0000C43EA0C0322EA0303D9
:106F600001B109780EB13678760019430DB12D784C
:106F7000AD0031430CB12478240229430FB13F788E
:106F80003F040C433C43C0F8004703B0F0BD1FB5BD
:106F90000DF10F03019300238DF80F1000931A4693
:106FA0001946FFF7ABFF05B05DF804FB38B50546A1
:106FB00008460C46FCF726FEB0B10846FCF716FE64
:106FC00090B90846FCF706FE2A6801238340C2F800
:106FD00008332A6803B202EB8303D3F8102522F0AA
:106FE0000302C3F8102538BD20460021BDE8384013
:106FF000FFF7CDBFFCF78CBEFFF7D8BF4FF0805333
:107000001A695869504370474FF0805318697047A8
:107010004FF0805358697047FDF7CCB908B5FFF7BA
:10702000FBFF002008BD08B1FBF790B9704770471F
:1070300040B1C368587810F001001EBF1878B0FA4C
:1070400080F04009704710B54FF02003EFF3118432
:1070500083F31288BFF36F8FFFF77FFE84F31188ED
:10706000BFF36F8F10BDFFF71CBCFFF70FBCEFF332
:107070000580003818BF012070472DE9F041069FB8
:10708000044615461E46FDF7E3FC38B93B4632463A
:1070900029462046BDE8F041FDF700BDBDE8F0817E
:1070A0000A460021FDF782BFFFF7F0BBFFF7F9BBEF
:1070B0000A460021FFF7F5BB01EB820204388A4241
:1070C00001D10020704752F8043D1BBA40F8043F3C
:1070D000F5E700006090FF7F01000000352300000D
:1070E000000000000D240000447100001D7000002D
:1070F00000000000F52800006C710000F528000079
:1071000058710000636D000000000000A16C0000D9
:1071100094710000836C0000807100000D26000057
:10712000000000008932000000000000676D0000D0
:1071300000000000152B0000000000007526000074
:10714000A87100003E7C00004074000058740000EC
:1071500040010020740E0020737C00009074000039
:10716000C074000044010020D00E0020817C00008B
:10717000A8740000C074000046010020DC0E00204E
:10718000977C0000FC74000054750000480100204A
:1071900018000020A57C0000287500005475000030
:1071A0004A01002034000020597C0000000000004B
:1071B000747400004201002000000000F93A000051
:1071C000DF6E000000000000DB670000947100002B
:1071D000116C000000000000DB67000000000000F0
:1071E000DB67000000000000DB6700007941000061
:1071F000DF6E000000000000DB6700000000000000
:10720000DB67000000000000DB67000000000000FA
:10721000DB67000000000000DB67000000000000EA
:10722000DB67000000000000DB67000000000000DA
:10723000DB67000000000000DB67000000000000CA
:10724000DB670000000000001933000000000000B0
:10725000DB67000000000000DB67000000000000AA
:10726000DB67000000000000DB670000000000009A
:10727000DB67000000000000DB670000000000008A
:10728000DB67000000000000DB670000000000007A
:10729000DB67000000000000DB670000000000006A
:1072A000DB67000000000000DB670000000000005A
:1072B000DB67000000000000DB670000000000004A
:1072C000DB67000000000000DB670000000000003A
:1072D000DB67000000000000DB670000000000002A
:1072E000DB67000000000000DB670000000000001A
:1072F000DB67000000000000DB6700008071000019
:10730000116C000000000000DB67000000000000BE
:10731000DB67000000000000DB67000000000000E9
:10732000DB67000000000000DB67000000000000D9
:10733000DB67000000000000DB670000E277000070
:1073400003000000FFFFFFFFFFFFFFFFFFFFFFFF46
:107350000200000000000000054C00003D4C000051
:107360000338FDD87047000002000000050000004F
:1073700001000000997B00008C73000002000000F7
:107380000500000002000000050000005B00000096
:1073900006000000000000000000000000C0000027
:1073A000A87100000100000000C000000002000001
:1073B000A87100000200000000C0000000A007004B
:1073C000A87100000300000000C20000009E07003A
:1073D000A87100000400000000C20000009E070029
:1073E000A8710000050000000060080000A0070070
:1073F000A871000000000000B76700000000002036
:107400000000000000000B06401D002040000000AE
:1074100000000B15020000001C74000000000000BA
:107420002F7C00002600020200000020377C0000B4
:1074300022000B11952300006523000000000000CE
:10744000B5240000D92300004D7C0000CF69000066
:10745000D5690000537C0000B56900004569000053
:10746000A769000000000000BB68000000000000E9
:1074700000000000FD6900008127000011270000C6
:107480006D2600005D26000004000000FF000000E3
:10749000FFFF00000003005000000000010000009A
:1074A0000060004000000000FFFFFFFF00000050F0
:1074B000000000000000000000600040000000002C
:1074C00089290000EB6A0000F96A0000116B0000D6
:1074D0001D6B0000296B0000F5270000436B0000C6
:1074E000000000001A00000000001A001400000054
:1074F000000016001F00000000001600008002407F
:1075000002000000000000000C7500000080024036
:107510001875000001000000207500000200000046
:107520002F0000002D00010000200040020000009C
:107530000000000038750000002000404475000085
:10754000010000004C750000020000000600000071
:1075500008000100C96B0000192D0000BB6B000082
:107560000200000005000000DC700000DC7000007C
:10757000247100002C71000044710000447100006F
:10758000FF8FFFFFFF8FFFFFFE8FFFFFFE8FFFFFCD
:10759000FD8FFFFFFC8FFFFFFC8FFFFF436F756CBC
:1075A00064206E6F74206C6F636B20706F776572F0
:1075B0002073617665206D75746578006D757465EE
:1075C000785F667265652063616C6C6564207769BD
:1075D0007468204E554C4C20706172616D65746505
:1075E0007200000043616E277420696E69746961DE
:1075F0006C697A65206D757465782C2077617320CD
:107600004E554C4C0D0A0000FFFFFFFFFFFFFFFF30
:10761000FFFFFFFF0000000000000000000000006E
:1076200001000000FFFFFFFFFCFFFFFFFFFFFFFF68
:10763000FFFFFFFF0000000000000000000000004E
:1076400001000000FFFFFFFF512563FCC2CAB9F330
:10765000849E17A7ADFAE6BCFFFFFFFFFFFFFFFF09
:1076600000000000FFFFFFFF0000000096C298D856
:107670004539A1F4A033EB2D817D0377F240A4635B
:10768000E5E6BCF847422CE1F2D1176BF551BF3764
:107690006840B6CBCE5E316B5733CE2B169E0F7C37
:1076A0004AEBE78E9B7F1AFEE242E34FFFFFFFFFAC
:1076B0007F000000800000000000000000000000CB
:1076C000FFFFFFFF7F0000008000000000000000BF
:1076D0000000000067E6096A85AE67BB72F36E3C86
:1076E0003AF54FA57F520E518C68059BABD9831F8D
:1076F00019CDE05B77C295F360D2EF7F3552500F22
:107700002CB6798025633A205374617274696E6770
:1077100020626F6F746C6F616465720A0025633A52
:1077200020556E61626C6520746F2066696E6420FE
:10773000626F6F7461626C6520696D6167650A00D4
:1077400025633A20426F6F746C6F616465722063C9
:107750006861696E6C6F61642061646472657373E3
:10776000206F66667365743A20307825780A0025A4
:10777000633A204A756D70696E6720746F20746873
:107780006520666972737420696D61676520736C2A
:107790006F740A0025633A2050726F746563742019
:1077A0006D6375626F6F7420666C617368206661CB
:1077B000696C65642C2063616E63656C2073746111
:1077C000727475702E0A0025633A204E65766572D4
:1077D0002073686F756C64206765742068657265D6
:1077E0000A006D6375626F6F740025633A20696EDD
:1077F00076616C696420666C617368204944202559
:10780000643B2065787065637465642025640A00B4
:107810002A8648CE3D030107002A8648CE3D020154
:107820000025633A20556E61626C6520746F206498
:10783000657465726D696E6520666C61736820732E
:107840006563746F72206F662074686520696D616E
:10785000676520747261696C65720A007072696D87
:10786000617279007365636F6E646172790025637C
:107870003A20496D61676520696E2074686520252E
:107880007320736C6F74206973206E6F742076613F
:107890006C6964210A0025633A20256420737461B1
:1078A000747573207772697465206661696C7320E2
:1078B000706572666F726D696E672074686520739B
:1078C0007761700A0025633A204661696C6564201F
:1078D000746F206F70656E20666C617368206172D2
:1078E00065612049442025642028696D6167652011
:1078F000256420736C6F74202564293A2025642C3C
:107900002063616E6E6F7420636F6E74696E75654F
:107910000A0025633A204661696C656420726561DE
:1079200064696E6720736563746F72733B20424FA6
:107930004F545F4D41585F494D475F534543544F46
:1079400052533D2564202D20746F6F20736D616C40
:107950006C3F0A0025633A204661696C65642072B9
:10796000656164696E6720696D616765206865613E
:10797000646572733B20496D6167653D25750A003A
:1079800025633A204661696C6564207265616469AB
:107990006E6720626F6F74207374617475733B201F
:1079A000496D6167653D25750A0025633A20706160
:1079B0006E6963210A0025633A2044657465637427
:1079C000656420696E636F6E73697374656E74208D
:1079D000737461747573210A0025633A2043616EE4
:1079E0006E6F7420757067726164653A206E6F7493
:1079F000206120636F6D70617469626C6520616DD8
:107A00006F756E74206F6620736563746F72730A8E
:107A10000025633A2043616E6E6F74207570677243
:107A20006164653A206D6F726520736563746F726F
:107A300073207468616E20616C6C6F7765640A00F6
:107A400025633A2043616E6E6F74207570677261B2
:107A500064653A206E6F742073616D652073656391
:107A6000746F72206C61796F75740A0062616400D2
:107A7000676F6F6400756E736574005072696D6135
:107A8000727920696D6167650025633A2025733A34
:107A9000206D616769633D25732C20737761705F8A
:107AA000747970653D307825782C20636F70795F2C
:107AB000646F6E653D307825782C20696D6167654F
:107AC0005F6F6B3D307825780A005365636F6E6495
:107AD00061727920696D6167650025633A20426FA4
:107AE0006F7420736F757263653A207072696D618F
:107AF000727920736C6F740A0025633A20426F6FAD
:107B00007420736F757263653A206E6F6E650A003C
:107B100025633A205374617274696E6720737761CC
:107B200070207573696E67206D6F766520616C6774
:107B30006F726974686D2E0A0025633A204E6F7467
:107B400020656E6F75676820667265652073706169
:107B5000636520746F2072756E2073776170207575
:107B60007067726164650A0025633A2072657175F9
:107B7000697265642025642062797465732062757A
:107B800074206F6E6C7920256420617265206176A7
:107B900061696C61626C650A003059301306072A0E
:107BA0008648CE3D020106082A8648CE3D030107DD
:107BB000034200042ACB403CE8FEED5BA44995A1BA
:107BC000A91DAEE8DBBE1937CD14FB2F245737E5CE
:107BD000953988D994B9D65AEBD7CDD5308AD6FE07
:107BE00048B24A6A810EE5F07D8B6834CC3A6AFC73
:107BF000538EFAC12D0020002B0030780030580041
:107C0000286E696C29004661696C656420746F2078
:107C10007265626F6F743A207370696E6E696E6719
:107C200020656E646C6573736C792E2E2E0A004687
:107C30004C4153485F30005352414D5F3000636CFC
:107C40006F636B4034303030303030300068666302
:107C50006C6B006C66636C6B00666C6173682D63A3
:107C60006F6E74726F6C6C65724034303031653099
:107C70003030006770696F4035303030303330302D
:107C8000006770696F403530303030303030000080
:107C90000102030405060775617274403430303206
:107CA00038303030007561727440343030303230EA
:107CB0003030007065726D00746573740042554712
:107CC0003B2063616E27742068617070656E00727E
:107CD00065766572740025633A205365636F6E6440
:107CE00061727920696D616765206F6620696D61D9
:107CF00067652070616972202825642E29206973C8
:107D000020756E726561636861626C652E205472C5
:107D100065617420697420617320656D7074790ADF
:107D20000025633A20496D61676520696E64657856
:107D30003A2025642C205377617020747970653A5D
:107D40002025730A0025633A20496D616765206923
:107D50006E6465783A2025642C2053776170207416
:107D60007970653A206E6F6E650A000401040304A1
:107D700002040104010403010303040104000000E0
:107D800000000101000000000000203030303030E1
:107D900030303030303030303000015465726D6931
:107DA0006E616C00000000000000545452205245E7
:107DB00047474553002A2A2A20426F6F74696E672D
:107DC000206E524620436F6E6E6563742053444BA1
:107DD0002076332E352E39392D6E6373312D3320B5
:107DE0002A2A2A0A0000000001000000FFFFFFFF0E
:107DF000A3680000E764000094730000B568000009
:107E00000000000000C201000001030000000000AB
:107E1000C8100020C7100020000000000000000073
:107E200000C201000001030000000000CA10002091
:107E3000C910002000000000000000000000000049
:107E40000000000000000000000000000000000032
:107E50000000000000000000000000000000000022
:107E60000000000000000000000000000000000012
:107E70000000000000000000000000000000000002
:107E800000000000000000000000000000000000F2
:107E900000000000000000000000000000000000E2
:107EA000000000000000000008000000FF000000CB
:107EB000000000000300000000000000FFFF0F00B2
:107EC000D8000020D800002000000000F946000083
:107ED000F00000200C01002004010020000100201F
:107EE000FC00002038010020300100202801002083
:107EF0000000000020010020114A00005D49000040
:107F000091490000D9490000B40F00203A00003A1E
:107F1000B80F00203A00003ABC0F00203A00003AA7
:107F2000C00F00203A00003A0000000000000000EE
:087F30000000000015E015E05F
:10C000003DB8F39600000000000200002078070011
:10C010000000000000000000000000000000000020
:10C02000FFFFFFFFFFFFFFFFFFFFFFFFFFFFFFFF20
:10C03000FFFFFFFFFFFFFFFFFFFFFFFFFFFFFFFF10
:10C04000FFFFFFFFFFFFFFFFFFFFFFFFFFFFFFFF00
:10C05000FFFFFFFFFFFFFFFFFFFFFFFFFFFFFFFFF0
:10C06000FFFFFFFFFFFFFFFFFFFFFFFFFFFFFFFFE0
:10C07000FFFFFFFFFFFFFFFFFFFFFFFFFFFFFFFFD0
:10C08000FFFFFFFFFFFFFFFFFFFFFFFFFFFFFFFFC0
:10C09000FFFFFFFFFFFFFFFFFFFFFFFFFFFFFFFFB0
:10C0A000FFFFFFFFFFFFFFFFFFFFFFFFFFFFFFFFA0
:10C0B000FFFFFFFFFFFFFFFFFFFFFFFFFFFFFFFF90
:10C0C000FFFFFFFFFFFFFFFFFFFFFFFFFFFFFFFF80
:10C0D000FFFFFFFFFFFFFFFFFFFFFFFFFFFFFFFF70
:10C0E000FFFFFFFFFFFFFFFFFFFFFFFFFFFFFFFF60
:10C0F000FFFFFFFFFFFFFFFFFFFFFFFFFFFFFFFF50
:10C10000FFFFFFFFFFFFFFFFFFFFFFFFFFFFFFFF3F
:10C11000FFFFFFFFFFFFFFFFFFFFFFFFFFFFFFFF2F
:10C12000FFFFFFFFFFFFFFFFFFFFFFFFFFFFFFFF1F
:10C13000FFFFFFFFFFFFFFFFFFFFFFFFFFFFFFFF0F
:10C14000FFFFFFFFFFFFFFFFFFFFFFFFFFFFFFFFFF
:10C15000FFFFFFFFFFFFFFFFFFFFFFFFFFFFFFFFEF
:10C16000FFFFFFFFFFFFFFFFFFFFFFFFFFFFFFFFDF
:10C17000FFFFFFFFFFFFFFFFFFFFFFFFFFFFFFFFCF
:10C18000FFFFFFFFFFFFFFFFFFFFFFFFFFFFFFFFBF
:10C19000FFFFFFFFFFFFFFFFFFFFFFFFFFFFFFFFAF
:10C1A000FFFFFFFFFFFFFFFFFFFFFFFFFFFFFFFF9F
:10C1B000FFFFFFFFFFFFFFFFFFFFFFFFFFFFFFFF8F
:10C1C000FFFFFFFFFFFFFFFFFFFFFFFFFFFFFFFF7F
:10C1D000FFFFFFFFFFFFFFFFFFFFFFFFFFFFFFFF6F
:10C1E000FFFFFFFFFFFFFFFFFFFFFFFFFFFFFFFF5F
:10C1F000FFFFFFFFFFFFFFFFFFFFFFFFFFFFFFFF4F
:10C20000C074022029000600079E060015000600E3
:10C2100015000600150006001500060000000000CD
:10C22000000000000000000000000000F500060013
:10C2300015000600000000008D0006001500060035
:10C24000550106007DCD060055010600550106008A
:10C25000550106005501060055010600550106006E
:10C260004DCD0600550106005501060067CD0600BC
:10C27000550106005501060055010600550106004E
:10C28000550106005501060055010600550106003E
:10C29000550106005501060055010600550106002E
:10C2A000550106005501060055010600550106001E
:10C2B000550106005501060055010600550106000E
:10C2C00055010600550106005501060055010600FE
:10C2D00055010600550106005501060055010600EE
:10C2E00055010600550106005501060055010600DE
:10C2F00055010600550106005501060055010600CE
:10C300002DE9F00791E8F807B2E802105B1854EB4A
:10C310000C04B2E802104D4156EB0C06B2E80210D4
:10C320004F4158EB0C08B2E8021059EB01095AEBE7
:10C330000C0A80E8F80780410130BDE8F00770473B
:10C340002DE9F00791E8F807B2E802105B1A74EBE8
:10C350000C04B2E802108D4176EB0C06B2E8021034
:10C360008F4178EB0C08B2E8021079EB01097AEB07
:10C370000C0A80E8F80780414042BDE8F0077047AA
:10C380002DE9F007524290E87800B1E880071740A5
:10C39000DB1918EA020854EB080419EA020955EB04
:10C3A00009051AEA020A56EB0A0678C090E87800F6
:10C3B000B1E8800717407B4118EA020854EB0804F3
:10C3C00019EA020955EB09051AEA020A56EB0A06B0
:10C3D00078C080410130BDE8F00770472DE9F007D3
:10C3E000524290E87800B1E880071740DB1B18EA5A
:10C3F000020874EB080419EA020975EB09051AEA48
:10C40000020A76EB0A0678C090E87800B1E8800767
:10C410001740BB4118EA020874EB080419EA020944
:10C4200075EB09051AEA020A76EB0A0678C0804124
:10C430004042BDE8F00770472DE9F00152424FF04D
:10C44000040890E8300091E8C000A31B1340E41AF0
:10C45000F618EB1B1340ED1AFF1830C0C0C1B8F13D
:10C460000108EED1BDE8F001704700BF00B592E8C9
:10C47000DC072DE9DC07B1E8805702B4A7FB0251C5
:10C480000A95A8FB020BE7FB6310E9FB62B00B9176
:10C49000A8FB0351EAFB6201E7FB64B5E7FB660515
:10C4A000E8FB6615CDF830B0A9FB03B6EAFB6316CE
:10C4B000ECFB6356E8FB640BE9FB641BEAFB645B83
:10C4C000ECFB646B0D90ACFB0230059CEEFB625004
:10C4D000E9FB6460EAFB64B0E7FB6431E8FB6451AC
:10C4E000069CE8FB6461E9FB64B1EAFB64010E931E
:10C4F000A7FB0432079CE7FB6462E8FB64B2E9FB3C
:10C500006402EAFB6412049CE9FB6453EAFB646383
:10C51000089CE7FB64B3E8FB6403E9FB6413EAFBF4
:10C5200064230F955DF8049B99E80006DDF8008010
:10C53000A9FB0854EAFB68B4DDF81080ECFB680442
:10C54000EEFB6814E9FB6824EAFB6834DDF804803C
:10C55000EEFB6865E9FB68B5EAFB6805DDF8148069
:10C56000ECFB6815EEFB6825E9FB6835EAFB6845DE
:10C570000F96DDF80880AEFB0876E9FB6806EAFB5B
:10C580006816DDF81880ECFB6826EEFB6836E9FBE0
:10C590006846EAFB6856DDF80C80ECFB68B7EEFBFA
:10C5A0006807E9FB6817EAFB6827DDF81C80ECFBED
:10C5B0006837EEFB6847E9FB6857EAFB686708B035
:10C5C00000BD00BF2DE9F14F87B0FFF74FFFDDF849
:10C5D0001C8008F1200888E8FF00FFBC87E87F087E
:10C5E000BDE8F08F00B591E89857A3FB0352019581
:10C5F000A3FB0401E3FB6420E3FB67100292A3FBAF
:10C600000752E3FB6802E4FB6415E3FB6805E3FB08
:10C6100069250391A4FB07B6E3FB6926E3FB6A5691
:10C62000E4FB670BE4FB682BE3FB6A5BE3FB6C6BEF
:10C630000490A4FB0810E4FB6950E3FB6C60E3FB8F
:10C640006EB0E7FB6721E4FB6951E4FB6A61E3FB41
:10C650006EB1E4FB6E010592A7FB0832E4FB6A624F
:10C66000E4FB6CB2E4FB6E02E7FB6E12E7FB68537F
:10C67000E7FB6963E4FB6CB3E7FB6C03E7FB6E135A
:10C68000E8FB6E230695A7FB0954E7FB6AB4E7FBBA
:10C690006C04E8FB6C14E8FB6E24E9FB6E34E8FBE9
:10C6A0006865E7FB6AB5E8FB6A05E8FB6C15E9FB22
:10C6B0006C25E9FB6E35EAFB6E450796A8FB09760B
:10C6C000E8FB6A06E9FB6A16E9FB6C26EAFB6C36B6
:10C6D000EAFB6E46ECFB6E56E8FB69B7E9FB6907BF
:10C6E000E9FB6A17EAFB6A27EAFB6C37ECFB6C474D
:10C6F000ECFB6E57EEFB6E6700BD00BF2DE9F14FFE
:10C7000087B0FFF76FFFDDF81C8008F1200888E88C
:10C71000FF00FFBC87E87F08BDE8F08F30B44FF022
:10C72000000310F8014B11F8015B013A84EA05049B
:10C7300043EA0403F5D1A3F101034FEAD37030BCFF
:10C74000704700BF4FF0000310F8012B013943EA96
:10C750000203F9D1A3F101034FEAD370704700BF80
:10C7600030B411F8014B12F8015B6C4000F8014B3A
:10C77000013BF6D130BC70472DE9F00791E8F8078E
:10C78000B2E802105B1854EB0C04B2E802104D4101
:10C7900056EB0C06B2E802104F4158EB0C08B2E819
:10C7A000021059EB01095AEB0C0A8941B3F1FF332E
:10C7B00074F1FF3475F1FF3576F1000677F100076B
:10C7C00078F1000879F101097AF1FF3A51F100019D
:10C7D0005B184C414D4156F1000657F1000758F1E6
:10C7E000000859EBD1795AEB010A80E8F807BDE857
:10C7F000F00770472DE9F00791E8F807B2E802105A
:10C800005B1A74EB0C04B2E802108D4176EB0C0657
:10C81000B2E802108F4178EB0C08B2E8021079EB15
:10C8200001097AEB0C0A89415B184C414D4156F1E4
:10C83000000657F1000758F1000859EBD1795AEB7F
:10C84000010A80E8F807BDE8F007704718EB040814
:10C8500059EB05095AEB060A5BEB070B5FF0000C7E
:10C860004CF1000C18EB050859EB06095AEB070AC6
:10C870005BEB070B50EB0C005FF0000C51EB0C0175
:10C8800052EB0C0263414CF1000CB8EB070879F154
:10C8900000097AF1000A7BEB040BA841B141A241E7
:10C8A000B3416CF1000CBBEB050BB041B941AA419F
:10C8B000BB416CF1000C4CF001068CF0020718EB48
:10C8C000060859EB6C095AEB6C0A7BEB6C0B70EBAE
:10C8D0006C0471EB6C0572EB670653EB6C076CEB49
:10C8E0006C0C18EB0C0059EB0C015AEB0C025BF1D1
:10C8F000000354F1000455F1000556EBDC7657EBCC
:10C900000C0770472DE9F14F87B0FFF7AFFDDDF859
:10C910001080DDF81490DDF818A0FFF797FFBDE850
:10C92000000FFFF793FF03B05DF8048B88E8FF006A
:10C93000BDE8F08F2DE9F14F87B0FFF753FEDDF82A
:10C940001080DDF81490DDF818A0FFF77FFFBDE838
:10C95000000FFFF77BFF03B05DF8048B88E8FF0052
:10C96000BDE8F08F2DE9F04F90E8F00F00F14000A6
:10C970004FF0040E59E0F0B4826BC36B04680525D8
:10C98000242687593C444FEA724787EAF24787EAF0
:10C9900092273C4442684FEAF21787EAB24787EA97
:10C9A000D2073C4440F8044B032D08BF6FF01B0630
:10C9B00087593A444FEA734787EAF34787EA932750
:10C9C0003A4443684FEAF31787EAB34787EAD30745
:10C9D0003A4440F8042B87593B444FEA744787EAAE
:10C9E000F44787EA94273B4444684FEAF41787EA00
:10C9F000B44787EAD4073B4440F8043B013DC0D12B
:10CA0000A0F13C00076A3C444FEA724787EAF247CC
:10CA100087EA92273C4402684FEAF21787EAB24756
:10CA200087EAD2073C44C463F0BC4FF0020288EAB4
:10CA3000781C8CEAF84C0BEBBC1C8AEA090303EA6D
:10CA4000080383EA0A039C4450F8043B9C4451F8D1
:10CA5000043B9C44674444EA050B0BEA060B04EADA
:10CA600005034BEA030BE34484EAF42383EA3453DB
:10CA70000BEBB30B87EA771C8CEAF74C0AEBBC1C78
:10CA800089EA080303EA070383EA09039C4450F890
:10CA9000043B9C4451F8043B9C4466444BEA040A22
:10CAA0000AEA050A0BEA04034AEA030AE2448BEAAB
:10CAB000FB2383EA3B530AEBB30A86EA761C8CEA33
:10CAC000F64C09EBBC1C88EA070303EA060383EA79
:10CAD00008039C4450F8043B9C4451F8043B9C449C
:10CAE00065444AEA0B0909EA04090AEA0B0349EA20
:10CAF0000309E1448AEAFA2383EA3A5309EBB309CA
:10CB000085EA751C8CEAF54C08EBBC1C87EA060329
:10CB100003EA050383EA07039C4450F8043B9C4462
:10CB200051F8043B9C44644449EA0A0808EA0B08AB
:10CB300009EA0A0348EA0308E04489EAF92383EA98
:10CB4000395308EBB30884EA741C8CEAF44C07EB05
:10CB5000BC1C86EA050303EA040383EA06039C443B
:10CB600050F8043B9C4451F8043B9C44E34448EA9D
:10CB7000090707EA0A0708EA090347EA03076744BF
:10CB800088EAF82383EA385307EBB3078BEA7B1C68
:10CB90008CEAFB4C06EBBC1C85EA040303EA0B039E
:10CBA00083EA05039C4450F8043B9C4451F8043B41
:10CBB0009C44E24447EA080606EA090607EA080335
:10CBC00046EA0306664487EAF72383EA375306EB0F
:10CBD000B3068AEA7A1C8CEAFA4C05EBBC1C84EAA0
:10CBE0000B0303EA0A0383EA04039C4450F8043B62
:10CBF0009C4451F8043B9C44E14446EA070505EA9D
:10CC0000080506EA070345EA0305654486EAF623B4
:10CC100083EA365305EBB30589EA791C8CEAF94CB3
:10CC200004EBBC1C8BEA0A0303EA090383EA0B0347
:10CC30009C4450F8043B9C4451F8043B9C44E04421
:10CC400045EA060404EA070405EA060344EA030485
:10CC5000644485EAF52383EA355304EBB304013ACF
:10CC60007FF4E5AEA0F14000BEF1010E7FF483AE8B
:10CC7000A0F1400C9CE80F00001949199219DB192A
:10CC8000ACE80F009CE80F004044494452445B4428
:10CC9000ACE80F00BDE8F08F2DE9F047A74D86B056
:10CCA000EA7B0023CDE902338DF80E206A7D8DF8F2
:10CCB0001020AA7D2B788DF81120EA7D8DF809309F
:10CCC0008DF812206B782A7E8DF80A308DF81320AB
:10CCD000AB786A7E8DF80B308DF81420EB7895F8E0
:10CCE00026208DF80C30C41D2B798DF80D300746A9
:10CCF0000E4624F007040AB18DF80F30002E08BF4D
:10CD0000204602A918BF002000F09EFD95F8008083
:10CD10006B784FF0000A984404445FFA88F8D146D3
:10CD20005FFA8AF34345C0F0F7800334002E24F005
:10CD3000030449460CBF2046002000F06DFFA9788F
:10CD4000044479B1EB78EA7BE01C20F00304002E68
:10CD50001A4408BF20466B89D2B218BF002000F0E9
:10CD6000CFFF044495F827308BB1697A79B195F8F3
:10CD70002830E01C002B20F0030414BFFF222522E2
:10CD8000002E0CBF2046002001F0AAF80444297BA5
:10CD900081B1AB7823B995F827305BB16B7A4BB191
:10CDA000E01D20F00704002E0CBF204600200EF0EE
:10CDB0006BFF0444624B1B6863B1297951B1E01CDD
:10CDC00020F00304002E08BF20466A7B18BF002015
:10CDD000984704445B4B1B6853B1A97B41B1E01CED
:10CDE00020F00304002E0CBF204600209847044486
:10CDF000554BD3F80080B8F1000F0FD0E97B69B133
:10CE0000E01CAB7C009320F00304002E08BF2046FA
:10CE10006B7C2A7C18BF0020C047044495F826305C
:10CE20006BB1297959B1E01C20F00304002E08BF32
:10CE300020462A7D18BF002001F088F80444E87FCE
:10CE400068B16B7EA97D033424F0070444F0040428
:10CE5000194422463346C9B201F0B8F8044495F8A3
:10CE60002010002962D0E01D20F00708002E4FF0AE
:10CE7000FB020CBF404600201AF047F808EB000404
:10CE80001EB9FB21404613F0F9FEA97E00294FD0C0
:10CE9000AB7F002B4CD0E01D20F00708002E4FF494
:10CEA0008C720CBF404600201AF02FF808EB0004EB
:10CEB0002B7EA97DA87F033424F0070444F00404EA
:10CEC000194422463346C9B201F072F804442EB91F
:10CED000A97E4FF48A72404613F0F2FEEB6A13B15A
:10CEE00006B9EC62283495F8241089B1E01D20F0D1
:10CEF0000705002E42F210720CBF284600201AF0DF
:10CF000004F82C1826B942F21071284613F0DEFE00
:10CF1000E01B06B0BDE8F0872B7AEA79A979687939
:10CF200019F0C5FF0AF1010A8144F9E68846A7E72E
:10CF3000002ED3D1324631463046CDE79825002029
:10CF4000540000205C000020580000208FB572B60D
:10CF5000194B1D6BE5B9BFF34F8F1849184BCA68C1
:10CF600002F4E0621343CB60BFF34F8F00BFFDE7D5
:10CF7000B4FBF6F4DAB20133002CF9D102F110035C
:10CF80006B440A2603F80C4C32B901A8A847E2E723
:10CF9000044600230A26EDE7531E04AC54FA83F43A
:10CFA000DAB2C3B2B3FBF6F706FB1733303304F83B
:10CFB0000C3CB0FBF6F0E7E79825002000ED00E020
:10CFC0000400FA051FB5164C237A8DF80930E37971
:10CFD0008DF80830A379ADF80C3002A86379ADF86C
:10CFE0000A300CF0C5FE18B1B5210320FFF7AEFFE3
:10CFF000012301A88DF804301BF075FA08B1B9219E
:10D00000F3E7A07C0CF0ECFE08B1BC21EDE7607CFE
:10D010000CF0E0FE08B1BD21E7E704B010BD00BF91
:10D020009825002038B50546002842D017F046FB69
:10D0300010B94FF0FF3038BD14F060F9B0F5FA7F49
:10D04000F7D81E4C1E482563002500F0B5FA2622AD
:10D050002946204684F8345084F8355084F8275007
:10D0600084F82850E56284F8265017F001FE1B2250
:10D07000627140F21B32E28040F2023240F2011350
:10D0800022811F222380628101234FF40272A37048
:10D09000A281237544F60112FB232282A3836384B9
:10D0A000EFF3108472B600F0B1FF2CB962B62046DF
:10D0B000C1E76FF01500BEE72846BCE798250020C1
:10D0C000C5CF000010B5002840F0A680554C94F85C
:10D0D0003430002B40F09D80A1B1002A6DD0013981
:10D0E000142900F29980DFE801F00B191C2C545C24
:10D0F00075325F6270383E4B507A7D8B8E91820024
:10D100001378237001210020FFF7C6FDB0F5803FA2
:10D1100080F28580012384F8353010BD1378637068
:10D12000F0E79378002B48D0D378002B45D01378C4
:10D130001A2B42D953781A2B3FD91368C4F80530FB
:10D14000E0E71378E278934237D3A370DAE71378F5
:10D15000A278934231D8E370D4E71378A27893424F
:10D160002BD8E373CEE713783BB35378013BDBB2A4
:10D17000F82B22D8138823822B4B92789A70C1E720
:10D180001078E07411F0E6FCBCE71378ABB12375BE
:10D19000B8E7137894F827200AB1012B0DD96372F0
:10D1A000B0E713886381ADE713782371AAE794F899
:10D1B0002610137821B9012B04D86FF01500ACE7C5
:10D1C000002BFAD0137863739CE71378082BF4D8FC
:10D1D000A37397E71388FF2BEFD8237392E7137895
:10D1E00063758FE713780E2BE7D8A3758AE713686A
:10D1F0000E49C4F81A3053684B6013890B8181E7DC
:10D200001378E3757EE7137863767BE713782376EC
:10D2100078E74FF0FF3080E76FF02C007DE76FF08C
:10D220000B007AE798250020A8250020B2250020D1
:10D2300070B50D460646F0B1E9B111F007041AD1F8
:10D2400000F0EEF8D0B1304617F0E4FA0D4E21466A
:10D2500086F836002846FFF71FFD1DF0BDFB96F847
:10D260003600F16A0CF08EFEFFF7ACFE012386F863
:10D270003430204670BD6FF01500FBE74FF0FF30F3
:10D28000F8E700BF9825002010B5084C94F834301A
:10D290002BB10CF093FE94F8360017F0D7FA19F082
:10D2A0007BFF002084F8340010BD00BF98250020CB
:10D2B00050B1074B03F1140253F8041B40F8041B50
:10D2C0009342F9D1002070476FF01500704700BFFE
:10D2D00008120800074B93F8352010B532B993F8BF
:10D2E00034401CB90CF0E0FD204610BD4FF0FF307B
:10D2F000FBE700BF98250020074B93F8352010B5B9
:10D3000032B993F834401CB90CF0E2FD204610BD50
:10D310004FF0FF30FBE700BF9825002010B50B4C05
:10D3200094F835307BB994F8343063B994F82830E8
:10D3300033B10CF00BFE012384F82730002010BD20
:10D340000CF0E8FDF7E74FF0FF30F8E798250020F4
:10D35000074B93F8352010B532B993F834401CB917
:10D360000CF052FD204610BD4FF0FF30FBE700BF30
:10D3700098250020074B93F8352010B532B993F863
:10D3800034401CB90CF032FD204610BD4FF0FF3088
:10D39000FBE700BF98250020074B93F8352010B518
:10D3A00032B993F834401CB91BF0E6F8204610BDA2
:10D3B0004FF0FF30FBE700BF98250020074B93F8A4
:10D3C000352010B532B993F834401CB91BF0D7F8AA
:10D3D000204610BD4FF0FF30FBE700BF982500202E
:10D3E000074B93F8352010B532B993F834401CB987
:10D3F0001BF0C7F8204610BD4FF0FF30FBE700BF21
:10D400009825002007C8024B83E8070000207047DA
:10D41000D0250020014B9B68184700BFD025002075
:10D42000024B9868003818BF01207047D0250020B3
:10D4300073B52E4D031D04462B6028460DF08CFE5F
:10D440000228064606D12949204618F02DFE30460E
:10D4500002B070BD042842D12B78092B0AD0252BAD
:10D460001ED02946204618F084FEB0F5817F2DD3CA
:10D47000722112E005213E2018F0E9FD0028F0D1CC
:10D48000EB782A7901A943EA02236846ADF8003017
:10D4900019F08DFA0028D0D053210820FFF756FD4F
:10D4A0001A213E2018F0D3FD0028DAD16B68C3F3AF
:10D4B0000F23ADF804306946112301A88DF806301A
:10D4C00019F097FA0028B8D06521E6E70028B4D013
:10D4D000A178207818F0BBFD0028B8D1ADE7082866
:10D4E000B5D10249204618F00EFEB0E7DC25002039
:10D4F000074B4FF0FF3141F6FF72C3E900120549B7
:10D500000022C1E900221F21C3E90212704700BFB7
:10D5100000000020E02600203F280CD801380B4BEB
:10D52000C0F3421200F01F0053F8223023FA00F03B
:10D5300000F001007047FF2806D04038C0F34212C7
:10D54000034B00F01F00EFE70120704700000020B0
:10D55000E02600200146074B006849681A4603C2CE
:10D5600040F48C221A6041F0107242F4FF625A605B
:10D57000704700BF000000200246024B006851685F
:10D5800003C37047E02600200246024B0068516842
:10D5900003C37047080000200138064BC0F3421255
:10D5A00003EB820300F01F009B6823FA00F000F0F9
:10D5B0000100704700000020014B1860704700BF59
:10D5C000E826002010B5FFF793FF1AF0CAF9034BC5
:10D5D0001B68044603B19847204610BDE82600208A
:10D5E0000B880288F0B5C3F30E049EB204F1180351
:10D5F000C57CC35A05352A442B4497B213FA82F3EB
:10D60000013B4288B3FBF7F313FB07439BB29A42FB
:10D61000044A93BF22EA0603324013439BB20B80B5
:10D62000F0BD00BF0080FFFF10B5114B00EB4104BF
:10D630001A786389B3FBF2F303FB0223013A1A441D
:10D64000B2F5706F027928BF00231A448378B2FBC9
:10D65000F3F0194403FB1020091AB1FBF3F003FBAC
:10D66000101313446FEA43436FEA5343638110BDC1
:10D67000EC26002010B5124BE0B15A78022A04D0F3
:10D6800040F259111720FFF761FC03225A7002681B
:10D6900012F0070102D04FF4AF71F3E75C685A60F3
:10D6A000224402609A60BDE81040302203F10C0071
:10D6B00017F0DEBA01225A70C3E9010010BD00BFA5
:10D6C000EC2600202DE9F041254E96F801E00EF001
:10D6D000FD0CBCF1010F04D040F273111720FFF7CD
:10D6E00035FC91F80680B8F1080F02D940F27511A7
:10D6F000F4E7CF7997B34546022D726838BF02250B
:10D700007B1D5C0002EB43036A1E13446D422B40F9
:10D710008D884544013DC8F100022A404FF6FE7550
:10D72000AA4202D94FF4C071D8E7BEF1030F12D15B
:10D7300006EB80001C1BC56815B140F28511CDE7D2
:10D74000C460A770228084F803C0087A0968207139
:10D75000080CE080218107FB02337360BDE8F08193
:10D76000EC2600202DE9F047364C6378012B65D07C
:10D77000032B04D040F295111720FFF7E7FBD4E903
:10D7800001329A4202D04FF4CC71F5E725460023CE
:10D7900005F80C3B1E460B22994655F82200013A2B
:10D7A00058B190F804808178B8F1FF0F2FD180F83C
:10D7B00004908E423CBFCEB20123511CEDD103B187
:10D7C00026700B2640F6FF6955F826709FBB013E78
:10D7D000FAD2042363700020BDE8F08755F82CE0EE
:10D7E000BEF1000F06D09EF804A0C24504BF9EF80B
:10D7F00002E077440CF1FF3CBCF1000FEEDA394453
:10D80000FF2907D903B126704FF49A71B4E7944603
:10D810000027F1E70771CCE707EB41033846A3F88F
:10D820000A90FFF701FF08F10108BB785FFA88F161
:10D830008B42F1D8CBE74FF00008F6E7022360688F
:10D840006370C9E7EC2600202DE9FF474A788B7802
:10D850001344FF2B06460C4604D940F2AB111720A7
:10D86000FFF774FB0B78934202D940F2AF11F6E751
:10D87000DFF8D481009038B198F80130022B02D043
:10D880000020FFF7E1FF6846FFF7F4FE00276F4A2C
:10D890006378019208254FF45A7201A93846ADF811
:10D8A00008208DF80B308DF80A508DF80C70FFF7BA
:10D8B00009FF674AA378019201A94FF47A72012007
:10D8C000ADF808208DF80B308DF80A508DF80C70EB
:10D8D000FFF7F8FE5F4AE37801924FF0FF094FF43B
:10D8E000AC7201A90220ADF808208DF80B308DF83C
:10D8F0000A508DF80C90FFF7E5FE574A2379019204
:10D9000001A990220320ADF808208DF80B308DF886
:10D910000A508DF80C90FFF7D5FE63794F4A0192BB
:10D920008DF80B30A822012301A90420ADF80820AE
:10D930008DF80C308DF80A50FFF7C4FEA379484AE1
:10D940000192CDE902778DF80A508DF80B308DF8F1
:10D950000C901BB111F0F2F8ADF8080001A90520F8
:10D96000FFF7B0FE3F4AE3790192082580224FF08D
:10D97000FF0901A90620ADF808208DF80B308DF8BD
:10D980000C908DF80A50FFF79DFE237A364A0192DB
:10D990008DF80B307822022301A90720ADF808206A
:10D9A0008DF80C308DF80A50FFF78CFE2F4A637A01
:10D9B000019200274FF40A7201A92846ADF8082009
:10D9C0008DF80B308DF80A508DF80C70FFF77AFE49
:10D9D000274AA37A019201A94FF48C720920ADF86D
:10D9E0000820DFF890A08DF80B308DF80C908DF8A2
:10D9F0000A504FF48879FFF765FEE37A8DF80B3013
:10DA000001A90A20CDF804A0ADF808908DF80A50BD
:10DA10008DF80C70FFF756FE237B8DF80B3001A9B3
:10DA20000B20CDF804A0ADF808908DF80A508DF8C1
:10DA30000C70FFF747FEFFF795FED8F80400801B37
:10DA400004B0BDE8F08700BFEC260020F9A7020073
:10DA500055A50200590701009FA8020061EB0100D3
:10DA600091A9020095A90200B58701001D87010058
:10DA700009880100B1880100F8B54FF6FF730380F3
:10DA8000184B03EB81030546D868B8B18678037953
:10DA9000B3FBF6F206FB1233DBB219460A1D00EBAC
:10DAA0004202B2F902705488002F09DB0131B1FB48
:10DAB000F6F206FB1211C9B28B42EFD10020F8BD7D
:10DAC000FF29FBD0C4F30E03C4782B8024B940F2A5
:10DAD000C7211720FFF73AFA5380BDE8F84019F044
:10DAE000C5B900BFEC2600201E4B03EB810370B5C7
:10DAF000DC6805464CB3B0F5706F04D340F2D52115
:10DB00001720FFF723FA0146204619F091F9FF2864
:10DB1000014604D02046BDE8704019F0A7B9A078AE
:10DB2000B5FBF0F300FB1353DBB219460A1D04EBFF
:10DB30004206B6F90260002E09DB0131B1FBF0F2BA
:10DB400000FB1211C9B28B42F0D1002070BDFF2939
:10DB5000FBD08B4204EB42021CBF0023E3705580D4
:10DB6000D8E700BFEC260020094B03EB810310B57A
:10DB7000DC680146204619F05BF9FF28014604D015
:10DB80002046BDE8104019F071B9002010BD00BF5B
:10DB9000EC2600200F4B03EB810370B5DC680146D7
:10DBA0000646204619F044F9FF28054610D00146E4
:10DBB000204619F05BF9E2882389014643EA0243D3
:10DBC0003046984720462946FFF72EFD002070BDBD
:10DBD0000320FCE7EC26002038B50E4B827903EBDE
:10DBE00082030446D86808B9022038BD8278E179FA
:10DBF0009142F9D24B1CE37100EB41035D89B3F90B
:10DC00000A30002BF3DBA58019F030F920600020EA
:10DC1000EBE700BFEC26002070B5044610F00300CF
:10DC20000E4603D049211820FFF790F919F0A4F807
:10DC3000054624B103483146046019F09DF8284692
:10DC400070BD00BF282700202DE9F04F1E4C85B085
:10DC500092462268BDF83CB098468146BDF83830FF
:10DC60000D461AB95B211820FFF770F91A460A21F0
:10DC70005046039318F013FF5A46064609214046C2
:10DC800018F00DFF31180746206819F0A0F8039B23
:10DC9000C9F8000018B9286005B0BDE8F08F8419F4
:10DCA0002C60D9F800000093524631460A2318F040
:10DCB000A8FE2868CDF838B009234246394605B099
:10DCC000BDE8F04F18F09DBE2827002070B50E4625
:10DCD000044618F0EDFE0546304618F0E9FE044B08
:10DCE0002A1821461868BDE8704019F09AB800BF9C
:10DCF00028270020014B186819F05CB8282700205D
:10DD0000F8B511441D4EC9B210F00305317003D0AF
:10DD10004E210920FFF71AF91F2B19D89B009BB23F
:10DD2000033323F003039BB208B17060338101EB2E
:10DD300081047668E2004FF0010C00EBC404EFB2FE
:10DD4000B94212D8D01D03FB010020F00700F8BD36
:10DD5000FF2B4FEA430204D9FF339342DFDB93B238
:10DD6000DEE77C2AFBDC7C23DAE710B186F800C012
:10DD70007460013528361C44E1E700BF2C270020E1
:10DD800038B5144A147853680021C8B2844203D8C5
:10DD9000A9210920FFF7DAF8184601310578283360
:10DDA000002DF2D001241289447000214468817052
:10DDB0008161C161920800F12001051D21F8022B4B
:10DDC000994245F8044B1444F8D100234361037091
:10DDD00038BD00BF2C2700200A4B1B89B3F5FF7FFD
:10DDE0004FEA930006D25A089B1A9BB2984238BF5A
:10DDF00018467047B3F5EE6F01D8FF22F4E740F202
:10DE00007263F3E72C2700202DE9F8434B78804616
:10DE10000C4602F0040602F0FB07D3B1DFB12F4B32
:10DE2000D4F804901D89BFBB01236370AD08A761BE
:10DE3000E76104F120034A46211D04F1280023F87C
:10DE4000025B984241F8042B2A44F8D10023636115
:10DE500001E0002FE3D0002E4FF0FF0318BF022691
:10DE6000A370A3191B7D032B03D1022F1CBF013606
:10DE7000F6B2A31901221A7506F10C0204EB86060C
:10DE8000002324F812307268A370C8F80020A8F8A4
:10DE900004304046BDE8F883002114226170A018C8
:10DEA00016F0E6FEB5F5FF7F0FD26B08ED1AADB2A6
:10DEB00009EB0502C4F804902584A2606384C4F8C9
:10DEC0000C90A5842261E384C5E7B5F5EE6F4FF0B1
:10DED000FF03EBD940F27265EAE700BF2C27002070
:10DEE0002DE9F7431FFA82F81FFA81F904460F461D
:10DEF00016462E214A46404618F0D1FD05465CB133
:10DF00002E230146CDF800904246204618F079FDB8
:10DF1000034B1C601F715E71284603B0BDE8F0839F
:10DF200038270020024B5A7919791868FFF7D8BFB3
:10DF300038270020014B1868704700BF38270020A1
:10DF4000014B5879704700BF382700202DE9F7436F
:10DF500005460C46F7200521904618F0A0FD064620
:10DF600085B115F0030703D08F211920FEF7EEFFCE
:10DF7000DFF83890C9F81050A9F81400A5B2BBB268
:10DF80009D4204D806FB04F003B0BDE8F083B9F865
:10DF900014C0D9F81000CDF8008007FB0C00052351
:10DFA000F722314618F02DFD0137E8E74827002019
:10DFB00007B5CDE900230B4603490246081D19F0B9
:10DFC000C5F803B05DF804FB6027002013B5064CCC
:10DFD000CDE900230B46024604F1080104F10C00D0
:10DFE00019F0B4F802B010BD60270020024B0146C2
:10DFF000D3E9002018F015BF60270020024B01462E
:10E00000D3E9022018F00DBF60270020134B012236
:10E0100000214FF0FF309A60C3F80012C3F80803E4
:10E02000C3F80015C3F804259A60C3F80803C3F8C1
:10E030000015C3F804250A490A4A03F580334FF452
:10E040000040C3F80825C1F88000BFF34F8FBFF32D
:10E050006F8FC1F88001C3F80825704700F00040B9
:10E0600000E100E00000F63F8C46382300B50CF8D4
:10E07000033B054B8E4607CBCEF80300CCF80410CB
:10E08000CCF808205DF804FB7C27002070B5234DF8
:10E09000E96AAC6A0B7803F00303032B04F1A804CC
:10E0A0001AD16B8E2A8E0120034342F400626B86E4
:10E0B00020746B6B2A869847E96A237E013B18BF60
:10E0C000012323764B7833B1D4E92232013342F174
:10E0D0000002C4E9223270BD002BEED04B78002B39
:10E0E000EBD02A8E42F400622A86AA6B002AF2D074
:10E0F000FB2B08D895F83C3063B16B6B0021BDE871
:10E1000070402020184795F83D3043F0100385F803
:10E110003D3070BD01230370CFE700BF70270020A2
:10E1200010B5114C11F006FC10F0D8FE636B208E78
:10E1300000219847237E4BB9236C94F83D1094F846
:10E140003E009847002384F8443010BD94E807004F
:10E1500004F10C0383E807000449022204F11900CA
:10E160001BF0B4FBE8E700BF7027002069E0000067
:10E17000034B93F8443003B97047FFF7D1BF00BF9A
:10E1800070270020012923D838B51C4DAB6C0446FC
:10E190009847D8B195F83D30C3B995F8240010B12F
:10E1A0001CB1002038BD012CFCD195F84C30DC06A8
:10E1B000C3F300110ED50023AA6B92B1C0B16A8ED1
:10E1C000920715D5AB6DDB78022BEAD0012038BD64
:10E1D000012070472B6D1B78C3F30013C3F10103BB
:10E1E000EAE7B5F85420002AE8D00029EED0E5E7A8
:10E1F000002BEBD16A8E002AD3D0E7E770270020EE
:10E2000008B5094B93F84420022A07D1DA7A42F084
:10E210000102DA72BDE80840FFF782BF40F23D21FB
:10E220002720FEF793FE00BF70270020F8B5254C8D
:10E23000A66A236DE36296F8CB30054606F1A8077F
:10E2400094F85C000BB10430C0B296F871100DB9AF
:10E25000FF282ED011F0D2F897F823301BB3206E90
:10E2600011F05CFF94F82430216EE06A003B18BF87
:10E27000012384F88030D7E92223C4E91E2310F05B
:10E28000D9FD3DB996F8710010F00C0018BF282098
:10E2900011F0AEFF96F87010002012F011F8022372
:10E2A00084F84430F8BDE06A11F038FF10F016FE33
:10E2B000E7E796F870209142D0D011F09FF897F8D8
:10E2C0002330CBE77027002070B57F4CA56A82B061
:10E2D00095F8CB20002305F1A8068DF8053094F8B9
:10E2E0005C300AB10433DBB210B9FF2B00F0B2800E
:10E2F00095F87010FF2011F081F8B37D032B00F228
:10E30000DE80DFE803F0021D807094F8C230ADF8C3
:10E3100006306E48A5F860300CF048F8002840F050
:10E32000A180D4F8C4000DF105020DF1060118F02A
:10E33000E1FBA06520B196F86130002B00F0A980C8
:10E340006348A065F37DDB0003F00802037803F067
:10E35000F3031343327E920002F00402134303F0EE
:10E36000EF0203F00303032B027002D1C378022BE8
:10E3700012D0D4F8C40018F040FC48B9A06D02785F
:10E3800002F00303032B07D00CF036F8002879D1F4
:10E39000A06D027842F01002027096F8223013B19C
:10E3A0004378002B43D111F0B9FE10F097FDA66D14
:10E3B0000DF074F820B1337803F00303032B64D01D
:10E3C00095F87110012011F07BFFA36D414A188868
:10E3D0009978A4F84C00012384F8C830917084F82F
:10E3E000443002B070BD39480BF0E0FF002861D026
:10E3F000A06DC3781B2BA5D1012105F1100011F0F0
:10E4000033F8A06D9EE7B5F86030D4F8C400ADF8DD
:10E4100006300DF105020DF1060118F06BFBA06549
:10E4200000288FD140F2D6212720FEF78FFD206EE5
:10E4300011F074FE94F82410206ED6E92023B1FA6E
:10E4400081F67609A16D84F88060C4E91E2310F07E
:10E45000F1FCACE795F8713095F870108B427FF4C1
:10E4600049AF4AE7638EA16D626B43F08003802061
:10E4700063869047A06D01217174C3781B2B7FF4D4
:10E4800061AFBAE7A06D027886E7012012F0D6FEF0
:10E4900096E79DF805302BB1BDF806101BF0D1F9B9
:10E4A000A06D4FE703808370A06D01211BF0B3F8CE
:10E4B000A06DF1E740F2DF212720FEF747FD4FF482
:10E4C0003B712720FEF742FD70270020C82700205F
:10E4D00000280020BC2700202DE9F041434C94F88F
:10E4E0004420A56A012A82B006460F4605F1A80518
:10E4F0005FFA82F874D12B7C6BB1638E002143F0FC
:10E50000040363862974636B0420984794F82430CD
:10E510000BB185F81280A16D0A7802F00302032A7C
:10E5200036D04B78EBB10223AB7595F82330F3B1BD
:10E53000A36A93F87110D5E92223C4E91E2394F845
:10E54000243094F85C20003B18BF0123013984F883
:10E55000803007293FD8DFE801F03B133E113E3EF3
:10E560003E380123AB7595F82330002BE0D106B976
:10E5700007BB02B0BDE8F041FFF7D2BD4FF0030882
:10E58000002300931A494346012010F0DBFBEEE71D
:10E59000AB7D63B9638E43F0020363860220636B35
:10E5A0009847A16D0B7803F00303032BB9D1032324
:10E5B000AB75BAE731463046FFF7E4FD0028D8D105
:10E5C00002B0BDE8F041FFF731BE4FF00208D7E7D7
:10E5D0004FF00008D4E740F2B9310620FEF7B6FC50
:10E5E00040F25C412720FEF7B1FC00BF70270020FD
:10E5F000D827002070B50C4B0C4C0D4A1A6094F8CB
:10E60000443063B906460D4603F0FF02012104F1D0
:10E61000900022761AF0FFFF2665256670BDDF2187
:10E620002720FEF793FC00BF600000207027002029
:10E63000E8EE0000044A92F8443003F0FF000BB902
:10E64000107670470C20704770270020024B012283
:10E6500083F83C20704700BF702700202DE9F0436D
:10E66000BA4C85B002AD85E8030094F844100C98CC
:10E67000002940F0D481002A00F0D181002B00F065
:10E68000CE81002800F0CB8101F0FF06206495E8E0
:10E690000300A36404F1240383E80300A56A626312
:10E6A00084F83C6084F83D6084F8C96084F83E607A
:10E6B00084F8C8606686268610F036FF10F00EFCDF
:10E6C00095F9740011F050F805F1A807A86A11F047
:10E6D00009FD286A11F04EF897F8330011F054F84C
:10E6E00094F82430002B69D0042016F077FBEA69F7
:10E6F00041F64B539A4294BF4D20962010F034FEC1
:10E70000A36A93F8D832002B40F01C8195F8711061
:10E71000012011F021FA002863D08D4B186811F008
:10E72000E7FC6B69C4F8C430AB69C4F8CC3095F829
:10E730007F301BB9A96F002940F0C380D7F8900043
:10E74000D7F89410D7F89820D7F89C30DFF804C297
:10E75000ACE80F00D7F8A030C4F88130D7F8A43067
:10E76000CCF80D30A36A94F8241093F8C520A2F1D8
:10E770002600002938D1012803D993F8C60026289D
:10E7800038D193F81A2393F87080002A40D0B8F15A
:10E79000080F3DD0B8F1040F00F02681082A00F0E0
:10E7A0002381042A00F02081B8F1010F30D0012A22
:10E7B00014BF4FF002084FF0010829E0032016F0C3
:10E7C0000DFBEA6941F64B539A4294BF4D209620C7
:10E7D00010F0CAFD95F87010002011F0BDF9002866
:10E7E0009BD105B0BDE8F08301287BD993F8C60022
:10E7F000262877D0213A012A40F2CC80242800F044
:10E80000E78093F87080B8F1040F08BF4FF0080854
:10E8100005F13809414648461BF016F941461AF001
:10E82000E3FAB5F8443095F871100246934228BFD8
:10E830001346484684F8C2301BF0CCF895F87110A6
:10E8400097F82390B5F84C80082908BF04211AF0E6
:10E85000CBFAB9F1000F01D1043080B2404528BF96
:10E8600040465FFA80F884F8D0800CF017FE20B1A3
:10E87000B8F12B0F38BF4FF02B0894F8241084F810
:10E880005C80002957D197F82230002B3AD0012321
:10E8900084F88030D7E92023C4E91E2395F870302E
:10E8A000E86941F64B52013B904294BF042000209E
:10E8B000072B00F29C80DFE803F01E9F9A1D9A9AB6
:10E8C0009AA1B7F84E20BB8A93427FF437AFB5F8D0
:10E8D0007C201344A7F84E3095F87E00012212F0F8
:10E8E00091FC2BE793F8B62393F87080002A7FF40D
:10E8F0004EAF8DE7032100220B4600921549FB2203
:10E9000010F020FA0120FFF7DFFC134BD3F850354D
:10E9100023F00803032B00F087800023C4E90033B1
:10E92000A3602A88B98A97F83330618022802371E6
:10E9300005B0BDE8F08397F823307BB90120FFF7DD
:10E9400075FCE2E710F0DEFDE0E600BF7027002076
:10E9500060000020D827002000100040D7E92201E5
:10E9600095F871300122013BC4E91E0184F8802032
:10E97000072B3CD8DFE803F005443B043B3B3B4618
:10E9800003260021009133462A494246012010F017
:10E99000D9F9D3E724281BD000293FF432AF93F8EC
:10E9A0006E2193F8708050071ED412F001032BD112
:10E9B00093077FF52DAFB8F1080F3FF429AFB8F1F9
:10E9C000040F11D0B8F1010F18BF4FF002081FE774
:10E9D00000293FF416AF93F8691093F86E2193F86D
:10E9E00070800A405107E0D54FF0080810E740F268
:10E9F000B9310620FEF7AAFA01217CE702217AE765
:10EA00000126BEE70226BCE7B8F1080F3FF400AFCD
:10EA1000B8F1040F14BF98464FF00808F8E64FF419
:10EA2000A8712720FEF792FA4FF4FD712720FEF718
:10EA30008DFA00BFD827002010B5184C94F8443048
:10EA4000EBB194F824308BB194F84430022B20D1F0
:10EA5000A36AD3F8F00211F099FBA16A91F87F3014
:10EA600003F0FF020BB98B6F63B910BD94F844300B
:10EA7000012BF2D040F20F212720FEF767FAFFF7B3
:10EA80004FFBEAE791F87E00BDE81040114612F016
:10EA9000B9BB40F213212720FEF758FA7027002057
:10EAA000FFF73EBB014B1876704700BF7027002070
:10EAB000014B93F8C800704770270020024B188E56
:10EAC000C0F38020704700BF70270020014B93F8EF
:10EAD000C9007047702700202DE9F0411E4FBC6A25
:10EAE000820782B005460E4604F1A80411D4EB0754
:10EAF0000CD5D4E92232217E013342F100020129F2
:10EB0000C4E922320CBF00230123237602B0BDE802
:10EB1000F081BB6BDBB1B7F85420F96A18460332B9
:10EB200091F8018016F02CF80DF1020201A9F862AB
:10EB3000D7F8CC0018F016F9019818F0FDF801226A
:10EB400030604146D7F8CC0018F0A2F8CFE740F289
:10EB50004D412720FEF7FAF9702700202DE9F047F4
:10EB6000B24C86B00023CDE904338DF80F3094F811
:10EB70004430A56A022B06460F4605F1A8055FFA48
:10EB800083F840F0A281238E13F0400106D1636B1D
:10EB900040209847238E43F040032386002E5AD00E
:10EBA00095F82330002B40F01881D4F82CA09AF867
:10EBB000011089B2A4F85410002940F025810023E7
:10EBC000A3639AF80000238EE97DC0F3800243F42A
:10EBD00080739142238600F0CC80A26A94F82410BE
:10EBE00002F1A80999F81620EAB1022A00F053812F
:10EBF000002389F8163021B199F81220002A40F03C
:10EC00003F8199F81130002B40F0168199F81730A8
:10EC1000D4F82CA0012B0CBF0023012389F8173056
:10EC20009AF80000238E43F4806222862A7EC0F385
:10EC3000C0039A424FF0000900F0A2800CF02EFCB5
:10EC4000C0B19AF8003003F00303032B12D1012066
:10EC500012F0F4FA0EE095F82320002A40F0B98073
:10EC600043F40073238694F8C930013384F8C93023
:10EC70004FF0000995F822305BB394F82430A26A73
:10EC8000B3FA83F3D06992F870105B0984F880308E
:10EC900041F64B53984294BF04200020D5E920232D
:10ECA0000139C4E91E23072900F2E280DFE811F0F0
:10ECB0008E000800E0008B00E000E000E0000A00A9
:10ECC0004FF001080022009259494346FB2210F000
:10ECD00039F847B994F8C9100120FFF753FA0746ED
:10ECE000002800F0998011F059FB01279DF80F30A2
:10ECF0007BBBB9F1000F08D094F82430002B59D118
:10ED0000B4F809300133A4F809303EB3B4F8053043
:10ED100000220133A4F8053084F8C92045480CF0DE
:10ED2000F1FE049840B118F007F8A16A002343727D
:10ED3000082201301AF0B8FD059B33B1A16A002208
:10ED40001A72059810221AF0AFFD6FB906B0BDE82F
:10ED5000F08705A90220FFF7BFFECAE7B4F8073025
:10ED60000133A4F80730D9E7FFF7DAF906B0BDE8B8
:10ED7000F0872A7EC0F3C0039A42B1467FF45EAFAB
:10ED80000CF08CFB00284AD0D4F82CA09AF8003064
:10ED900003F00303013B012B41D89AF8012094F8BA
:10EDA000D0309A423BD994F83D3043F0100384F8B8
:10EDB0003D3043E7B4F80530B4F80710AA8A0B4396
:10EDC0001343A2D09CE74FF003087BE74FF0000805
:10EDD00078E710F0EDF8238E42E710F0AFF810F06E
:10EDE00091F8D4F82CA09AF8011000287FF4E1AE35
:10EDF000002942D09AF800302A7EC3F3C0039A4219
:10EE00005DD089B2A4F85410D4F8CC0017F016FFE6
:10EE1000D4F82CA0A063D4E6FFF756FA66E70DF10C
:10EE20000F00FFF733F9D4F82CA007E77027002074
:10EE3000D8270020942700204FF0000A89F811A05D
:10EE40000BF0C4FA00284AD0638E43F008036386AF
:10EE50005146636B08209847D9F880300133C9F8D0
:10EE60008030D9F8843043F10003C9F88430CDE60E
:10EE700040F2B9310620FEF769F8A4F854109EE676
:10EE800089F812301946638E43F010036386102010
:10EE9000636B9847B5E6D4F8C40004A917F04DFE9B
:10EEA000C0B1D9F8803094F824100133C9F880300B
:10EEB000D9F8843043F10003C9F8843098E601237F
:10EEC00084F83E30FFF72CF940E740F2CF4127208D
:10EED000FEF73CF840F2CB312720FEF737F840F23E
:10EEE000E2312720FEF732F801E200005DEB00007E
:10EEF000D9E4000071E100000B46062203F8032B61
:10EF0000B0F809C0C27AA1F803C09A70704700BF78
:10EF100006230B70D0F80F301A88A1F8032093F85D
:10EF2000CD304B71024B5B6800229A67704700BF7F
:10EF3000843000200B46172203F8032BD0F809C0B9
:10EF4000D0F80D20C1F803C05A60704710B53923BE
:10EF500001F8033B00F109032930D3F800E0D3F8AE
:10EF600004C09A68DC68CC6010338342C1F800E0CA
:10EF7000C1F804C08A6001F11001EED11B880B803A
:10EF800010BD00BF124B134A33F8113003F2E733C0
:10EF9000A2FB0323082900F1FF324FEA93134FEA43
:10EFA000C2120FD0042907D0022914BFF02160211A
:10EFB000134401FB0030704740F2BE21134401FBB3
:10EFC000003070474FF4D261134401FB00307047AA
:10EFD000F8160700D34D621030B5D928844628BFF3
:10EFE0004FF0D90C0CF1300CBDF80C401FFA8CFC22
:10EFF000BCF1FF0F28BF4FF0FF0C04F0020514F026
:10F000000104864638D1002D64D001F5A570082A88
:10F0100000F01481042A00F0C580022A14BF4FF4C6
:10F0200014714FF49671014412F00C0F40D1082A6C
:10F0300000F00C81042A00F00C81022A14BF4FF466
:10F04000B070B4209C31014401F19800B4BB002B96
:10F0500000F0AC80082A00F03C81042A00F099817D
:10F06000022A40F6480308BF4FF48563BEF1D90F6A
:10F07000184400F2428130BD01F5A570002DC6D1C3
:10F08000002B42D1082A00F01C81042A00F09C8148
:10F09000022A00F0B7810CF1050C1FFA8CFC282124
:10F0A00008250CFB051C12F00C0F0CEB0001BED068
:10F0B00001F6144101F19800002CC8D0082A00F094
:10F0C000C180042A00F0C880022A14BFC023642330
:10F0D000184430BD01F5A5702BB3082A00F0438118
:10F0E000042A00F07981022A40F6480308BF4FF451
:10F0F0008563BEF1D90F1844BDD9AEF1D903C54916
:10F100009BB2F63381FB0341FEE0082A00F0D68073
:10F11000042A00F03B81022A40F6480114BF8C46C5
:10F120004FF4856CBFE7082A00F01181042A00F033
:10F130005B81022A00F004810CF1050C1FFA8CFCA3
:10F14000282408230CFB034CBEF1D90F604492D94C
:10F15000B149AEF1D90E1FFA8EFEA1FB0E31AEEB16
:10F16000010301EB5301042AC1F3C71146D1C1EBDE
:10F170004113C1EBC303AEEB030341F208329BB270
:10F1800002FB0100002B3FF476AF03F1080292B2BC
:10F1900005324FF4BF74102100F5A57302FB014244
:10F1A000D01830BD40F2CE5101443DE77346F12BFB
:10F1B00028BFF123082A53D0042A00F0FE80022A37
:10F1C00000F01A8113339BB228214FF0080C03FB87
:10F1D0000C13BEF1D90F18447FF64DAF8E49AEF136
:10F1E000D90E1FFA8EFEA1FB0E31AEEB010301EB2F
:10F1F0005301042AC1F3C71100F09280C1EB4113FF
:10F20000C1EBC303022AAEEB030E40F6921540F2A7
:10F2100072541FFA8EF318BF2C4604FB01000CBF7A
:10F2200018242824002B3FF426AF0833022A9BB26F
:10F2300003F105020CBF04210821ADE741F2D02102
:10F240000144F1E64FF4CA63184442E74FF43560D5
:10F25000F8E640F2EE30F5E640F2AE23184438E727
:10F2600013339BB200EB8310BEF1D90F00F5C870C9
:10F270007FF601AF684AAEF1D90E1FFA8EFEA2FBEF
:10F280000E32AEEB020302EB5302C2F3C712C2EB23
:10F290004213C2EBC303AEEB030E44F2DA311FFAA2
:10F2A0008EF301FB0200002B3FF4E5AE03F10802F0
:10F2B00092B205324FF4C87440216DE744F2902CAD
:10F2C000F1E60CF1050C1FFA8CFC4FF4C8714025D7
:10F2D000E7E601F58640BEF1D90F00F128007FF680
:10F2E000CAAEAEF1D9024B4B92B2F63283FB021397
:10F2F0001344DB1144F2DA310FE0AEF1D901454B92
:10F3000089B2F63183FB01430B4440F6921440F27C
:10F310007251DB11022A18BF214601FB030030BDE8
:10F32000C1EB4113C1EBC303AEEB030E41F2083254
:10F330001FFA8EF302FB0100002B7FF426AF30BDD5
:10F340000CF1050C1FFA8CFC18240423FAE60CF1CE
:10F35000050C1FFA8CFC00EB8C13BEF1D90F03F5E2
:10F36000C87087D887E644F2DA32BEF1D90F01EBD4
:10F3700002007FF680AEAEF1D901264B89B2F6319C
:10F3800083FB01430B44DB111146C6E741F2BE1C6F
:10F3900089E601F59250BEF1D90F00F116007FF613
:10F3A0006AAEAEF1D9021B4B92B2F63283FB021366
:10F3B0001344DB1141F20831AFE713339BB24FF432
:10F3C000BF714FF0100C02E70CF1050C1FFA8CFC1A
:10F3D0004FF4BF71102564E641F20832BEF1D90F37
:10F3E00001EB0200C7D830BD0CF1050C1FFA8CFCF4
:10F3F0004FF4BF741023A5E613339BB218214FF0CE
:10F40000040CE4E60CF1050C1FFA8CFC1821042511
:10F4100047E600BFC9F9A98491F353092DE9F043E8
:10F42000314ED6F800C0DCF80F300B624FF0000808
:10F430009CF8153062F3070862F30F2815469CF814
:10F4400014201B0443EA02239CF8132013438B620D
:10F4500083B00746BCF819000C4619F024FD336848
:10F46000E06181464946987D19F02AFD336820867F
:10F470004946B3F8170019F041FD3368E062B3F86C
:10F480001B20A284B3F81D20E28493F8242002F00C
:10F490001F0284F8D920D3F81F00009093F823307E
:10F4A0008DF80430694604F1CD0019F08FFD336802
:10F4B00093F82430A4F870805B0984F8D932FF23D4
:10F4C00015F00C0F14BF0121002104F1380084F85D
:10F4D00072300BF03DFF97F91410204619F0CCFC68
:10F4E00003B0BDE8F08300BF44280020F8B544888D
:10F4F0008C46054614F00401134618BF05F1770148
:10F500006246C07F0BF086FAC207044606D4A30702
:10F5100012D484F00400C0F38000F8BD012385F804
:10F520006830E87F0BF04EFB0368C5F869308388CC
:10F53000A5F86D30A307ECD5084E0127306885F893
:10F54000767005F1770119F024FE3068394619F01C
:10F5500034FE84F00400C0F38000F8BD442800208D
:10F560000B46132270B503F8032B0C4600F1090279
:10F570002930166855689168D2F80CC0C3F80CC0E1
:10F58000103282421E605D60996003F11003F0D179
:10F5900012781A70A6880125A57129463046FEF713
:10F5A000E3FA48B1E27842B100880AF0BFFE29468A
:10F5B0003046FEF7EFFA20B970BDBDE870401AF092
:10F5C000F1BF40F242212D20FDF7C0FC1323F7B517
:10F5D0000B700023CB7083691A888A80054601224C
:10F5E0008A71D8690C4619F04BFCAB6960839A8C20
:10F5F000A283DA8CE28393F8D92284F82020FF22B8
:10F6000084F821206A69128962845A7A012A04F1F5
:10F610000E012ED1DA7B02F0C002402A29D1D3F8A4
:10F620000A20C4F80E20DB898B80154B5868436D87
:10F630006361B0F858302383AF69BE78E671002368
:10F640000622694654300093ADF8043015F032FAC2
:10F6500010B146F00206E671D7F80330A360B7F8A0
:10F660000730A381A86940B103B0BDE8F0401AF0AB
:10F6700099BF0023C4F80E30D6E703B0F0BD00BF39
:10F680008430002070B504460D46C869164619F04E
:10F69000F7FBAB8CA4F8A630EB8CA4F8A830A4F848
:10F6A000A400A37F95F8D92284F8AA201BB194F86E
:10F6B0006830012B24D00022C4F89820A4F89C20A4
:10F6C0001F4B1B681A78C2F3801284F89120082E11
:10F6D000D3F8032023D0C4F89E20B3F80730A4F851
:10F6E000A23004F1920204F1910130460BF034F99A
:10F6F00008B394F8913043F0020384F8913070BD60
:10F7000094F86E3003F0C003402BD4D1D4F86920B4
:10F71000B4F86D30C4F89820A4F89C30D0E7C4F851
:10F720009220B3F80710A4F896100023C4F89E3076
:10F73000A4F8A23070BD40F64A412D20FDF706FC2A
:10F74000442800200B46162203F8032BD0F809208A
:10F75000C1F80320CA7890F80DC083F804C01AB12C
:10F7600030F8AC3C1B0700D5704710B5B1F8054028
:10F7700001212046FEF7F8F938B100880AF0D6FDDD
:10F7800001212046FEF706FA00B910BD40F286219D
:10F790002D20FDF7DBFB00BF2DE9F0438A4D8B4A9E
:10F7A000AB6A87B05B680292894A03920026894A55
:10F7B0006E71044680F8816002A8CDE904232E8290
:10F7C000AE60AE7110F094FC0FF0AEFE10F05EFD76
:10F7D0000FF02CFA80480FF0CDFF804810F082FC2B
:10F7E00004F13007304615F0F9FA384601F0BCFB59
:10F7F000384601F0BFFB0FF0C7FF217925200FF03D
:10F80000FDFD94F914000FF0AFFF2179304610F0A0
:10F81000A3F9E86028B901232B71002007B0BDE8E7
:10F82000F08304F15001E06C17F0FFFB04F1580184
:10F830000646E06C17F020FC07463EB194F82480A1
:10F84000B8F1000F02D04FF0010903E0002F5CD1A6
:10F85000B846B946A37F13B9638859071BD5D4E9C5
:10F8600018236FF000418B4208BFB2F1FF3F54D024
:10F870001BF0F4FBD4E91823904271EB03034CD343
:10F88000414601222046FFF731FE00284FD1B9F151
:10F89000000F40F09480002E08BF3E4694F883305D
:10F8A000002B71D1002E6FD1286803300BF0A0F827
:10F8B0006388A874DB07B0D50023266ACDE900333E
:10F8C0000122FF238DF8062085F8203006F10A0773
:10F8D0006846FEF781F900289FD1009CA642F7D028
:10F8E000727A607A3B4604F10A0119F055F9002852
:10F8F000EED0A37885F82030D4F80320C5F8212075
:10F90000374BB4F807209A8087E794F82580B8F140
:10F91000000918BF4FF001099CE7B9F1000FBAD0F8
:10F92000012211462046FFF7E1FD002847D00BF0E9
:10F930000DF880461BF092FB4FEA4813B3EB080327
:10F940004FEAD86262F10002520242EAD3525B02ED
:10F9500013EB080342F1000C4FEA8C1E9A014EEAA9
:10F96000936ED31A6EEB0C0213EB080342F1000204
:10F970001B1842EB0101C4E91831002E08BF3E46B6
:10F9800094F88330002B8DD06388DA068CD4666CB3
:10F99000C6F30B260BF088FDC0F30B039E42F9D093
:10F9A00094F8463084F84500C0F3032123F00F0398
:10F9B0000B43002284F8463084F8832074E740F635
:10F9C00014212D20FDF7C2FA44280020E100010097
:10F9D0001DFD0000E9FB0000D6BE898E555555007F
:10F9E000652800202DE9F047032984B00446164617
:10F9F00040D090F8803023B10025284604B0BDE8FF
:10FA0000F087052967D0464F97F812804FF001091B
:10FA1000B8F1000F39D13378082B70D0396894F8D9
:10FA20006F2011F8030B04F17003C0F3801019F07C
:10FA3000B3F83968054611F8030BC0F3801019F0CC
:10FA4000E5F882460BF0D0F80746002830D133782D
:10FA5000082B4FD0002D34D063885907CDD4002F08
:10FA6000CAD1B8F1000F53D1637D0BB14B45C3D15F
:10FA70000125C2E743889A07BED5294F97F812801F
:10FA80004FF00209B8F1000FC5D019F0C9F80828E5
:10FA9000307034D002AA0DF107010AF05DFF002892
:10FAA00038D09DF8070002A91AF03FFC8046B2E763
:10FAB000BAF1080F13D13378082B1BD00027002D83
:10FAC000CAD1E57FED1A6388B5FA85F559074FEA83
:10FAD000551592D4C3E74388DB0794D48CE750468E
:10FAE0000AF03EFE33780028E6D1082B84D0002DA2
:10FAF000B2D1E6E7638858073FF57FAFB1E73968D1
:10FB000011F8030BC0F380101AF00FFC804685E754
:10FB1000454672E740F63D712D20FDF717FA00BF0C
:10FB20004428002038B52E4DB0F84830AA7C013367
:10FB30000446A0F84830B2B900232B7194F8813004
:10FB40005BB9637C1BB1B4F848209A4212D22046BC
:10FB50000021BDE8384002F08FBD20460121BDE8FC
:10FB6000384002F089BD10F091FB0FF05FF80023E0
:10FB7000AB74E1E70121204602F07EFD6388DB07DC
:10FB80000FD5236A1D880AF035FA68B9637C21789D
:10FB900084F8B8104322A4F8B95084F8B720A3B170
:10FBA00011E00AF027FA00B138BD637C207884F8B0
:10FBB000B8004FF0FF32432184F8B92084F8BA200E
:10FBC00084F8B7100BB194F8483084F8BB3004F1D6
:10FBD000AE000449BDE83840022219F065BE00BFFE
:10FBE0004428002045F7000060B951B1074A137955
:10FBF000916AD06A096903F18043043B51F82330CC
:10FC000018477047014BD86AFFF78CBF4428002083
:10FC10002DE9F04182B008230DF1070205210446C9
:10FC20008DF80730FFF7DEFE00286BD06279216A7D
:10FC30002046FFF7F3FB216A002384F88D30088803
:10FC4000A4F88E004FF6FF73FF2284F8AB20A4F8CF
:10FC5000AC309DF807202046FFF714FD236A2D4A9B
:10FC600019881568A4F8C51093F8CD2084F8C7202A
:10FC700025B1184601222146A847236A264D286847
:10FC8000D0F80320C3F80320B0F80720A3F807201A
:10FC90000678D4F820800027C6F3801688F8026022
:10FCA0000821078019F045FA2868394619F0BFFB8A
:10FCB00028683A464FF0030119F0C0FB3A46062384
:10FCC000286804F1690119F08CFB94F86810286821
:10FCD00019F066FA2868314619F06FFA06230122F6
:10FCE000286808F1030119F07CFB6179FF200FF00F
:10FCF00085FB286810F012FA092301202B7102B04D
:10FD0000BDE8F0812046FFF70DFF012002B0BDE8FD
:10FD1000F08100BF6C00002044280020F0B54D4C5D
:10FD20002379022B85B003D02379032B40F0868002
:10FD3000E36A1D6A0DB195F8755088B9A37C1BB1B3
:10FD400010F0A4FA0EF072FFE06A02F0BBFA40B3C2
:10FD50000FF0F0FDA36A9B6805B0BDE8F0401847BE
:10FD6000216893F8682011F8096B6933F00918F0DD
:10FD700013FF0028E2D006F00F06052E206827D0DA
:10FD8000294619F043FA0028D8D02379E06A022BDB
:10FD90000DD02379032B0AD040F6C5412D20FDF765
:10FDA000D5F8E06A05B0BDE8F040FFF7BBBE2379A7
:10FDB000A26A03F180435269023B314652F8233074
:10FDC0009847A37C002B3ED10028BDD105B0F0BDE3
:10FDD00090F8243003F01F03102BD1D9E76AFB7C85
:10FDE000002BCDD008230DF10F02314638468DF897
:10FDF0000F30FFF7F7FD0028A0D097F8E130002B77
:10FE00009CD1216807F1E202CB1C23311E685D689A
:10FE10009868D3F80CC0C2F80CC010338B4216603F
:10FE20005560906002F11002F0D11B8813800A49DE
:10FE3000022207F1D90019F037FD7FE740F6EC41C7
:10FE40002D20FDF783F8019010F020FA0EF0EEFE61
:10FE50000198B9E7442800204DEF00002DE9F0415A
:10FE600004460E46002940F08E80704D286894F8B4
:10FE70007670002303806388103B0D2B00F2C7804F
:10FE8000DFE803F07CC5771EC507C5C5C5C5C5C578
:10FE9000C507012119F04DF92868037823F02003E4
:10FEA00043F020030370002F00F0948004F17701E9
:10FEB00019F06FF92868012119F07FF9286809E025
:10FEC000002119F036F92868037823F0200343F065
:10FED0002003037004F1690119F04DF994F86810DA
:10FEE000286819F05DF9638823F008039BB2152B8D
:10FEF00005D094F85420216D286819F068F9286815
:10FF000010F00CF904232B71F6B16388102B6CD020
:10FF100004F130084046EF6801F0BEF8064640465E
:10FF200001F096F8013E301A61882822C0B201F033
:10FF3000F3F863881B0707445CD422793946002014
:10FF40000FF056FF00286CD06388103B0D2B63D850
:10FF5000DFE803F00D6207076207626262626262B5
:10FF6000620721790120BDE8F04110F0A9B9BDE890
:10FF7000F081062119F0DDF82868ABE7022119F0BD
:10FF8000D8F82868A6E700F13007384601F060F895
:10FF9000A8B963881A0735D5384601F07DF80546BB
:10FFA000384601F055F8281AC0B2204D01F0AEF8DD
:10FFB000AB6803443846AB6000F0D6FF00E01B4D51
:10FFC000384600F0D7FF0FF0DFFB217925200FF036
:10FFD00015FA4BE704F1700119F0DBF8286894F882
:10FFE0006F1019F0EAF8286874E7217900200FF003
:10FFF000D1FBA9E7AB681F4401F060F83844C4F8AE
:020000040001F9
:1000000018019AE72046BDE8F041FFF78BBD40F2AA
:1000100049612D20FCF79AFF40F675512D20FCF721
:1000200095FF40F661512D20FCF790FF44280020F9
:1000300038B54388102B1FD0124DAB7C044663B9F2
:10004000286810F06BF8608810F004000BD00020D6
:1000500010F0CEF802232B7138BD0EF0C9FD402000
:1000600010F008F9ECE7217910F02AF9002010F0DF
:10007000BFF802232B7138BDBDE838400121FFF7DE
:10008000EDBE00BF442800200121FFF7E7BE00BFFE
:10009000024B0121D86AFFF7E1BE00BF44280020CF
:1000A00070B50C4E337963B90378FF2B054608D041
:1000B000FFF772FB044610B93379012B04D12046B7
:1000C00070BD0C24204670BD01462846FFF7C6FED1
:1000D000204670BD442800200121FFF7BFBE00BFAD
:1000E00010B5164CA37CF3B9E06A02F0EBF8A8B1A6
:1000F000E06A438803F018038BB12379022B02D006
:100100002379032B14D12379A26A03F18043D268A7
:10011000023BBDE8104052F823301847E06ABDE8C2
:100120001040FFF7FFBC10F0B1F80EF07FFDDBE7E9
:1001300040F6F4312D20FCF709FF00BF44280020D1
:1001400038B51D4C2379002B35D02379E56A022B75
:1001500019D02379032B16D014F082FE94F8303096
:10016000F3B1284602F0AEF8D0B1E46A63881B0709
:100170001BD404F1300000F06BFFB0B92046BDE89D
:100180003840FFF7CFBCA37C002BE5D010F07EF801
:100190000EF04CFD14F064FE94F83030002BE0D1EA
:1001A0002846BDE83840FFF7BDBC20460121BDE828
:1001B0003840FFF753BE38BD4428002030B50B68E7
:1001C00083B0002B51D00C460546184600F064FF62
:1001D00094F810E0627CBEF1040F3BD0254B264919
:1001E00033F81E30042A03F2E73323D0A1FB0313B4
:1001F0004FEA931CBEF1080F00F1FF334FEAC3131F
:1002000025D0BEF1020F14BFF0216021634401FB31
:100210000031A388009328460023FEF7DDFED4E9D1
:100220000223D730824273F100032CBF012000204B
:1002300003B030BDA1FB03234FEA931CBEF1080FAE
:1002400000F1FF334FF008024FEAC313D9D14FF446
:10025000D261DBE7431E042A4FEAC3134FF02C0C94
:10026000F5D108224FF4D261D0E740F2FD312D20C4
:10027000FCF76CFEF8160700D34D62102DE9F04F25
:1002800090F8803087B0002B3DD1458815F00105EE
:10029000044638D0774E03F0FF0AB37C002B40F0C1
:1002A000C680316811F8030BC0F380101AF03DF8D6
:1002B0004FF008098346316894F86F2011F8030B5A
:1002C00004F17003C0F3801018F066FC3168074633
:1002D00011F8030BC0F3801018F098FC80460AF068
:1002E00083FC019018B1B8F1080F40F08680B9F195
:1002F000080F00F0AF80638857B95A0740F18A8031
:10030000E37F4B4506D00025284607B0BDE8F08FB7
:100310005B077FD53168584B11F8030B96F8202006
:10032000C0F3801018F038FC07460028EBD1216A92
:1003300033681A7891F8CD3003EA521303F00103C1
:1003400081F8CD3001222046FFF768F8216A84F851
:100350008D70FF23088884F8AB304FF6FF73A4F844
:10036000AC304A46A4F88E002046FFF78BF943498B
:10037000022204F1840019F097FA236A40491A888E
:10038000A4F8C52093F8CD3084F8C730022204F1D8
:10039000BC0019F089FA236A1F8809F02BFE88B97E
:1003A000637C2278A4F8B97084F8B70084F8B82088
:1003B000002B56D1334984F8BB30022204F1AE0041
:1003C00019F072FA304B1B680022327113B1206AA7
:1003D000214698473368226AD3F80310C2F8031005
:1003E000B3F80710A2F807101B78226AC3F3801332
:1003F0002846937007B0BDE8F08F40460AF0B0F988
:10040000019B00287FF473AFB9F1080F3FF47BAF75
:100410009A4670E7BAF1000F7FF475AFBBF1000F99
:100420007FF478AF637D012B3FF66DAF72E718F074
:10043000F7FB082881463FF434AF04AA0DF10F0101
:100440000AF08AFA80B19DF80F0004A919F06DFF37
:10045000834630E763885907E0D5002F3FF453AF58
:1004600058E794F84830A5E740F63D712D20FCF799
:100470006DFD00BF442800206528002061F50000C4
:10048000F9EE000045F700006C0000202DE9F04770
:10049000032984B00CD0052946D1684B1C681CB1D7
:1004A000A04780F00104E4B2204604B0BDE8F08724
:1004B00043880546980737D5614EB37C002B38D169
:1004C000316811F8030BC0F3801019F02EFF4FF0C4
:1004D00008088146316895F86F2011F8030B05F183
:1004E0007003C0F3801018F057FB3168074611F80D
:1004F000030BC0F3801018F089FB82460AF074FBEE
:10050000044638B1BAF1080F04D050460AF028F971
:10051000002875D0B8F1080F41D000246B88DFB9EE
:100520005A0766D4002C3DD00124204604B0BDE813
:10053000F08718F075FB08288046C1D002AA0DF19B
:1005400007010AF009FA00286ED09DF8070002A9F9
:1005500019F0EBFE8146BDE75B07E3D52B7C4BBB77
:10056000306800240480042118F0E3FD306805F1B0
:10057000690118F000FE95F86810306818F010FE58
:1005800095F85C20A96D306818F030FE30680523BE
:1005900033710FF0C3FD204604B0BDE8F0876B88CF
:1005A00059072AD4B9F1000FD8D16B7D13F0FD0F94
:1005B000BAD1D3E795F8D030002BD1D12B7885F87C
:1005C000D130B8F1080F1FD005F1D30205F1D201E7
:1005D00040460AF0C1F960B395F8D23043F0020307
:1005E00085F8D2301749022205F1C80019F05CF9EC
:1005F000B6E7EB7F434597D1B0E7002F94D0ADE746
:10060000B8F1080F8AD14FE731680B4613F8032B76
:10061000C2F3801285F8D220D1F80320C5F8D32088
:100620009B88A5F8D730DDE740F63D712D20FCF71B
:100630008DFC40F6BA712D20FCF788FC6800002084
:100640004428002035EF000008B590F88C3043B9FD
:1006500090F8C4302BB990F8B63003F0FF0013B90E
:1006600008BD012008BD09F0C5FC80F00100C0B242
:1006700008BD00BF10B50948037913B10C2420460A
:1006800010BD03F0FF0424222146043014F0F0FAD8
:100690000FF0FCFD0EF0CAFA204610BD44280020E1
:1006A00010B50E4C002323712379206023B140F252
:1006B0001E312D20FCF74AFC03F0FF012422201DEF
:1006C00014F0D6FA0FF0E2FD0EF0B0FAA36A03B10F
:1006D00010BD40F221312D20FCF738FC44280020C9
:1006E00030B54FF4AC7285B004460D46002114F0CD
:1006F000BFFA42F21073FF211322E384217062805B
:10070000FDF73EFB00220146E0646846FDF77CFBF6
:10071000E06C0022012116F06BFCE16C04226846BB
:10072000FDF772FB0022E06C114616F061FC04F14B
:100730003000257500F0F6FB02A80AF0A1FB30B1ED
:1007400002A904F1360018F041FC05B030BD40F2BA
:100750003A312D20FCF7FAFBFF23C86C0B7016F022
:1007600014BC00BF014B024A9A6270474428002023
:100770000C0F0100054A0649064B074810B4074C08
:100780001460074A10BC08601A60704768000020B7
:100790006C00002064000020012601007D020100A1
:1007A00011FC00000078FF3818BF0120704700BF1F
:1007B00070B5044682B030300D4600F06DFC6388A1
:1007C000D9062ED49A0794F804E01B4A1B4932F844
:1007D0001E20844602F2E7324CBFB4F85C00B4F845
:1007E0005400A1FB02120CF1FF36BEF1080F4FEAD4
:1007F00092124FEAC61611D0BEF1040F18D0BEF106
:10080000020F14BFF02160210093324401FB0C2140
:100810002B466279FEF7E0FB02B070BD4FF4D26167
:10082000F2E72822194602B0BDE8704000F04ABC49
:1008300040F2BE21E8E700BFF8160700D34D621072
:10084000428812F0180F01D00120704710B586B011
:1008500000F1300403460094D3E90234B0F804C038
:10086000ADF8042008466946CDE90234ADF810C061
:10087000FFF7A4FC06B010BDD0E90201704700BF2D
:10088000407D003818BF0120704700BF2DE9F041BE
:10089000857DAB1EDBB2012B04468CBF00270127F0
:1008A000002D59D0B5F1020818BF4FF00108012BF7
:1008B0000BD943889A0665D40826022D67D0637F3A
:1008C000002B56D10020BDE8F08100F1700190F8B6
:1008D0006F0018F09BF963889B06064605D408282C
:1008E000EAD009F049FF0028E7D1E677A77784F836
:1008F00068800AF02BF805461AF0B0FB6B015B1B11
:100900004FEAD56C6CF1000C4FEA4C2C4CEAD35CEE
:100910005B025B194CF1000E4FEA8E164FEA831C06
:1009200046EA9366BCEB030366EB0E0C5B194CF1D5
:10093000000C1B184CEB01010022C4E9183184F8AB
:10094000762011462046FEF7D1FD0028BBD140F2AB
:10095000B6412D20FCF7FAFA4388990614D40826EC
:1009600004F16901002009F06DFD0028AAD0A84615
:10097000BBE7D4F81730C4F86930B4F81B30A4F8DA
:100980006D30B2E70826B0E7A8460826ADE7454631
:10099000E6E700BF0B68C0F817308A88A0F81B2074
:1009A00001234377704700BF2DE9F04F84460C4682
:1009B00090F8058090F812A00546BCE80F009DB0A5
:1009C00010AF0FC7BCE80F000FC79CE80F0008AEC0
:1009D00087E80F00304600F0A5FA237DA27A059241
:1009E000013BDBB2227861780692022B00F2E180B3
:1009F000724A134401F07F07C90693F8149008D493
:100A0000A37D013BDBB2022B00F2D380134493F8A9
:100A10001480BAF1010F09D1B9F1080F08BF4FF0E6
:100A20000409B8F1080F08BF4FF00408617A304696
:100A300000F080FA237DA27E022B08BF617D02F1C7
:100A4000010206BF0131C9B20121D2B2304600F025
:100A500073FA3A076FD500231A46CDE90332E86CE2
:100A6000A37C079394F818A016F050FB8346E86C1B
:100A700016F05CFB5845AAF1010A38BF5846BAFA8D
:100A80008AFA80B2DDE903324FEA5A1A00283CD1D3
:100A900007998DF85510CDE9123205998DF8561049
:100AA00006998DF850A0ADF842708DF840108DF881
:100AB00044908DF8458010AF0FCFAC46ACE80F00E6
:100AC0000FCFACE80F0097E80F008CE80F0096E816
:100AD00003002863A986E27A95F8463012F0FD0FEC
:100AE0004FF0000E14BF0122724685F86F20E268B5
:100AF0002A67228AA5F87420E27D62F3071385F83D
:100B0000463070461DB0BDE8F08F17F0180FCDE9E4
:100B10000C320A96ADF82C708DF838908DF839802B
:100B2000B6D10AA9FFF74AFBDDE903320028AFD1AD
:100B30004FF0450EE5E7304600F0AEFA6378DB068D
:100B4000824626D52822394600F0BCFA1C4B217972
:100B500000F53672A3FB0232E37843EA01236179A0
:100B6000520A43EA014340F2712101FB02F201FB08
:100B700003F39A420BD9E079A37943EA0023207A60
:100B800043EA004301FB03F39A4298BF1346002255
:100B900063E7FDF721F94946034650469A46FEF7BA
:100BA000F1F900970146012350464246FEF714FA38
:100BB000CCE740F29A210620FCF7C8F9F8160700A6
:100BC0005917B7D1438813F0100005D013F0040F64
:100BD00014BF00201F2070479A0702D4DB0701D5FD
:100BE000EE207047FDF7F8B808B5438813F0100001
:100BF00004D083F00403C3F3800008BD9A07FCD43B
:100C000013F00100F9D1FDF7E7F8003818BF012013
:100C100008BD00BF438800221D2B08BF1146A0F865
:100C200048204174704700BF90F91400704700BF1E
:100C3000408800F0010070474088C0F340007047D2
:100C40004088C0F3C000704708B54388C06CDA061E
:100C500005D49B0703D5BDE8084016F04EBA16F040
:100C60004CFA012008BD00BF4088C0F30010704757
:100C70004088A0F10900B0FA80F04009704700BF39
:100C800040797047024B9A6AD8621368184700BFD0
:100C90004428002090F8683001624B72D0F8693027
:100CA000C1F80A30B0F86D30CB81704738B5304CA0
:100CB0002379012B01D0002038BDB0F84830A27C48
:100CC00001330546A0F84830002A36D100232371AD
:100CD00095F8813063BB6B7C1BB1B5F848209A4214
:100CE00004D20021284601F0C7FCE4E70121284690
:100CF00001F0C2FC6B88DB0726D52B6A1C8809F043
:100D000079F90028D7D16B7C297885F8B81043226F
:100D1000A5F8B94085F8B7200BB195F848301549CA
:100D200085F8BB30022205F1AE0018F0BDFDC2E728
:100D30000121284601F0A0FCBDE70FF0A7FA0DF055
:100D400075FF0023A374C1E709F054F90028B2D15C
:100D50006B7C287885F8B8004FF0FF32432185F886
:100D6000B92085F8BA2085F8B710002BD7D0D4E782
:100D70004428002045F7000038B52E4DB0F8483023
:100D8000AA7C01330446A0F84830B2B900232B7185
:100D900094F881305BB9637C1BB1B4F848209A4267
:100DA00012D220460021BDE8384001F065BC204643
:100DB0000121BDE8384001F05FBC0FF067FA0DF08B
:100DC00035FF0023AB74E1E70121204601F054FC1C
:100DD0006388DB070FD5236A1D8809F00BF968B912
:100DE000637C217884F8B8104322A4F8B95084F8C1
:100DF000B720A3B111E009F0FDF800B138BD637C64
:100E0000207884F8B8004FF0FF32432184F8B920ED
:100E100084F8BA2084F8B7100BB194F8483084F8FD
:100E2000BB3004F1AE000449BDE83840022218F09E
:100E30003BBD00BF4428002045F7000038B543887B
:100E40001A07044632D4DB071AD5236A1D8809F035
:100E5000D1F888B9637C217884F8B8103C22A4F8D2
:100E6000B95084F8B720F3B91B4984F8BB3002228B
:100E700004F1AE0018F018FD012384F8813038BD6C
:100E800009F0B8F80028F7D1637C207884F8B8001E
:100E90004FF0FF323C2184F8B92084F8BA2084F85E
:100EA000B710002BE0D094F84830DDE7036A0B4917
:100EB0003C2280F88D201888A4F88E004FF6FF732E
:100EC000FF2284F8AB20A4F8AC30022204F18400A5
:100ED00018F0EAFC6388B6E745F7000061F500000A
:100EE00080F88010704700BFFF2380F88330704780
:100EF00080F8241080F82520704700BF8D04010081
:100F000031000100D900010089000100A1000100A9
:100F10004101010091000100080F0100000F0100D4
:100F2000FC0E0100002240F20113C0F802200380F1
:100F3000704700BF8170704708B590F802C04270DA
:100F4000CCF380030170CCF3400003440CF0010C9F
:100F5000634413FB01F303FB02F2FE2A00DC08BD2D
:100F60005C212E20FBF7F2FF00234371A0F8033031
:100F7000704700BF08B58378DA070DD5C17811F046
:100F8000010C09D1427990F801E00132D2B29645C4
:100F9000427142D0252008BD990703D5C27812F0CE
:100FA000020C23D05A0713D4427941780132D2B2CD
:100FB0009142427108D1C17800229942427103D115
:100FC0000379C2700133037139212E20FBF7BEFF74
:100FD000C27812F0040CE7D1417990F801E00131B8
:100FE000C9B28E45417126D0272008BD417990F8BD
:100FF00001E00131C9B28E45417101D0262008BD02
:1010000042F00202934280F805C0C270F6D1037923
:1010100080F803C001330371F0E741F001018B4216
:1010200080F805C0C170B5D1037980F803C00133E1
:101030000371252008BD42F00402934280F805C0E8
:10104000C270D1D1037980F803C001330371CBE7BB
:1010500010B590F802E004790178C27890F801C0E8
:10106000CEF38003091B4479CEF3400003440EF015
:10107000010011FB0CF1184410FB01F0C2F38003D6
:10108000C2F340010B4402F00102001B134403FBB6
:101090001C00C0B210BD00BF837842780178C3F352
:1010A000400CC3F38000604403F00103184412FBBA
:1010B00001F310FB03F0C0B2704700BF40F2EF2015
:1010C000704700BF0138022808B519D8132907D87E
:1010D00011290CD810290FD10B4B33F8100008BD83
:1010E000152909D1084B03EB4000008908BD064BC8
:1010F00003EB4000008A08BDD8212F20FBF726FF14
:10110000CA212F20FBF722FF1017070040F25A33A5
:1011100003FB00F0704700BF08B5431EDBB2012B94
:1011200006D91D293AD140F25A3303FB00F008BD1D
:1011300010390D292DD801A252F821F07F1101009C
:101140009311010075110100751101009311010047
:101150008911010093110100931101009311010005
:1011600093110100931101009311010093110100EB
:10117000271101000B4A02EB4303188C08BD094AF2
:1011800002EB4303188B08BD064A02EB4303988B1E
:1011900008BD4FF481712F20FBF7D8FEEE212F20E0
:1011A000FBF7D4FE1017070008B540F24F310620B8
:1011B000FBF7CCFE70B582B00446FFF755FD18B9B9
:1011C0006124204602B070BD2046FFF731FDD0B14A
:1011D00064265A240DF106000FF0C8FD0DF107003A
:1011E0009DF906500FF0C8FD9DF807301D436DB204
:1011F000002D18BF344613F063FE60B11834A4B25A
:10120000204602B070BD2046FFF716FD0028DFD152
:101210005A265024DEE713F0AFFD0028D1D00F345A
:10122000A4B2CEE72DE9F04182B0002800F03F8162
:101230000446082900F22681DFE811F0DB00E9000E
:1012400009000900D6002401D00002012001FFF7A7
:101250000BFD002800F0FE802046FFF7E9FC002887
:1012600000F01C8164275A250DF106000FF07EFD69
:101270000DF107009DF906600FF07EFD9DF8073027
:101280001E4376B2002E18BF3D4613F019FE00280B
:1012900000F0FC801835ADB2B4F82A31A4F838510A
:1012A00000210122082B84F8301184F83B2100F240
:1012B000DE801344D4F80C219BB2A4F82A3112B179
:1012C000092B00F0D980022384F83A3119F0C6FEC8
:1012D000D4F84021D4F84431171A63EB01080546CD
:1012E0000E4610F011F8B4F83831D23303449BB2F3
:1012F0009F4278F1000204DA5B1946F10006C4E966
:10130000503604F598750021284617F03CFD94F8F6
:10131000503103F0FF01002B40F0A180D4E95202CC
:101320006FF000439A4208BFB0F1FF3F13D0204650
:10133000D4E95067FFF73CFAD4F84831D4F84C218F
:101340009B1B00F1F70062EB07021B1A62F100021F
:10135000002AC0F2818094F80801294612F08CF826
:10136000002800F0B280D4F84011D4F82001D4F85D
:101370004431D4F82421884272EB030344D220463E
:10138000FFF77AFA50EA0103074688463CD0D4E9D1
:101390005001D4F82031C01AD4F824313A4661EB18
:1013A0000301434613F02EFB07FB01F5D4E9483156
:1013B000A7FB002600FB08559A18354445EB0105AC
:1013C000C4E9482520E0E81A6F284FF0030138BF30
:1013D0006F2012F0D7FDC4F8345138B3204602B064
:1013E000BDE8F041FFF7C8BC02B0BDE8F0410EF027
:1013F000E9BFFFF747FC00285DD1D4F83401E73896
:1014000012F018FD00285BD002B0BDE8F081FFF7B4
:1014100017FC014650B92046FFF7CAF9D4F8343119
:1014200000F1F7059D42CED8C4F834512046FFF7AD
:101430003DFC0028E8D040F2A2213020FBF786FDD9
:1014400090F8080111F0A6FE002384F8283102B0BC
:10145000BDE8F08161251FE72046FFF7EFFC94F817
:10146000080111F097FE002384F828317BE7D4F8B7
:101470000C31002B3FF427AF012325E7EA21302070
:10148000FBF764FDEE213020FBF760FD13F074FCE8
:1014900000283FF401AF0F35ADB2FDE62046FFF75F
:1014A000CBFB00287FF4DEAE5A275025DCE6CA21AC
:1014B0003020FBF74BFD40F277213020FBF746FD53
:1014C0004FF41F713020FBF741FD40F2AC6130203A
:1014D000FBF73CFD2DE9F04F04468BB00020029352
:1014E00094F87130069017460E46059317F006F9EA
:1014F00094F8D9220B2A00F27983AD4B33F81250BD
:1015000094F8C6200392284487F0010285B2049221
:101510002FB3B4F868A3B4F8BC90A6EB0A0A0FFA8C
:101520008AFAA6EB0909BAF1000F0FFA89F904F556
:101530005078C0F2C9819F4ADDF808B0127802F0F5
:10154000FF07002A40F0D18194F82433032B00F2E6
:101550005E83DFE813F03301F9009800300094F85F
:101560002423032AD5D1039A0E2AD2D1B4F8B42366
:10157000B242CED1B4F86A23B4F8F6120A44C4F8E1
:101580002023D4F82C23C4F81823E269C4F81C23C0
:1015900020460BF0AFFFD4F8B823E262B4F8B623CC
:1015A0002286D4F8BC23E261D4F8C023626202220E
:1015B00084F82423ADE7E569029B05FB0AF2002BC2
:1015C00040F02F8294F83B33002B00F0DA82794B05
:1015D0005868D4F82C33EB1AA3F5AB75D4F8603304
:1015E000D71B854228BF05460697DF19D4F8643318
:1015F000C4F8F05243F10003C4F85433002384F8D4
:1016000040336E23A4F84833C4F8507304F1380013
:1016100018F0DEF9D4E9D4230544C4E9D823C4F88A
:101620004453A4F868630BF025F820B1D4F8443390
:101630001E33C4F84433B4F8E012039A8E1B00231F
:1016400036B29E4284F84A33C4BF022384F84A3338
:101650000E2A029A00F05F82002A40F05F8294F81E
:101660002433002B40F07B8294F86C03414611F048
:1016700003FF002800F0BC82049B84F8383300206C
:101680000BB0BDE8F08FE36AD4F81C032946184478
:101690000FF00AFE2946C4F82803E069464D0FF012
:1016A00003FEE26994F8719041F64B539A4298BF59
:1016B0000230C4F82C0348460FF0CCF900F55F4027
:1016C00019F00C0F00F14100A5FB003014BF2821D8
:1016D000002101EB90118031204618F011FAB4F886
:1016E000F632002B00F07481D4F81C33E26AD4F88F
:1016F000285313445B1B0693D4F81833D4F82023E3
:1017000094F871A002FB0355238E30351AF00C0FAC
:1017100003EB450540F0538150460FF09BF9264BF3
:1017200000F52340A130A3FB00304FEA901950464A
:101730000FF088F94D441F4B069A28445860012346
:10174000E56984F8243344E7D4F82C03E269D4F83B
:101750002833D4F82013B4F8F652121A0AFB02F216
:101760000692D4F8182394F871A03033A94402FBF0
:101770000133C943258E894400FB09301AF00C0F50
:1017800005EB400540F0218150460FF063F90A4B0C
:1017900000F52340A130A3FB00304FEA90195046DA
:1017A0000FF050F94D44034B069A2844586089E0E5
:1017B0003417070078280020D34D621094F8711078
:1017C00094F8EE02DFF828A317F038FB8146E06AB0
:1017D000294648440FF068FD2946C4F82803E0690B
:1017E0000FF062FDE26941F64B539A4298BF023016
:1017F000C4F82C0307A908A80EF0D8FD079B009396
:10180000D4E9D801DDE9082312F03CFE94F87130E8
:101810000593054618460FF01DF9059B00F55F403E
:1018200013F00C0F00F1410014BF28210021AAFB86
:10183000003001EB90118031204618F061F9D4F8A6
:101840007033E26A94F87100069305920FF002F982
:101850004AF2A13B00EB0B03AAFB0331069B059A5E
:10186000D4F82803203B13441B1A4B445B1BA3EB07
:101870009113069394F87130B4F8309000F130056C
:1018800013F00C0F4FEA450509F1220940F09A8048
:10189000184605930FF0DEF88344AAFB0B3A059B2C
:1018A0004FEA9A1A18460FF0CDF84D44914B069A1C
:1018B000554428445860D4F87033D31AB3F5D67F12
:1018C00040F29B81E56984E6002284F83B23894A43
:1018D000D4E9D6011278C4E9D801CA464FF0010B09
:1018E00002F0FF07002A3FF42FAE0FF087FD0746F6
:1018F00000283FF429AEB4F80C23012A40F2F58009
:1019000094F82423022A00F0F08094F83A23002A65
:1019100040F0EB80E06941F64B57B84240F243811A
:1019200094F8D9220B2A00F26181734B33F81250DC
:1019300094F8243305F5C865012BADB240F037812A
:1019400094F8C930032B40F04681D4F81C03E76AB1
:10195000074429460FF0A8FC03463846D4F818730C
:10196000C4F81833DB1BD4F82073294603FB07F7B0
:101970000FF09AFCD4F82833C4F82803C01A07449F
:101980002946E0690FF090FCE36941F64B5293421F
:10199000B4F8F632D4F820234B446FEA0202A3EBEA
:1019A0000A031344D4F82C2398BF0230C4F82C0344
:1019B000801A00FB0377012384F83A33C4E54FF023
:1019C0006509B4E64FF0650A6CE74FF06509E6E695
:1019D000029B002B3FF488AE94F871B0D4F81C231E
:1019E000E36A584602EB03090FF034F8D4F8743375
:1019F0008246A9F1200958469944D4F828B30FF03B
:101A000021F80AF5234AA9EB0B090AF1A10AA9EB6F
:101A10000009A5FB0A35A9EB95150695D4F82853BE
:101A20006AE6B4F8F632002B7FF4CCAD84F83B3391
:101A3000D4F82C1301FB1A2A94F8C520CDF818A06D
:101A4000262A5BD094F8C620262A57D0BBF1000F77
:101A500027D033BBD4F874B3BBF1000F00F0D280B1
:101A600094F8710010F00C0F40F09B800EF0F2FF24
:101A70001F4DD4F874B300F52340A130A5FB003509
:101A8000AD0994F8710010350EF0DCFFAAF1100AD0
:101A90000AEB0B02551B2D1AB4F8F632D4F82C13AE
:101AA0000695059803EB090B01FB0BFB0BF1300BC3
:101AB00010F00C0F4FEA4B0B61D10EF0CBFF0C4D29
:101AC00000F52340A130A5FB0030850905980EF0F4
:101AD000B9FF084B054405EB0B00E569586041F67A
:101AE0004B539D4250D9069A73E500272CE500BF61
:101AF000D34D62107828002034170700B4F8B423BF
:101B0000B21A1204A2D4059894F8B723002A18BF79
:101B1000104605909AE7002A3FF4A6ADB4F80C23CE
:101B2000D2B1B4F80E0394F8101300FB01118A42ED
:101B300000F101007FF798AD002B3FF495AD002335
:101B400084F84A33A4F80E0309F0AEFC00F0070055
:101B5000013084F8100387E5A4F80E2384E5E169D9
:101B6000D4F82C334046C91A17F00DF980B200287A
:101B70003FF47AAD149BC3B11880012080E5652540
:101B8000A4E7B4F8F63253E7234A284606AB594691
:101B900017F0D5F9214B84F83B03069A5868E5699C
:101BA00017E5752570E71746CEE4012068E529465C
:101BB0000FF07AFBE369BB42B4F8F672D4F82C3329
:101BC00098BF02304F44A7EB0A07C4F82C03C01A91
:101BD00000FB07F7EFE694F8711094F8EE02E76A5D
:101BE00017F02CF90744D4F81C03B2E6FFF7DCFA2F
:101BF00040F29D513020FBF7A9F940F2ED41302031
:101C0000FBF7A4F940F23F513020FBF79FF940F277
:101C100054513020FBF79AF97C28002078280020C6
:101C20002DE9F04385B0002800F0708104460829B2
:101C300000F25281DFE811F08800FE00090009007F
:101C40007000500175007D004C0119F007FAD4E9CD
:101C5000D623801A61EB0301012871F10003C0F261
:101C600063816FF00102002382428B41C0F25781F1
:101C7000E3690BB1B0FBF3F394F8C6200E2A00F031
:101C80002081B4F8BC10B4F836230B449BB2D11AAF
:101C9000090454BF531C01339BB2A4F8363394F8A3
:101CA0003933B4F8361323B9B4F8E4328B4200F078
:101CB0002081B4F8FC20B4F8BC30B4F8FA00134426
:101CC000013BB4F86A231B1A9EB2531C721A120409
:101CD000A4F86A3300F1C9800DF10E0500230095C8
:101CE0001A462046FFF7F6FB002840F0A880A36FB5
:101CF0003BB3B4F8F620B4F836339B1A1BB2002B72
:101D00001FDDB4F87C100B44013BB3FBF1F313FB74
:101D10000123A4F8F63014E005B0BDE8F0430EF05E
:101D200051BB01200FF08AFA05B0BDE8F043FCF783
:101D3000B7BE90F82433042B40F0FB80002380F8DA
:101D4000243305B0BDE8F08390F838330022C0F8A2
:101D50007423002B00F0A480B0F83623B0F8BC3018
:101D60009A4200F0CB80D31AA0F8E632A0F8BC204B
:101D7000D4E9D4232046C4E9D6230BF099FA94F889
:101D8000EB32002BDDD094F87120E769D4F82C33C6
:101D9000DFF8A88112F00C0F14BF4FF4EE794FF466
:101DA000DA799F4288BFFF1A98F8083098BF002759
:101DB000002B00F0958004F1380017F009FE94F82C
:101DC0007160054630460EF045FED4F8F03280339F
:101DD00000F55F421D445A4B413216F00C0FA3FB35
:101DE000023205EB921514BF2823002302201D4464
:101DF00012F07AF87F1B27EAE776864228BF06466C
:101E00000221304612F0BEF800B935444A46294650
:101E1000204617F05DFEE269D4F8F032C8F80C00F5
:101E2000D01812F007F800288BD140F2A3313020EF
:101E3000FBF78CF805B0BDE8F04318F0A2BB012811
:101E400068D1B4F83613B4F8E0228B1A13F4004FBB
:101E5000BDF80E30194489B2A6EB01032CD11BB298
:101E6000002BA4F83613BFF639AF94F8C9303549C2
:101E7000002B0CBF3E23082384F8E73004F1DE007A
:101E800017F01EFD204618F07EFB002384F8243353
:101E900094F86C0311F07EF9202384F86C3350E73A
:101EA000B0F83433B0F8BC10B0F83423A0F8BC203C
:101EB0005B1AA0F8E6325BE71B0416D4A4F83613CD
:101EC0000CE7B4F83613013189B2A4F83613F0E602
:101ED000BE213020FBF73AF8C2213020FBF736F85C
:101EE000A36B9F4228BF1F4665E7B31A1BB211467A
:101EF000B6E7013189B2A4F83613DAE6B0F8E43275
:101F0000A0F8BC309B1AA0F8E63231E794213020CB
:101F1000FBF71CF840F25A613020FBF717F840F24B
:101F20001B613020FBF712F840F21A613020FBF7FA
:101F30000DF8B8213020FBF709F800BF7828002001
:101F4000D34D621039B501002DE9F0470026054652
:101F500080F81061D0F80C010127D5E9508982B0D2
:101F600080F8EE228A4685F82861394685F829717D
:101F700008F096FED5F80C41C4E9D68995F80831E9
:101F800084F86C33C4E9D889C4F870A384F8246356
:101F9000A4F8686333460096324631462046FFF780
:101FA00099FAC8B984F82473C4F82003C4F8180354
:101FB000A4F83603A4F83403B4F8BC3084F8390329
:101FC000013BA4F8BC30A4F86A030DF063FD02B035
:101FD000BDE8F04710F01ABF40F21B213020FAF79D
:101FE000B5FF00BFD0F80C01704700BF2DE9F043EA
:101FF00085B000230222CDE9003301268DF80620AA
:102000006846FBF7E9FD044620BB009D95F82831A2
:10201000002BF5D085F8506101212846FEF760FFBE
:1020200095F82831002BEBD095F8080111F094FCBD
:1020300095F8080112F0DAF895F8080111F0AAF8FD
:1020400000283BD085F828416846FBF7C5FD0446CB
:102050000028DAD0DFF87880012688F810600025A3
:102060004FF6FF771AE0029BE3B193F86C23202A26
:1020700018D01888B8421BD00121FBF775FD8146A6
:1020800008B390F86C0312F0B1F899F86C0389F872
:10209000244311F07FF8202389F86C33CDE90255F1
:1020A0008DF80E6002A8FBF797FD04460028DAD0F1
:1020B000002088F8100005B0BDE8F08340F2072149
:1020C0003020FAF743FF40F21F113020FAF73EFFAD
:1020D00078280020054B0022012142F210701A726C
:1020E000588219701A74FFF781BF00BF782800204A
:1020F00090F82831002B40F0A4802DE9F0410446EF
:102100000F4601465648154603F0FF0811F018F82F
:10211000202806466ED04146502204F5847012F005
:10212000A7FD012384F80861C4F80C7184F82831F4
:1021300037B109F0D1F900F00700013087F810033A
:102140002046FFF737F800274FF48173A4F83801D1
:10215000A4F83A3184F830710FF0D6F8B4F8386149
:10216000D23606442046B6B2FEF76AFD002844D0B7
:1021700016F0C4FA00F5CD6189B228460FF094F844
:102180002844C4F8340118F069FF301841F1000107
:102190000126C4F84001C4F8441184F81061E784B2
:1021A0002046FEF765FD002843D031462046FEF765
:1021B000FFFAA5F2F3452D1AC4F814514FF0FF327F
:1021C0006FF00043C4E9522394F8080104F59871B4
:1021D00011F052F900283ED0D4E9502300252046C2
:1021E000C4E94823A4F82A512946FEF779FE284677
:1021F000BDE8F0810C20BDE8F08101462046FEF7E5
:10220000D7FA184FF730C4F83401788A08B1E08C57
:10221000C8B9064418F022FF361841F10001C4E99C
:102220005061002DCAD0AE1941F10001C4E95261DC
:10223000CAE73046FEF76AFFF73D2D1AC4F814517D
:10224000BCE70C20704709F047F97B8AB0FBF3F23A
:1022500002FB1300DDE740F2E9113020FAF776FEC9
:10226000251201007828002090F828310BB90020B1
:10227000704710B50121044680F85011FEF730FE7A
:1022800094F828310BB9002010BD94F8080111F022
:1022900063FB94F8080111F0A9FF94F8080110F00D
:1022A00079FF20B1002384F82831002010BD40F2CE
:1022B00007213020FAF74AFE014B1872704700BF21
:1022C0007828002090F8502182B910B502F0FF0460
:1022D00090F8102112B90122104610BDD0E9453105
:1022E0009942F9D9FEF7AAFD2246F5E700221046E9
:1022F000704700BF10B504460DF07AF8074BDA6856
:10230000824208D3E16941F64B52914203D9187CCD
:1023100080F0010010BD002010BD00BF7828002013
:1023200008B54FF4FD7117F0FEFBB0F5296F28BF1B
:102330004FF4296080B208BD90F8EB32002B66D1D3
:1023400070B503F0FF0590F82433032B84B00446E6
:1023500001D004B070BD18F081FED4E9D623801AF4
:1023600061EB0301012871F10003F2DB6FF001035F
:10237000834275EB01034DDBE369B4F8BC20002B0D
:1023800046D0B0FBF3F080B2531C184480B2A4F8DE
:102390003403B4F83423B4F8E4329B1A1BB2002B94
:1023A000D7DD94F86C0311F0D7FA0028D1D0B4F837
:1023B000BC50B4F8FC10B4F8FA20FF230D4484F8A4
:1023C0003933013DAD1AB4F83433ADB2EB1A1A0407
:1023D000BFD40DF10E06B4F834130096002389B271
:1023E00001222046FFF776F80028B2D0012816D146
:1023F000B4F83433BDF80E2012FA83F39BB2A4F87C
:102400003433B4F83433EB1A1B04E4D5A1E7704736
:102410001846B9E740F2D1513020FAF797FD40F263
:102420000A613020FAF792FD2DE9F047044682B0A8
:10243000052900F2D980DFE801F0501603131C369D
:10244000042384F824330DF025FB10F0DFFCB4F8EE
:10245000BC20A4F836230023A4F86A3384F8393367
:1024600002B0BDE8F087032380F8243302B0BDE852
:10247000F0870CF0B7FF0546C4F8745394F8710068
:102480000EF0E0FA8542C0F0A88094F87100D4F80C
:1024900074430EF0D7FA574BDA681444241ADC6000
:1024A00002B0BDE8F08790F8715028460EF0D2FADD
:1024B000514900F55F4015F00C0F00F14100A1FB00
:1024C000003014BF2821002101EB901180312046FB
:1024D00002B0BDE8F04717F013BBD0F874339BB9D6
:1024E000444B1B7C03F0FF02002BA9D1B4F8E4128B
:1024F000009201232046FEF7EDFF0028A3D040F212
:10250000E4613020FAF722FD90F83A33002BE7D04F
:1025100090F82433032BE3D190F8719016F0EEF885
:1025200094F8D9320B2B5DD8344AD4F8745332F86E
:102530001330C61803F5C86348469FB20EF082FAFE
:1025400019F00C0FA5EB0008B6B248463CD10EF0CE
:1025500081FADFF8A4A0D4F8F05200F2E733AAFB26
:1025600003234846A8EB93180EF06CFA2D1A484640
:102570000EF070FA00F52343A133AAFB03239B0955
:10258000EB1A5A08603B293206FB03F3B3FBF7F35F
:102590006033A2EB530141454FEA530302D8134481
:1025A000434501D20FF016F9E06931460EF07CFE8A
:1025B000E26941F64B539A4298BF02300023C4F8B7
:1025C0002C0384F83A338BE7D4F8F0520EF03AFA41
:1025D000A8F13C082D1A6523D2E74FF46A71302028
:1025E000FAF7B4FCFEF7E0FD4FF4EE613020FAF7A5
:1025F000ADFC00BF78280020D34D621034170700CF
:10260000012A70B5064609D0022A14460D461ED08E
:102610004AB140F29A713020FAF798FC0CF0E8FECB
:10262000C6F8700370BD0CF0E3FE22460146284652
:10263000FFF78AFC0F4995F8080132460EF0D2FDEB
:102640000028EFD140F283713020FAF77FFCD0F8F8
:10265000701301222846FFF777FC064995F8080118
:1026600032460EF0BFFD0028DCD140F294713020DC
:10267000FAF76CFC211C0100F8B5044651B10129A0
:1026800063D1002380F810310DF004FABDE8F84062
:1026900010F0BCBBC58C002D4FD12046D4E9487644
:1026A000FEF7EAF8401941F10001C01946EB0106B6
:1026B0004FF481730022C4E95006A4F83A3184F83B
:1026C00030212046FEF776FDD4E9505694F850317B
:1026D000A4F83801C4E9485603F0FF017BB9D4E9F6
:1026E00052026FF000439A4208BFB0F1FF3F0FD192
:1026F00094F8080104F5987110F0BEFE50B3002361
:10270000A4F82A310DF0C6F9BDE8F84010F07EBB00
:102710002046FEF74DF8D4F84831D4F84C215B1B25
:1027200000F1F70062EB06021B1A62F10002002AB8
:10273000DEDA2046FEF782FBE1E708F0B5FEE58C25
:10274000B0FBF5F303FB1505A7E740F2AA713020B3
:10275000FAF7FCFB40F204713020FAF7F7FB00BFF8
:1027600090F82801704700BF014B5882704700BFA6
:102770007828002008B5032807D8DFE800F0040215
:102780000402002008BD012008BD40F22521772069
:10279000FAF7DCFB0B46062203F8032B044AB2F8D7
:1027A000330092F83520A1F803009A70704700BFFB
:1027B0009028002008B540F2B6313220FAF7C6FB67
:1027C000044A0023A2F8BA3082F8703082F8BC3094
:1027D000704700BF9028002008B508F027FB034B86
:1027E00018700DF0A7F8052008BD00BF10000020EC
:1027F00008B508F01BFB024B02461A70012008BD09
:10280000100000202DE9F041064617469846A1B178
:10281000B3681BB12FB13846BDE8F0810120BDE897
:10282000F081B8F1000FF6D01549B27C91F845005F
:10283000BDE8F041463116F0AFB9114D05F15B032B
:1028400095F85A2095F8900005F1890116F0A4F941
:1028500095F87830082B03D095F87B209A4207D062
:1028600095F85630012BD3D033B90028D0D1D6E714
:1028700095F85630012BCBD90020BDE8F08100BF80
:1028800090280020F8B5554C0546D4F8C000002328
:10289000032D03803AD0052D45D0514916F079FC1F
:1028A00094F89010D4F8C00016F087FC94F87D30AE
:1028B00094F845707BB194F85430032B2CD094F8E5
:1028C000780008F07FF9474B002806461ABF012719
:1028D00006461E4600E0434ED4F8C000314616F0CE
:1028E0004AFCD4F8C000394616F05AFCD4F8C000AF
:1028F0000DF014FC052D00D0F8BD236D3268C3F82F
:102900000A20B288DA81236D5F72F8BD294616F07D
:1029100010FCD4F8C000C0E794F84D30002BCED0A6
:1029200094F87B00CDE70E46294616F002FCD4F859
:10293000C070397821F0200141EA46113970236DC9
:102940001B6AC7F80F30226D936AFB74190A1B0CBF
:102950007B753975D169108E16F0C5FAB875236D7F
:10296000D4F8C060D969D86A16F0D1FA030AF075B4
:102970003376236DD4F8C060D86916F081FA030A63
:102980007076B376236DD4F8C0609A8CF276120A12
:102990003277DA8C7277120AB277D3F8CE20C6F883
:1029A0001F2093F8D23086F82330236D96F8242028
:1029B00093F8D93022F01F0203F01F03134386F867
:1029C000243007F065FB96F8243003F01F0343EA38
:1029D000401386F82430D4F8C0005EE79028002029
:1029E00019290020D6280020F8B51D4C1D4A94F85E
:1029F0007A30D75C054638460E460CF0C5FE94F892
:102A0000983084F88F701C4494F8BD40631E072BE7
:102A100020D8DFE803F0041D1F041F1F1F04FBF76D
:102A20008FFA402828BF4020C0B221460CF0E6FCB7
:102A300030460DF073FB214601202DB10DF08CF8CE
:102A4000003818BF0120F8BD0CF0A4FE0120F8BD2D
:102A50000D20EAE740F619113220FAF777FA00BFA5
:102A6000902800208817070010B5FBF763FA04468A
:102A7000FBF766FA81B2204614F0E0F848B10DF099
:102A80004DFB00200DF0B4FB044B062283F87020B0
:102A900010BD4FF4C3613220FAF758FA9028002095
:102AA00038B5114DFF2095F8B9100CF0A7FCFBF7D5
:102AB00041FA0446FBF744FA81B2204614F0BEF80E
:102AC00068B10DF02BFB95F8B90010F00C0018BFA1
:102AD00028200DF08DFB092385F8703038BD40F2B9
:102AE00043613220FAF732FA9028002070B506468A
:102AF000FBF720FA0446FBF723FA81B2204614F0D4
:102B00009DF8002846D0324C94F85430013B022BFB
:102B100004D941F2E1413220FAF718FAE6B994F803
:102B20007030042B45D994F870300A2B3CD894F8B7
:102B30007030D4F8C42003F180439269053B52F809
:102B4000233098470E282AD8D4F8C4301B69BDE832
:102B5000704053F820301847054616F025FD20B97F
:102B6000284616F03CFD0028D9D094F87030042B8C
:102B700024D994F870300A2B25D894F87030D4F802
:102B8000C42003F180435269053B284652F82330A4
:102B90009847D7E741F2DB413220FAF7D7F941F203
:102BA000F6413220FAF7D2F941F2D2413220FAF757
:102BB000CDF941F2D1413220FAF7C8F941F2714121
:102BC0003220FAF7C3F941F272413220FAF7BEF926
:102BD0009028002038B5224C94F87D30002284F8EB
:102BE000A82083B1D4E928126FF000439A4208BFAD
:102BF000B1F1FF3F07D018F031FAD4E92823904211
:102C000071EB030303D2022384F8703038BD012036
:102C100007F064FF0028F6D007F098FE054618F08C
:102C20001DFA6B015B1B4FEAD56262F10002520292
:102C300042EAD3525B025B1942F1000C4FEA8C1E50
:102C40009A014EEA936ED31A6EEB0C025B1942F1B5
:102C500000021B1842EB0101C4E92831D3E700BF91
:102C60009028002070B5474C0022236D62721A88AC
:102C7000628182B00546D8690E4616F001F9236DCF
:102C80002084998CDA8C61844FF47F43E3844FF67F
:102C9000FF73A2842385002D62D00121304616F0F7
:102CA000BFFB32780346D20994F87D1009B1002A9F
:102CB00033D194F87900344A002308286361938063
:102CC00039D0324A511E07F047FE002854D0637BAA
:102CD00043F002036373002D3DD12D480268C4F810
:102CE0001A202C4B82889A8094F95810206D16F087
:102CF000C3F829492348022216F0D6FD236D27493F
:102D00001D88274893F8CD30A4F83350022284F868
:102D1000353016F0DBFD02B070BD5A7902F0C0020A
:102D2000402AC6D11868606194F87900164A9B88D9
:102D300093800828C5D1154B94F89000D4F88910D9
:102D400060730022B3F87F00C4F80E10C4F81A2094
:102D500098801A82C8E70021304616F061FBBDE773
:102D6000D4F8C000694616F00DFAD4F8C0201278E5
:102D70006B46C2F3801297E741F22C513220FAF7EA
:102D8000E5F800BF90280020A42800209E280020FD
:102D900019290020AA280020693301009527010085
:102DA000BA28002008B508F041F8034B187002F06B
:102DB000E1FE012008BD00BF10000020024B0322ED
:102DC00083F8702004F096BC9028002008B540F2EB
:102DD00041413220FAF7BAF810B504788CB004F00B
:102DE0000F04224602A903F0F5FA0CF0A3FD08F047
:102DF0001DF8224A042C107002D005200CB010BD22
:102E0000039B1F4993F800C091F88940A445F4D171
:102E100093F801C091F88A40A445EED193F802C01E
:102E200091F88B40A445E8D193F803C091F88C4009
:102E3000A445E2D193F804C091F88D40A445DCD1BB
:102E40005C7991F88E309C42D7D19DF8194091F869
:102E500090309C42D1D17F280ED000907F2491F8F1
:102E60008F30147002A891F8A82091F8791002F020
:102E700079FF05200CB010BDFFF7A8FF100000205F
:102E8000902800202DE9F047054684B006290AD88D
:102E9000DFE801F0631F0F0909090400B44C94F83E
:102EA0008230002B7DD10CF045FD052004B0BDE83B
:102EB000F0870CF03FFDAE4A92F882302BB192F8C9
:102EC0005430013B012B40F2DB80052004B0BDE80B
:102ED000F087A74C837C94F87D6094F88280012B66
:102EE00086F001067CD04FF0000994F85430032B93
:102EF00000F0BC8094F87870082F40F0A68094F819
:102F000045704FF0000A3A46032B75D16B6894F870
:102F10005B101878884200F05081002794F87830D0
:102F2000082B04D094F87B10994208BF0127BAF10E
:102F3000000F40F0A380002E40F0DE80B8F1000FBB
:102F4000B1D094F85630012B03D0002BABD1002F19
:102F5000A9D0002EA7D00C20A8E7854C94F8823089
:102F6000002BA0D094F85430022B00F0CD80012B20
:102F700000F05881032B40F06D81436894F85B208A
:102F80001978914200F0938094F85630012BE2D0EA
:102F900094F87B30082B86D094F878209A4282D11E
:102FA000D9E794F85430022B00F0C880012B7FF44D
:102FB0007AAF704991F900307F2B00F0498102937C
:102FC00094F88F30019394F8793000937F260E7037
:102FD000FF2304F14602062102F006FE052065E704
:102FE000836893F8059009F0C009A9F14009B9FA7E
:102FF00089F94FEA591978E70CF09CFCB8F1000FF9
:103000003FF463AFAB68AA7C5B4994F8450015F0C8
:10301000C3FD18B9BAF1000F00F0B080554991F91D
:1030200000307F2B00F01481029394F88F2094F8E5
:10303000793000937F24019228460C704E4A3B461B
:10304000012102F0D1FD052030E7384607F094FB5E
:10305000002818BF0646B9F1000F40F0D38094F85D
:10306000457094F854303A46CA464DE794F84D20DE
:10307000002A3FF43FAF94F87B703DE701265DE7FF
:103080003C4991F900307F2B00F0E280029392F8E6
:103090008F30019392F8793000937F2428460C708A
:1030A000FF234632022102F09FFD0520FEE65978FB
:1030B00094F85C2091427FF467AF997894F85D2092
:1030C00091427FF461AFD97894F85E2091427FF409
:1030D0005BAF197994F85F2091427FF455AF5A792C
:1030E00094F860309A427FF44FAF427C94F85A30A3
:1030F0009A427FF449AF2EE71046AB68AA7C1E497E
:1031000015F04AFD064619E71A4A92F900307F2B5E
:1031100000F09E80029394F88F30019394F87930F8
:1031200000937F211170FF2304F14602002102F079
:103130005BFD012384F8A8300B20B7E60D4A92F915
:1031400000307F2B00F08480029394F88F3001933D
:1031500094F8793000937F211170FF2304F1460227
:10316000062102F041FD002384F8A8300B209DE6E3
:103170009028002010000020D628002094F8553018
:10318000023B012B3FF6A1AEB9F1000F3FF49DAE1B
:10319000334991F900307F2B5AD0029394F88F2055
:1031A00094F8793000937F260192FE230E702D4A09
:1031B0002846012102F018FD87E6587894F85C1043
:1031C00088427FF4AAAE987894F85D1088427FF424
:1031D000A4AED87894F85E1088427FF49EAE187939
:1031E00094F85F1088427FF498AE597994F8603073
:1031F00099427FF492AE6F7C94F85A30FB1A5F428A
:103200005F418BE63846A96807F09CFC94F845209E
:1032100094F854308246174600283FF475AE42F0C9
:10322000020771E60E4991F900307F2B10D002930E
:1032300094F88F30019394F8793000937F260E70C4
:10324000FF2304F14602002102F0CEFC05202DE60A
:10325000FFF7BCFD4FF46A613220F9F777FE00BF3B
:1032600010000020D628002010B5164B93F900203E
:103270007F2A84B023D07F241C70134B93F87040B6
:10328000052C15D093F87040082C0CBF03240124A2
:10329000039493F87940CDE9014293F88F400B4AAB
:1032A00093F8B930009402F043FE18B904B010BD91
:1032B0000024EDE704B0BDE8104002F01BBCFFF7AE
:1032C00085FD00BF1000002090280020D628002097
:1032D00010B5104A92F87030042B10D992F8703063
:1032E0000A2B11D892F87030D2F8C42003F1804331
:1032F000D268053BBDE8104052F82330184741F230
:10330000D8513220F9F722FE41F2D9513220F9F793
:103310001DFE00BF902800200B46182203F8032B47
:10332000104AB2F83FC092F84100A1F803C0CA7831
:103330009870012A00D0704710B58C880021204673
:10334000FAF712FC38B1204606F0F0FF00212046C3
:10335000FAF720FC00B910BD40F219413220F9F70C
:10336000F5FD00BF9028002038B5244B5A7A0C4652
:1033700052BB1A6DD3F80E10C2F80310598AA2F886
:1033800007105A7B1B6D12F0FD0F14BF01220022A3
:103390009A7022461A4B132102F8031B03F1200EE8
:1033A0001D6858689968D3F80CC0C2F80CC0103377
:1033B000734515605060916002F11002F0D11978E8
:1033C00011700023A37138BD58890021FAF7CCFB96
:1033D000054668B1008806F0A9FF28880021FAF7A1
:1033E000D9FB0028D5D040F2FD313220F9F7AEFDEF
:1033F00040F2F9313220F9F7A9FD00BF90280020F2
:10340000992800202DE9F041264C94F8BC305F2B20
:1034100006460D4631D85A09234B13441F7994F8B8
:10342000BA00C0F3050800F03F000CF0ADF984F8D5
:103430008F80B6B1394601200CF08EFB78B194F83C
:103440008830022B39460CBF4020FF200BF0D6FFFE
:1034500094F8A8309BB128460CF060FE0120BDE82E
:10346000F081616F3A4601200CF0C2FC0028E6D1E1
:1034700040F648113220F9F769FD0027CFE7681DB3
:1034800007F0B6FA84F87C000028E4D017F00C0F9F
:1034900014BF552450240BF0ABFB20460CF0EAFE81
:1034A000D9E700BF9028002088170700F8B53D4CE9
:1034B00094F8BC305F2B054629D85A093A4B13447F
:1034C0001E79636F73B1FAF735FD0746FAF738FDD9
:1034D00081B2384613F0B2FB014600285DD00020CF
:1034E000FFF790FFD4F894000CF050FE94F854309D
:1034F000022B31D0032B0CD0EDB140F20113A4F814
:10350000A930002384F8B96084F88030F8BD002623
:10351000D7E794F88830012BEED116F00C0F2AD0A3
:1035200094F85930012B14BF3146042100200CF0CF
:10353000C7FE002DE1D194F88830022B13D0012B67
:103540001BD0002BDDD102F08BFC84F8A90002F027
:103550004DFA84F8AA00D4E794F88830022BDCD026
:10356000002DCAD1EBE70023A4F8A95084F8B96074
:1035700084F88030F8BD3146D8E794F8B930A3F12B
:103580000203B3FA83F35B094FF0000263F307020F
:1035900063F30F22A4F8A920B3E74FF4BB613220F4
:1035A000F9F7D4FC902800208817070038B50546A5
:1035B0000C4606F047FD420704D4A37803F0E0036D
:1035C000402B0DD006F03EFD830704D4A37803F012
:1035D000E003202B04D0237803F03F03242B01D9F0
:1035E000002038BD0BF0E0FE94F90030A17862783D
:1035F000002B01F01F03ACBF4FF01E0C4FF4967C64
:1036000042EA03230CFB03F31A1AB2F5877FE7D3D0
:103610009842E5D8054B2288A3F8BA2083F8BC105D
:103620002846BDE8384003F0FDBF00BF90280020C9
:1036300070B5294C94F8823086B06BB394F8A830FA
:10364000054633B90378002B0CBF0123022384F80D
:10365000A83094F87030082BDAB231D0092A14BFA0
:10366000012602261D4890F900307F2B32D0CDE98B
:10367000023694F8793001934FF07F0C94F88F3034
:103680000093174A80F800C094F8B930284602F039
:103690004FFC20B9022E15D1002006B070BD68780D
:1036A00010F0100611D0A9690220FFF77FFF0590E6
:1036B00040B1002384F888300CF03CF90598ECE721
:1036C0000326CFE702F056FAE6E702F013FA304697
:1036D00006B070BDFFF77AFB902800201000002094
:1036E000D628002010B504468AB007F09FFB237847
:1036F000174A03F00F03072B107002D001200AB005
:1037000010BD6946204602F0FFFE9DF80030002201
:103710000292002BF2D19DF80130DB07EED50D4C63
:10372000019994F890209DF8110004F1890315F097
:1037300033FA0028E2D0012104F1840014F0ADFF37
:10374000FF216846FFF774FF0028D7D00320D6E793
:10375000100000209028002070B5574C94F870306D
:10376000012B05460E4603D9DAB2032A40F08D80BC
:103770002B7B84F898302344AA6893F8BD3084F8F2
:10378000B9302B68C4F8943062672B79022B52D180
:103790006B7B2BB194F8693013B9616E00297AD133
:1037A0002B79012B2AD03BD894F87A30434A013345
:1037B000A2FB031505F4FF7000EB550094F84C10C4
:1037C0001B1A41FA03F5ED07D8B215D40133A2FB59
:1037D000030525F0010000EB55001B1A41FA03F523
:1037E000E907D8B208D40133A2FB030222F001009A
:1037F00000EB52029B1AD8B284F87A0094F9580070
:103800000BF0B2FF31460120FFF7EEF830B1FFF7C1
:10381000E1F92B4BD3F85035032B42D0002070BD7B
:10382000023B012BF5D894F958000BF09DFF0423BF
:1038300084F87030EDE70BF077FE0CF027FD0BF00D
:10384000F5F920480CF054FC1F480CF04BFC1F48C5
:103850000BF090FF94F86C30CBB1022011F0BEFA5F
:103860002B79032B05D030460CF058FC2B79032B19
:103870008ED1636FD3B931460120FFF7C3FD002815
:10388000CCD06B7B002B85D18AE70C2070BD01204A
:1038900011F0A4FAE4E794F8680001220DF0B2FCFC
:1038A0007EE740F68C213220F9F750FB40F6662186
:1038B0003220F9F74BFB00BF90280020ABAAAAAA40
:1038C00000100040A001002055555500D6BE898E3D
:1038D0002DE9F04104468AB007F0A8FA2378434A5C
:1038E00003F00F03082B107004D0012528460AB0FE
:1038F000BDE8F0816946204602F09EFD9DF800502B
:10390000002DF2D19DF8013003F00303032BECD11D
:10391000374E96F84D307BB396F87B7096F87C3036
:103920006BBB344B96F8902001999DF8110015F06F
:1039300033F90028D9D096F87D3096F84580002BD1
:1039400040D12D4B9DF812000299012829D0424602
:1039500015F022F90028C8D02848012114F09DFE56
:1039600096F87C30002B39D121460120FFF77AF9F7
:10397000032004F05BF8B9E796F87870CEE715F00D
:103980004FF908288046CCD086F87900194B96F874
:10399000902001999DF8110015F0FEF8B845CAD0A5
:1039A000C7E74A7902F0C002402AD0D1424615F05A
:1039B000F3F80028D0D10299384607F0C3F8002860
:1039C000CAD192E7384607F0FDF80B4A00280346B3
:1039D0001ABF4FF0010803461346B3E70CF056FC3C
:1039E0000BF024F9002386F87C30BDE7100000209E
:1039F0009028002019290020D62800201429002012
:103A00002DE9F0430729044685B040680D46174666
:103A10003ED1002877D0637C012B00F09C806B4E58
:103A200096F87800082852D002AA0DF1070106F096
:103A300093FF002800F0C5809DF8070002A916F04A
:103A400074FC8146062D96F84D8077D8B8F1000FAA
:103A500008BFC8465E4B86F882801B6823B1394692
:103A60002046984786F88300636843B1627C86F8F5
:103A700090201968C6F88910564A9B889380B6F83A
:103A80008230A06808B1072D31D005B0BDE8F083C1
:103A900000287AD0637C012BC1D1437903F0C003A5
:103AA000402BBCD1494E96F87C30002BB8D015F095
:103AB000B7F84FF0000360F3070360F30F23A6F895
:103AC000783008284FF0010386F88030ACD1616867
:103AD000607C16F02AFC404A61688146607C06F0F2
:103AE00075FE03460028ADD1A6F88200C9E796F816
:103AF00078100829C9D0002BC7D006F069FF012330
:103B000086F88130C1E7002A45D0304E96F84D80C6
:103B1000814696F88230002B51D06368002B95D1F6
:103B200002F09EF918B196F88230002B47D1B8F117
:103B3000000F8FD106F044FE80468BE7082D27D872
:103B4000002FE6D16368002B80D16378DB06E7D5D0
:103B50004FF001087EE7437903F0C003402B7FF468
:103B60005EAF1A4E96F87C30002B3FF459AF002F11
:103B70009DD196F8B910012999D106F00BFF86F86E
:103B80007C0000283FF44CAF91E7104E814659E786
:103B90004FF000085EE70D4C012584F8825094F840
:103BA000AB30002B3FF471AFD4F8AC00503016F0BE
:103BB0009FFE00287FF469AF84F8835065E798463C
:103BC00048E740F6FC413220F9F7C0F99028002080
:103BD0007000002019290020082900202DE9F04F4D
:103BE000354F847C97F87D80012C83B006468A4649
:103BF0009346994688F0010833D0002497F87C500A
:103C00002346E5B197F85420032A31D07268FAB1FF
:103C100097F87850082D21D02846019306F0ACFD86
:103C2000019B002818BF8046CBB197F88130002B4C
:103C30003AD014F0FFFF0023054687F881308BF857
:103C400000508AF8004089F8008003B0BDE8F08F8A
:103C5000019302F005F9019B0028D9D17BB9002519
:103C6000EDE783685B7903F0C003402BC5D1C5E75E
:103C700097F84D20002AC9D097F87B50CAE797F8EB
:103C800080100029EBD1B068019106F083FE054653
:103C900087F87C000028D2D014F0C2FF08280199D0
:103CA00008D087F87800CAE72846B16806F04AFFCE
:103CB0000546C4E70D46C2E79028002008B507F086
:103CC000B5F8024B02461A70012008BD1000002012
:103CD00038B51B4C0E2094F8B9100BF08FFBFAF797
:103CE00029F90546FAF72CF981B2284612F0A6FF09
:103CF00000B305460CF012FA94F8B90010F00C006D
:103D000018BF28200CF074FA681D94F8B95006F01A
:103D10006FFE84F87C0048B115F00C0F14BF5525D8
:103D200050250AF065FF28460CF0A4FA0A2384F80F
:103D3000703038BD40F22C613220F9F707F900BF2E
:103D40009028002010B50B4C07F070F80A4A94F840
:103D50007C3010701BB90BF0EDFD052010BD0CF090
:103D600095FA0AF063FF002384F87C300BF0E2FD43
:103D7000052010BD902800201000002010B50C4C2C
:103D800094F87C305BB90B4A0023A4F8BA300121C7
:103D9000937084F87010BDE8104003F01BBE0CF067
:103DA00075FA0AF043FF002384F87C30EBE700BF8C
:103DB000902800204A29002010B50E4C94F87C3041
:103DC0007BB90D4BD4F8C0100020A4F8BA0098704D
:103DD00084F87000FEF746FFBDE81040022003F0B3
:103DE00025BE0CF053FA0AF021FF002384F87C3042
:103DF000E7E700BF902800204A29002070B54E4C0C
:103E000094F87030012B05460E4603D9DAB2032A26
:103E100040F082802B7B84F898302344AA6893F882
:103E2000BD3084F8B9302B68C4F8943062672B79C0
:103E3000022B14D16B7B002B61D194F958000BF04D
:103E400093FC31460120FEF7CFFD30B1FEF7C2FEF4
:103E50003A4BD3F85035032B69D0002070BD0BF0DE
:103E600063FB0CF013FA0AF0E1FE35480CF040F960
:103E700034480CF037F934480BF07CFC94F86C3083
:103E8000002B4BD0022010F0A9FF2B79032B34D04C
:103E900030460CF043F96B7B8BBB2B79032B41D065
:103EA000002BCAD194F87A30284A0133A2FB0315BB
:103EB00005F4FF7000EB550094F84C101B1A41FA02
:103EC00003F5ED07D8B215D40133A2FB030525F0A5
:103ED000010000EB55001B1A41FA03F5E907D8B2BF
:103EE00008D40133A2FB030222F0010000EB5202CE
:103EF0009B1AD8B284F87A009FE76B7B93B194F851
:103F00006930002BC9D1616E0029C6D094F86800D1
:103F100001220DF077F9C0E70C2070BD012010F0F0
:103F20005DFFB2E740F645213220F9F70FF840F681
:103F300053213220F9F70AF89028002000100040A1
:103F4000A001002055555500D6BE898EABAAAAAA5D
:103F500010B50C4C94F87C305BB90B4A0023A4F8E4
:103F6000BA300121937084F87010BDE8104003F05E
:103F700031BD0CF08BF90AF059FE002384F87C3037
:103F8000EBE700BF902800204A29002010B50E4C16
:103F900006F04CFF0D4A94F87C3010705BB90C4A67
:103FA0000023A4F8BA300121937084F87010BDE8A2
:103FB000104003F00FBD0CF069F90AF037FE002342
:103FC00084F87C30EBE700BF902800201000002030
:103FD0004A29002010B50F4C01F0CCFD06F026FF59
:103FE0000D4A94F87C3010705BB90C4A0023A4F899
:103FF000BA300121937084F87010BDE8104003F0CE
:10400000E9BC0CF043F90AF011FE002384F87C307F
:10401000EBE700BF90280020100000204A29002074
:1040200010B506F003FF104C104B0246002104F1BE
:1040300084001A7014F031FB94F87C305BB90C4AA0
:104040000023A4F8BA300121937084F87010BDE801
:10405000104003F0BFBC0CF019F90AF0E7FD002393
:1040600084F87C30EBE700BF90280020100000208F
:104070004A29002010B506F0D9FE104C104B02461C
:10408000002104F184001A7014F007FB94F87C30CE
:104090005BB90C4A0023A4F8BA300121937084F86C
:1040A0007010BDE8104003F095BC0CF0EFF80AF07A
:1040B000BDFD002384F87C30EBE700BF9028002092
:1040C000100000204A29002038B5052003F0AAFA84
:1040D00048B1114C012094F8B9100CF0F1F80D23FF
:1040E00084F8703038BD0C4D95F87C305BB90B4AC4
:1040F0000023A5F8BA300121937085F87010BDE84F
:10410000384003F067BC04460CF0C0F80AF08EFD9E
:1041100085F87C40EBE700BF902800204A2900206A
:1041200038B503200021FEF7ADFB032003F07AFA37
:1041300040B1012108460CF0C3F80E4B0B2283F866
:10414000702038BD0B4D95F87C305BB90A4A0023CE
:10415000A5F8BA300121937085F87010BDE8384099
:1041600003F038BC04460CF091F80AF05FFD85F8C6
:104170007C40EBE7902800204A29002070B5F9F731
:10418000D9FE0446F9F7DCFE81B2204612F056FD56
:10419000A8B31D4C0E230546012084F8703003F0AF
:1041A00045FC00210520FEF76DFB062003F03AFADE
:1041B000064670B194F8B91001200CF081F82B7804
:1041C000226DC3F34013012184F8913082F8CD10A1
:1041D00070BD94F87C305BB90C4A00230121A4F82F
:1041E000BA3084F870109370BDE8704003F0F2BBF1
:1041F0000CF04CF80AF01AFD84F87C60ECE740F211
:10420000AF613220F8F7A2FE902800204A29002052
:1042100070B5274C94F8BC305F2B2AD85A09254B2F
:1042200013441D79636F6BB1F9F784FE0646F9F705
:1042300087FE81B2304612F001FD014698B300209E
:10424000FFF7E0F8D4F894000BF0A0FF94F8543096
:10425000022B1CD0032B0ED040F2011100220823A8
:10426000A4F8A91084F8B95084F8802084F870303C
:1042700070BD0025D6E794F88830012BECD115F0FD
:104280000C0F09D1294600200CF01AF8E4E794F845
:104290008830022BE0D1F2E794F85930012B14BF9B
:1042A00029460421EFE74FF4BB613220F8F74EFEB8
:1042B000902800208817070010B5B8B9A9B11C4A8A
:1042C00092F870300A2B29D992F870300E2B2AD828
:1042D00092F87030D2F8C42003F1804392680B3B0F
:1042E000BDE8104052F82330184710BD104C94F828
:1042F0007C305BB90F4A0023A4F8BA3001219370D7
:1043000084F87010BDE8104003F064BB0BF0BEFFF2
:104310000AF08CFC002384F87C30EBE741F2A851D2
:104320003220F8F713FE41F2A9513220F8F70EFEC1
:10433000902800204A29002070B582B0F9F7FAFDD4
:104340000446F9F7FDFD81B2204612F077FC002803
:104350003AD0204E0C230546002086F8703003F03A
:1043600065FB336D297893F8CD4004EA511404F0CD
:10437000010405202146FEF785FA042003F052F9D6
:1043800048B12B78326DC3F3401386F8913082F830
:10439000CD4002B070BD96F87C3063B90E4A002360
:1043A0000121A6F8BA3086F87010937002B0BDE80B
:1043B000704003F00FBB01900BF068FF0AF036FC71
:1043C000019886F87C00E9E740F287613220F8F72F
:1043D000BDFD00BF902800204A29002070B53A4C4E
:1043E00094F8BC305F2B2ED85A09384B13441D79F2
:1043F000636F73B1F9F79EFD0646F9F7A1FD81B22F
:10440000304612F01BFC0146002858D00020FEF771
:10441000F9FFD4F894000BF0B9FE94F85430022B55
:104420002DD0032B11D094F88830022B13D0012B00
:1044300015D0DBB30022072384F8B95084F880201C
:1044400084F8703070BD0025D2E794F88830012BD5
:1044500019D0022BEDD10023A4F8A930EAE794F893
:10446000B930A3F10203B3FA83F35B094FF0000202
:1044700063F3070263F30F22A4F8A920DAE794F8A4
:104480008830022BD3D115F00C0F08D1294600201B
:104490000BF016FF94F88830022BC8D1DBE794F8B4
:1044A0005930012B14BF29460421F0E701F0D8FC54
:1044B00084F8A90001F09AFA84F8AA00BAE74FF448
:1044C000BB613220F8F742FD9028002088170700D2
:1044D000B0B582B0F9F72EFD0446F9F731FD81B28F
:1044E000204612F0ABFB00286CD0394C054601F099
:1044F000CBFA94F898302344002093F8BD7084F8E8
:10450000B97003F08FF8002843D094F87030022B74
:104510002DD1012F1ED1E81C06F06AFA84F87C0028
:1045200028B140250AF064FB28460BF0A3FE94F85E
:104530005430023B012B21D9002340F6080105220B
:10454000A4F87810C4F8803084F8A83084F870207B
:1045500002B0B0BD681D06F04BFA84F87C0000285C
:10456000E5D017F00C0F14BF55255025DAE7294682
:104570000020FEF739FA012FCDD0EBE794F8983000
:10458000234493F8BD100129D6D100200BF098FEEA
:10459000D2E794F87C3063B90E4A00230121A4F8D5
:1045A000BA3084F87010937002B0BDE8B04003F0E8
:1045B00011BA01900BF06AFE0AF038FB019884F8FA
:1045C0007C00E9E74FF4A1613220F8F7BFFC00BF9F
:1045D000902800204A29002008B506F027FC044B4B
:1045E00018700BF0A7F9BDE80840FFF771BF00BFD6
:1045F0001000002010B50D4C06F018FC0C4A94F881
:104600007C3010702BB90BF095F9BDE81040FFF726
:104610005FBF0BF03BFE0AF009FB002384F87C30FF
:104620000BF088F9BDE81040FFF752BF902800203A
:104630001000002038B5184C94F869300BB9616E41
:10464000D9B994F87030012BDAB207D9022A03D114
:10465000FFF73EFF002038BD0C2038BD94F87C30B9
:1046600093B90E4B00250122A4F8BA509D7084F82E
:10467000702003F0AFF9284638BD94F8680003F0C5
:10468000FF020CF0BFFDDCE70BF000FE0AF0CEFAF3
:10469000002384F87C30E4E7902800204A29002099
:1046A00038B5244C94F869300BB9616E39BB94F875
:1046B0007030042B3BD8DFE803F003031D03120026
:1046C00094F87C305BBB1C4B00250122A4F8BA5047
:1046D0009D7084F8702003F07DF9284638BD94F869
:1046E000A8509DB92846FEF7E1FE072384F87030F4
:1046F000284638BDFFF7ECFE0025284638BD94F863
:10470000680003F0FF020CF07DFDD0E70120FEF70A
:10471000CDFE0025082384F87030284638BD0BF004
:10472000B5FD0AF083FA002384F87C30CBE70C2532
:10473000E3E700BF902800204A290020F0B5054695
:104740008FB006F073FB2C78774B024604F00F0411
:104750001A702846224604A901F03CFE072C4BD1D2
:104760000598002800F091809DF82130012B00F081
:10477000B2806E4D95F8780008285ED002AA0DF13F
:10478000070106F0E9F8002800F0C8809DF807004E
:1047900002A915F0CAFD0646062C95F84D7000F2E8
:1047A0008680002F08BF3746614B85F882701B68F2
:1047B00023B1002104A8984785F88300059B4BB1DD
:1047C0009DF8212085F890201968C5F88910594A6C
:1047D0009B889380B5F88200069B0BB1072C47D0CD
:1047E000214604A8FEF74EFB95F87C300446002BCA
:1047F00034D120460FB0F0BD059E002E69D09DF843
:104800002130012BB5D1737903F0C003402BB0D117
:10481000464D95F87C30002BACD014F001FA4FF0E7
:10482000000360F3070360F30F23A5F8783008282E
:104830004FF0010385F88030A0D105999DF8210043
:1048400015F073FD3C4A059906469DF8210005F0D8
:10485000BDFF0028A0D1A5F88200BDE70BF016FD32
:104860000AF0E4F90023204685F87C300FB0F0BD53
:1048700095F878100829B3D00028B1D0184606F072
:10488000A7F8012385F88130AAE7284D012685F88D
:10489000826095F8AB30002BA2D0D5F8AC00503038
:1048A00016F026F800289BD185F8836098E7082C3D
:1048B00029D8059B002B7FF474AF9DF81130DB06DF
:1048C00023D401F0CDFA10B395F88230FBB11F4626
:1048D0006AE7164D60E7437903F0C003402B7FF48D
:1048E00048AF124D95F87C30002B3FF443AF95F85C
:1048F000B910012991D106F04DF885F87C00002807
:104900003FF438AF89E700274EE701274CE7002F37
:104910007FF44AAF05F054FF074645E740F6FC41F7
:104920003220F8F713FB00BF100000209028002071
:104930007000002019290020082900202DE9F041ED
:104940009D4C94F8573086B05BB194F882300546A0
:104950006BB12E78012E11D0022E00F0A580002E12
:1049600042D00AF0E7FF052006B0BDE8F08194F8D8
:104970008330002BF5D02E78012EEDD10AF0DAFF2E
:1049800094F8B930022B6B7800F0C08003F0180364
:10499000182BE8D194F85430032B00F0BD80874ADF
:1049A00092F900307F2B00F00481029394F8793063
:1049B00001937F2194F88F300093117000220392AD
:1049C00094F8B9307E4AFF21284601F0B1FA002858
:1049D000C9D0A9690120FEF7E9FD0028C3D0012351
:1049E00084F888300320BFE70AF0A4FF94F854301D
:1049F000032BB8D06B7813F0100F14BF08220122DC
:104A0000C3F3001732EA0303ADD1AB688DF815602C
:104A10008DF816608DF81760002B00F094800DF172
:104A200017030DF115020DF116012846FFF7D6F810
:104A30009DF8153094F84580002B40F0AE80AB68AF
:104A4000AA7C5F49404614F0A7F878B994F855302D
:104A5000023B012B87D89DF81630002B83D09DF8A0
:104A60001530002B7FF47FAF4FF0FE08002F6DD084
:104A7000524890F900307F2B00F09B80029394F80D
:104A800079300193002694F88F3000937F270396A6
:104A900094F8B93007704A4A4146284601F048FA6E
:104AA00000283FF460AF26E00AF044FF94F8543049
:104AB000032B3FF458AF6B7803F01803182B7FF4E7
:104AC00052AF3E4991F900307F2B72D0029394F897
:104AD00079300193002294F88F3000937F20039265
:104AE00094F8B9300870364AFF21284601F020FAC0
:104AF00000283FF438AFA9690120FEF757FD0028D0
:104B00003FF431AF84F8886003202DE703F01903E8
:104B1000192B3FF43FAF26E769680023B1FA81F112
:104B20001A4649092846FDF76DFE00283FF41BAFE1
:104B3000AB699B7813F0E00332D194F87E30002B00
:104B40007FF42DAF0FE74FF0FF088FE71B4A92F974
:104B500000307F2B2DD094F870107F200529107025
:104B600005D094F87020082A0CBF0326012694F87B
:104B7000792094F88F100091CDE90123039694F8E1
:104B8000B9300F4A4146284601F0D2F900283FF4D7
:104B9000EAAE00F0AFFF0520E6E648F0020865E760
:104BA000402B7FF4FCAE94F87F30002B7FF4F7AEFF
:104BB000D9E6FEF70BF900BF902800201000002076
:104BC000D628002030B505468BB006F02FF92C789A
:104BD0004E4B024604F00F04284669461A7001F055
:104BE00093FC072C3CD04A4D002221466846FEF734
:104BF00007FF95F8B930013B072B71D8DFE803F0C8
:104C00000F06700470707004072C24D00AF092FE16
:104C1000052495F87C3083B920460BB030BD062CB6
:104C200002D0F3D8022CF1D821466846FEF72AF9C3
:104C300095F87C300446002BEED00BF027FB09F0F2
:104C4000F5FF0023204685F87C300BB030BD9DF881
:104C50000030012BDAD16846FFF770FE0446D8E732
:104C60009DF80030022B13D0294D012B95F8B92067
:104C70003BD0BBB912F00C0F14D09DF80120D10627
:104C800010D522F0030201938DF80120029309E070
:104C90009DF801301E4D002223F0030301928DF890
:104CA00001300292002207216846FEF7A9FE95F81E
:104CB000B930013B072B13D801A252F823F000BFF3
:104CC000574C01004F4C0100E14C0100574C0100D2
:104CD000E14C0100E14C0100E14C0100574C0100A6
:104CE00041F267313220F8F731F99DF801100023C5
:104CF0006FF34101022A8DF801100293D2D0CAB29B
:104D000063F3000201938DF80120CBE7100000202F
:104D100090280020F0B5B04C91B00D4606A901F0E6
:104D2000F3FB94F8A9303BB19DF8193000226FF3E2
:104D300000038DF81930079294F8AA303BB19DF822
:104D4000193000226FF341038DF8193008929DF855
:104D5000180094F88830984209D000F00BFF012524
:104D600094F87C30002B62D1284611B0F0BD294662
:104D700006A801F0F1FA78B99DF819301B07ECD5B7
:104D80000B9B58781A7800F00F0142EA01210009C4
:104D900001F002FB0028E0D02A46072106A8FEF712
:104DA0002FFEB4F88230002BD7D0089B00228DF85C
:104DB00015208DF816208DF81720002B41D00DF10D
:104DC00015020DF117030DF1160106A8FEF706FFF7
:104DD0009DF8152094F845609DF816700AB146F0CC
:104DE00002069DF817309DF81850012D73D0022D42
:104DF0002BD0002DB1D194F85430032BAFD09DF8B7
:104E000019309B0700F19880FF2694F8833033B166
:104E1000724B1B681BB10D9808B10F99984731462A
:104E200006A8FEF705FC002899D0032598E70BF0AB
:104E30002DFA09F0FBFE0023284684F87C3011B0DF
:104E4000F0BD1F461A46FF26CDE794F854100329FB
:104E500085D09DF8190000F00905092D7FF47FAF7A
:104E6000022900F0CF8010F0020000F091804AB9D2
:104E7000089B9DF82A205A4994F8450013F08CFEAF
:104E800000284AD0574A92F900307F2B00F0F98071
:104E900094F870107F200529107000F0F48094F8C9
:104EA0007020082A0CBF03220122039294F8792073
:104EB000CDE9012394F88F20009294F8B930484A44
:104EC000314606A801F034F800283FF448AF00F05E
:104ED00011FE012544E79DF8190094F8A91000F08F
:104EE000090CBCF1090F06D000293FF438AF10F0CF
:104EF000080F3FF434AF94F854C0BCF1030F73D0E3
:104F000010F0020044D082BB089B9DF82A2034494F
:104F100094F8450013F040FE38BB94F85530023B3E
:104F2000012B3FF61CAF002F3FF419AFFE2106A85E
:104F3000FEF79AF9012513E7002A7FF466AF089B74
:104F40009DF82A20264994F8450013F025FE0028F4
:104F50007FF45BAF94F85530023B012B3FF6FFAE78
:104F6000002F3FF4FCAEFE264FE71E4A92F90030B8
:104F70007F2B00F0868094F870107F200529107038
:104F800078D094F87020082A08BF032503958DE790
:104F9000144A92F900307F2B73D094F870107F255B
:104FA0000529157005D094F87020082A0CBF03203D
:104FB000012094F8791094F88F20CDE90230CDE9E2
:104FC000002194F8B930064AFF2106A800F0B0FF8E
:104FD00000283FF4C4AE7AE7902800206401002046
:104FE000D62800201000002006A8FDF70BFC0028A2
:104FF0003FF4B5AE254813F072FB00283FF4AFAE86
:105000000E25ADE610F0020136D062B9002B84D037
:10501000089B9DF82A201E4994F8450013F0BCFD1A
:1050200000283FF47AAF1B4B93F900507F2D18BF37
:10503000002126D07F2203201A70FDF723FC0123D4
:10504000039394F8793094F88F200092CDE90135DC
:105050000F4A94F8B930314606A800F069FF0028DD
:105060003FF47DAE094813F03AFB00283FF477AED9
:105070000D2575E6002589E7064B93F900507F2D35
:10508000D8D1FDF7A3FE00220FE700BF14290020AE
:10509000D62800201000002010B5044605F0C6FEFA
:1050A0002378084A03F00F03072B107005D1204620
:1050B0000321BDE81040FFF72DBE00F05BFD01208D
:1050C00010BD00BF1000002010B5044605F0AEFE74
:1050D0002378084A03F00F03072B107005D12046F0
:1050E0000121BDE81040FFF715BE00F043FD01208F
:1050F00010BD00BF10000020034B93F83E000038A5
:1051000018BF0120704700BF90280020024B187A7A
:10511000003818BF012070479028002010B5094CB6
:10512000236D53B1022262721B88074963812046B6
:1051300014F0BAFB0023236510BD40F22B4132204E
:10514000F7F704FF902800206933010038B5234C9D
:1051500094F87030012B054602D094F87030D3BB20
:10516000F8F7E0FE00F056FC94F87C305BBB42227E
:1051700000211A480FF07CFD002040F2071384F84C
:10518000540084F87A0084F8585084F8A800A4F8F1
:105190004C30FF2284F8692084F86800606684F847
:1051A0006900012140F2012284F8AB00C4F8AC0090
:1051B00084F8BD1084F84400A4F85420A4F84C30BE
:1051C00084F8570038BD0BF061F809F02FFD00237B
:1051D00084F87C30CBE70C2038BD00BF902800203D
:1051E0000F4BD3F8C42010B5C3F8C00072B1002231
:1051F0000C46A3F8BA2083F8BC2083F8702000F096
:1052000009FC2046FFF7A2FF28B910BD40F6B311F4
:105210003220F7F79BFE40F6B9113220F7F796FEE1
:1052200090280020024B034AC3F8C420704700BFF7
:105230009028002084010020024B034AC3F8C420B8
:10524000704700BF902800206801002070B5054617
:10525000F8F770FE0446F8F773FE81B2204611F0AD
:10526000EDFC40B1064BD3F8C43001461B6828461C
:10527000BDE87040184740F696213220F7F766FEE9
:1052800090280020024BD3F8C4305B68184700BF59
:105290009028002010B50D4C00F06CFC94F87C3088
:1052A0005BB90B4A0023A4F8BA300121937084F84B
:1052B0007010BDE8104002F08DBB0AF0E7FF09F066
:1052C000B5FC002384F87C30EBE700BF9028002079
:1052D0004A290020014B83F84C0070479028002099
:1052E00010F0010316D00C4A012382F8BD300221D0
:1052F000820706D5084A1A444FF0020C0B4682F882
:10530000BDC0020704D5044A1344082183F8BD1028
:10531000002070470121EBE790280020014B83F823
:10532000570070479028002010B5124C94F8443074
:10533000A3F1020CBCF1010F08D913B1023B18BF55
:105340000123BDE81040184605F094B80028F5D1B7
:1053500011F0FD0F14BF01200020114613F056FC80
:10536000082801D0012010BD94F84430002BE5D16D
:10537000E7E700BF90280020044B93F8443013F077
:10538000FD0F14BF0120002005F074B89028002004
:10539000014B83F8440070479028002038B5234C17
:1053A00094F8443013F0FD0F14BF0120002004F1E5
:1053B000460184F8450005F045F894F84430023B76
:1053C000DBB2012B94BF0123002384F87D3000D988
:1053D00038BD05F0BBFA054615F040FE6B015B1BBE
:1053E0004FEAD56262F10002520242EAD3525B02F6
:1053F0005B1942F1000C4FEA8C1E9A014EEA936E43
:10540000D31A6EEB0C025B1942F100021B1842EB3F
:1054100001010020C4E9283105F060FB0028D7D144
:1054200040F654313220F7F791FD00BF902800205C
:10543000002810B50C4C0CBF0123002384F84D301C
:105440004FF0080384F8560084F87B300AD111F03D
:10545000FD0F18BF0120114608BF002013F0D6FB36
:1054600084F87B00002010BD9028002008B5A1B171
:105470000C4B83F85A000A68C3F85B201A6D8888C1
:1054800093F84510A3F85F005172D3F84610C2F8A4
:105490000A10B3F84A30D38108BD40F67331322088
:1054A000F7F754FD90280020034B032883F854009D
:1054B00008BF19650020704790280020024B83F830
:1054C0007E000020704700BF90280020024B83F828
:1054D0007F000020704700BF902800200D4A92F8FE
:1054E0005430032B0ED0013B012B01D90020704713
:1054F00092F8550000F0FD00A0F10100B0FA80F034
:105500004009704792F85600A0F10100B0FA80F00F
:105510004009704790280020014B93F854007047D1
:105520009028002010B5104C94F869300BB9616ECA
:1055300091B994F87C303BB90C4B0020A4F8BA0028
:10554000987084F8700010BD0AF0A0FE09F06EFBA0
:10555000002384F87C30EFE794F8680003F0FF0242
:105560000BF050FEE5E700BF902800204A290020FC
:1055700008B5024813F0BCF8002008BD142900202B
:1055800000B50C4B93F85420032A0DD04FF0000CBB
:10559000E64683F83FE0084908485DF804EBA3F8C5
:1055A00040C0022214F080B91A6D4FF0010EB2F81B
:1055B00000C0EEE79028002019330100C628002023
:1055C00010B5027812F0010C43D04178234B032927
:1055D00008BF002483F854104FF0010108BF1C6578
:1055E00083F8BD104FF0020E94070FD590F802C05B
:1055F00083F854C0BCF1030F194408BF0024F446DB
:105600004FF0020E08BF1C6581F8BDE052070BD5B4
:10561000C27883F85420032A08BF00219C4408BFA5
:10562000196508218CF8BD10027983F8442042796D
:1056300083F8552012F0FD0F0CBF0122002283F8E1
:105640004D20827983F84C20C27983F857200020BE
:1056500010BD024B4FF0010E6146C5E790280020B7
:10566000004870474829002010B50F4C94F870305E
:10567000032B13D1023801280BD839B90B4A002368
:10568000A4F8BA30937084F8703010BD00F072FA4C
:10569000F4E740F62F413220F7F758FC40F621415D
:1056A0003220F7F753FC00BF902800204A29002041
:1056B0000A4B5A6E7AB1FF22002083F8692058669F
:1056C00093F868C0064983F86900012202FA0CF2D7
:1056D000C1F8082570470C20704700BF90280020B3
:1056E00000F00140034B93F8AB00003818BF0120D5
:1056F000704700BF902800202DE9F04F012A8DB09F
:1057000005460C4608BFA0F10905F8F713FC07464B
:1057100011F0FEFA0646002800F04081014601AA79
:10572000384611F003FB8046F8F70AFC80B240458A
:1057300040F02F81019802A900F0E6FE304611F0FA
:10574000FBFA854240F02081D5F81A10287FD5F861
:105750001220D5F81630D5F81E60C4F80B10D5F815
:105760002A10C4F80320C4F80730D5F82220D5F851
:105770002630C4F81B10C10604F10308C4F80F60FA
:10578000C4F81320C4F817301AD5420740F1E0805E
:105790000023E3720423237004F02CFC814680BBB9
:1057A000384611F0CBFA002800F009810021384674
:1057B00011F0E8F9864B00225A700DB0BDE8F08F69
:1057C000834E3378002B40F08F8095F82D30242BBA
:1057D00040F288800023E3724FF00109637B03F0FD
:1057E0006002202A00F0A980002333700423237074
:1057F00004F000FC28B9B9F1000FD1D10DB0BDE81B
:10580000F08F2378042B40F0CE8094F80DA01AF08E
:10581000100F00F0D0806E4ED4F80300D8F80410BA
:10582000D8F80820D8F80C3094F80BB0351D0FC507
:10583000D8F81000D8F81410D8F8182007C504F1CB
:105840001F015A4606F120000FF09AF91AF00401E0
:105850001DD0F37DFE2B1AD12373B38BA4F8113026
:10586000737BE3743379E37001232371737963717C
:105870007389B069D6F8062063811123C4F80D003E
:10588000C4F806202370B9F1000FB7D088E7514B58
:1058900032799B8863810BF10A0313FB02F3E270F8
:1058A000023372796370627104EB0B03D6F8062041
:1058B000707BC4F80620032284F80CB02270587361
:1058C0001AF008002ED004232371BBF11F0F6ED8ED
:1058D00041495A4604F10D000FF052F9B9F1000F99
:1058E0008CD05DE7012333709DF80830022B3FF424
:1058F00071AF73780198E52204F11F0113F0DAFD0E
:105900007378E07218447070019813F0CBFD7378CF
:10591000834234D0637B012262F3461363734FF0FA
:1059200000095BE70AF00303032B21D0E9B9022B3E
:1059300028D0002B48D12271C7E73278012A19D02C
:10594000022A0FD0002A7FF451AF012333704DE7B4
:105950009DF8185005992A4604F11F000FF010F920
:10596000E57217E70323337040E701232371ACE7A7
:105970002071AAE79B07F5D50223337036E74FF075
:1059800001092BE72371A0E740F2DF113320F7F77D
:10599000DDFA4FF4EA713320F7F7D8FA4FF4E571E6
:1059A0003320F7F7D3FA50213320F7F7CFFAA121AC
:1059B0003320F7F7CBFA51213320F7F7C7FA40F23B
:1059C0001D213320F7F7C2FA9E213320F7F7BEFAE4
:1059D000582900205E290020782900200122FFF7A5
:1059E0008BBE00BF0022FFF787BE00BF00B583B0AB
:1059F000F8F7A0FA0DF1020201A911F0B3F901982C
:105A000011F09AF990F82500FF3818BF012003B073
:105A10005DF804FB00B583B0F8F78CFA0DF10202D3
:105A200001A911F09FF9019811F086F90023C0F83F
:105A30001A3090F81CC0134AC0F812304FF0010E13
:105A4000FF216EF3461C4FF07F0EC0F81E30C0F8E9
:105A50002230C0F82A30C0F8163080F82CE0C0F8A8
:105A6000263080F82010C17480F8251080F81CC002
:105A70001364A2F84430137082F8463003B05DF826
:105A800004FB00BF5829002000B583B0F8F752FA94
:105A90000DF1020201A911F065F9019811F04CF91C
:105AA0000023C0F81A3090F81CC01149C0F8123019
:105AB0004FF0010EFF226EF3461C4FF07F0EC0F830
:105AC0001E30C0F82230C0F82A30C0F8163080F8F6
:105AD0002CE0C0F8263080F82020C27480F8252001
:105AE00080F81CC00B64A1F8443003B05DF804FBDF
:105AF0005829002070B582B0F8F71CFA0DF10202A7
:105B000001A9044611F02EF9019811F015F9C67F8C
:105B1000EEB90546204611F058F8012815D0F8F7DF
:105B20000FFA012281B2204611F0B2F8C8B1204626
:105B300011F04BF880B10D492E720622284613F061
:105B4000B3FE0B4B0022A3F8442002B070BD2046E8
:105B500011F03BF80028F4D140F2E2213320F7F7AE
:105B6000F5F940F2DE213320F7F7F0F9E5590100AD
:105B700058290020F0B583B0F8F7DCF90DF10202E6
:105B800001A911F0EFF8019811F0D6F8C37FD3B155
:105B9000124D2C6C94B1237F95F84670022262F36B
:105BA0004613237700260E4926720622204613F05C
:105BB0007BFE57B900232B6485F8463003B0BDE85F
:105BC000F040FFF797BF03B0F0BD064966740622A8
:105BD00004F1090013F068FEECE700BF582900202B
:105BE000E5590100DD5901002DE9F04F83B00D4664
:105BF00090461F469DF830909DF834A09DF938B02E
:105C00000646F8F797F9044610F0DFFF012822D086
:105C100020460DF1020201A911F0A4F8019811F03B
:105C20008BF80023C0F81230C0F81630C0F81A30D4
:105C3000C0F81E30C0F82230C0F82630C0F82A3034
:105C4000012304468374062D7BD8DFE805F0074561
:105C5000587A7A7A5D0003B0BDE8F08F037F23F0B5
:105C6000130343F013030377B9F1080F04F114028F
:105C70003DD0484604F1130104F06EFE00286AD0BE
:105C8000E37C43F00203E374227F84F81BB001231A
:105C9000E38352074FF0FF0384F820303BD484F8AD
:105CA00025307F2384F82C3084F82DA0F8F742F9B2
:105CB0000546F8F745F9012281B2284610F0E8FFC1
:105CC000002843D02649002306222046237203B031
